:020000040800F2
:1000000000200010553B0308B9F60208C15D000846
:10001000B5F60208B1F60208ADF6020800000000CD
:10002000000000000000000000000000A9F6020827
:10003000A5F6020800000000A1F60208817600087B
:10004000BD3B0308BD3B0308BD3B0308BD3B0308A4
:10005000BD3B0308BD3B0308254700086548000871
:1000600025480008E5470008A5470008E9150008ED
:10007000D9150008C9150008B9150008A915000808
:100080009515000881150008BD3B0308BD3B03081A
:1000900061FB0208BD3B0308BD3B03086547000840
:1000A000D96D0008296E0008BD3B0308396E0008B1
:1000B000196E0008096E0008BD3B0308BD3B03082C
:1000C000BD3B0308BD3B0308BD3B0308BD3B030824
:1000D000BD3B0308897700080D770008BD3B030886
:1000E000E7460008BD3B030891F60208BD3B030844
:1000F000E96D0008BD3B0308F96D0008BD3B03082E
:10010000000000000000000000000000BD3B0308EC
:10011000BD3B0308BD3B03089D3F0208813F020829
:100120006D1500085915000845150008311500081F
:100130001D150008BD3B0308000000000000000082
:10014000BD3B0308BD3B0308BD3B030800000000A6
:10015000000000000000000000000000000000009F
:100160000000000000000000BD3B0308BD3B030889
:10017000BD3B03080000000000000000000000007C
:0801800000000000BD3B030874
:10018800F0B58F7A8D79CC7ACE790A7C4B7C9FED4D
:100198005B4A4FEA072C0CF4706C45EA0C053F01EA
:1001A80007F4706E03EE905A4FEA042C0D7A24017E
:1001B80004F470670CF4706C46EA0E0404EE904A7E
:1001C80045EA0C0405EE104A4C7A16023C4312012B
:1001D80002F4706505EE904A4A7B0C7B06F4706663
:1001E80034432A431D021B0106EE104A06EE902AEC
:1001F80003F470648A7BCB7B05F470652A43234340
:1002080007EE102A07EE903AB8EEC55AF8EEE33A30
:10021800F8EEE55A25EE045AF8EEE44AB8EEC66A56
:10022800F8EEE66AB8EEC77AF8EEE77A65EE845A31
:1002380063EE843A64EE844A26EE046A66EE846AC3
:1002480027EE047A67EE847ABCEEC55ABCEEE34A20
:10025800FCEEE55A87B015EE102AFCEEE44ABCEE37
:10026800C66AFCEEE66ABCEEC77AFCEEE77A15EEE3
:10027800907A8DED014ABDF80410ADF80C2017EE08
:10028800104A17EE902A14EE90EA16EE106A16EE4F
:10029800905AADF80E700DF10A07ADF81440ADF89C
:1002A8001620ADF808100B46ADF80AE0ADF810605E
:1002B800ADF812503A4606AC01E032F8023BA3F51D
:1002C8004873B3F5AF6F0CD8A242F6D1831E0E3037
:1002D80001E037F8021B23F8021F9842F9D107B052
:1002E800F0BD074B1B78162BF9D1064A064913882F
:1002F80001339BB213800B8007B0F0BDABAA2A3F35
:10030800D4460020581D0020D8460020044A93787F
:100318003F2B03D8D118013308719370704700BF81
:10032800581D0020024B00229A7083F84420704721
:10033800581D0020012380F84530704790F8203080
:1003480033B1012B03D14FF40063838270477047A8
:100358004FF480638382704770B40468037B22681B
:10036800022101FA03F31A4213D042690A495C20B8
:1003780000FB02124FF6FE7650685289C568006885
:10038800296831402960C168D24392B20A40C260EC
:10039800636070BC704700BF4858002030B40A4BF7
:1003A8001D7875B1094B002003EBC5051A689988BB
:1003B8005062D4682143D160083323F8040CAB425F
:1003C800F4D130BC704700BF285B00202C5B0020B4
:1003D80010B40268047B11680223A340194209D0B3
:1003E8000649406800240C7001684FF6FE742140ED
:1003F800016053605DF8044B704700BF623F002006
:1004080010B490E80600047B40690223A3404B60C7
:1004180013685DF8044B4FF6FE710B40136007F04C
:10042800EDB900BF70B5202003F0E7F82D4B186038
:1004380018B1272200238271C371002103F071FBD8
:10044800262003F0DAF8284B186018B1052200239B
:100458008271C37128F022FD2B2003F0CEF8234CC3
:10046800A06418B1272200238271C37128F016FDF9
:10047800A06C1F4D03F016FD212003F0BEF8286084
:1004880018B1272200238271C37128F007FD2220AA
:1004980003F0B3F8174E306018B127220023827199
:1004A800C37128F0FBFC3D2003F0A7F8E06418B105
:1004B800272200238271C37128F04CFDE06C03F001
:1004C8001BFD0D4B84F8500030681B6803F0EAFCF4
:1004D800286803F0E2FC094B1A780AB903221A705B
:1004E80070BD00BF801E0020C01E0020581D0020C7
:1004F800281F0020341F00209C550020123900209E
:1005080038B50E4CE36C0546ABB1184603F0F4FC65
:10051800024694F850000A4B40B9187884F85020E5
:1005280018B115B1002228461A7038BD002AF4D136
:1005380001211970F2E7024B1878F1E7581D0020E5
:10054800F82C002023F04CBC38B5184C184A94F805
:10055800513012781844C0B290420D4684F85100C8
:1005680005D3801AC0B29042FBD284F851003620DD
:1005780023F050FC0021232094F85140FFF7E2FFBC
:1005880000212420FFF7DEFF00212520FFF7DAFFF6
:10059800084B23440A201979FFF7D4FF05B938BD61
:1005A8003A20BDE8384023F035BC00BF581D002074
:1005B800691E0020881E002038B50F4C0546E178DA
:1005C8000C20FFF7BFFF08211820FFF7BBFF85B9F4
:1005D80061780920FFF7B6FF0D210720FFF7B2FF6A
:1005E80016211920FFF7AEFF0A20BDE8384006F0B3
:1005F800A5BF0321EDE700BF881E002008B540F223
:10060800E93300E09BB10289013B12F0020F9BB273
:10061800F8D0017340F2E93300E043B10289013BAD
:1006280012F0010F9BB2F8D0007BC0B208BD04F0F5
:100638007DF9C0B208BD00BF38B530200D4C0E4D55
:1006480023F0E8FB4FF47A7006F01EFF236AA28CB1
:100658001A8528468E21FFF7D1FF2846FF21FFF78C
:10066800CDFF236AA28C9A61A0F1C400B0FA80F091
:10067800400938BDDC5000200030014038B5094C35
:10068800094D236AA28C1A8540F080012846FFF79D
:10069800B5FF2846FF21FFF7B1FF236AA28C9A61B4
:1006A80038BD00BFDC500020003001402DE9F0418A
:1006B800114F04463B200D4623F0ACFB3B6ABA8C35
:1006C8001A857F210D48FFF799FF80465DB1013DEE
:1006D8000A4E54FA85F5013C14F8011F3046FFF71D
:1006E8008DFFAC42F8D13B6ABA8C9A61352023F071
:1006F80091FB4046BDE8F081DC500020003001400D
:100708002DE9F0410F4F3B6ABA8C1A8504460D4615
:100718000D48FF21FFF772FF804665B1013D0A4E83
:1007280054FA85F5013CFF213046FFF767FF04F8CE
:10073800010FAC42F7D13B6ABA8C9A614046BDE8DA
:10074800F08100BFDC5000200030014001382DE965
:10075800F8430C4604281FD8DFE800F0390377A8CF
:100768002000A84DA84A95F95830696D7D2BC4BF63
:10077800822385F8583013685B1A322B00F22B81DC
:10078800A24B186803F0B8FB30B1FB20FFF776FFE7
:1007980010F07F0640F0E280BDE8F8839C4B1B78A0
:1007A800002B00F025819B4D2824286803F07AFB54
:1007B800322006F0C3FE286803F06FFB322006F0F3
:1007C800BDFE631E13F0FF04EFD1BDE8F8830120DE
:1007D800FFF796FE18B98E4B1B78002BDCD08D4B9B
:1007E800186803F05FFB14211920FFF7ABFE864A57
:1007F800844B12685A65822211460C2083F85820CF
:10080800FFF7A0FE0C210720FFF79CFE0821182007
:10081800FFF798FE362023F0FDFA00212320FFF78A
:1008280091FE00212420FFF78DFE00212520FFF7EF
:1008380089FE00210A20FFF785FE3A2023F0EAFA14
:100848003420BDE8F84323F0E5BA704B186803F08C
:1008580053FB0028A0D0FB20FFF710FF10F07F0506
:100868009AD0294625442046FFF74AFF15F9013C4E
:10087800002B91DAA378012B8ED16579002D8BD1CD
:10088800634AE178237951706FF004009370001B7C
:10089800611D04F10A0643182B4411F8015F134443
:1008A800B1421D713FF478AF6579F4E7554D95F87D
:1008B8005930782B04D93620BDE8F84323F0AABA7A
:1008C800524B186803F018FB00283FF465AFFB2073
:1008D800FFF7D4FE10F07F063FF45EAF31462046A6
:1008E800FFF70EFFA31913F9013C002BBFF654AF15
:1008F800A378012B7FF450AF454AE17853789942A9
:100908007FF44AAF2179937899427FF445AF6179B2
:1009180095F859308B420F467FF43EAFF31E2344BF
:1009280004F10508002004E005288EF804C063D00F
:10093800617918F801CF93F8009002EB000EE145B9
:10094800C6B28E4400F1010002D0BCF1000FEBD119
:100958002C2FE9D9304B31441970ACE73146264485
:100968002046FFF7CDFE16F8013C1A067FF514AFB6
:10097800A478012C7FF410AF03F07F03312B3FF6EE
:100988000BAF234B95F85820DA70362023F042FA43
:1009980000212320FFF7D6FD00212420FFF7D2FDF8
:1009A80000212520FFF7CEFD00210A20FFF7CAFD10
:1009B8003A2023F02FFA142006F066FD342023F0A5
:1009C80029FA154A05230021117085F85930204667
:1009D800BDE8F843F0E595F8583012686A650533C4
:1009E800DBB219460C2085F85830FFF7ABFDC7E697
:1009F800BDE8F84305F016BA053785F85970BDE823
:100A0800F88300BF581D00209C550020801E002040
:100A1800881E0020C01E0020691E00202DE9F84F06
:100A2800074606F0E5FCCF4D064695F85A0009281A
:100A38002CD8DFE810F02F00EB00EB00EB00EB0008
:100A4800EB00F20006010A002200DFF84C83C64BD7
:100A5800186803F051FA002840F04081EA6D42F22C
:100A68002833044603FB02F3D8F80020B61A9E4246
:100A780000F3FD802046BDE8F88F06F0B9FC6B6EE8
:100A880040F26352C01A904200F236810024204698
:100A9800BDE8F88FB54BB64A1B6812689B1A0A2B3B
:100AA800F4D9FFF7C9FD01210220FFF74BFD0C2106
:100AB8001720FFF747FD18210846FFF743FD1921C6
:100AC8000620FFF73FFD05210820FFF73BFDFF212A
:100AD8003E20FFF737FD08210B20FFF733FD0021EB
:100AE8000C20FFF72FFD5C210D20FFF72BFD762151
:100AF8000E20FFF727FD27210F20FFF723FDAA214E
:100B08001020FFF71FFD39211120FFF71BFD1121D0
:100B18001220FFF717FD23211320FFF713FD7A2179
:100B28001420FFF70FFD42211520FFF70BFD1621BA
:100B38001920FFF707FD6C211A20FFF703FD032199
:100B48001B20FFF7FFFC40211C20FFF7FBFC912135
:100B58001D20FFF7F7FC56212120FFF7F3FC102199
:100B68002220FFF7EFFCA9212320FFF7EBFC0A2145
:100B78002420FFF7E7FC00212520FFF7E3FC1121E3
:100B88002620FFF7DFFC59212920FFF7DBFC88210D
:100B98002C20FFF7D7FC31212D20FFF7D3FC0B21A8
:100BA8002E20FFF7CFFC07210320FFF7CBFC002105
:100BB8000920FFF7C7FC362023F02CF90421072071
:100BC800FFF7C0FC00210C20FFF7BCFC00243620F6
:100BD80023F020F9E1B20A20FFF7B4FC332023F018
:100BE80019F94FF4617006F04FFC2320FFF746FD1A
:100BF8002420FFF743FD01342520FFF73FFDFF2C9C
:100C0800E5D1012385F85A30002433E7394600241A
:100C1800FFF79CFD2046BDE8F88F564B2F22002099
:100C28001A70FFF7C9FC01210846072385F85A30D6
:100C38000124FFF789FC342023F0ECF82046BDE8B6
:100C4800F88FDFF8548108230020C8F8006085F881
:100C58005A30FFF755FC00283FF4F9AE0024322340
:100C6800C8F800402C6685F85A40EB6502E7424B0D
:100C7800186803F012F9EB6D012B00F08F8095F8DE
:100C880083305A1C13F0010F3C4B85F883201868F9
:100C98004FD103F007F93A4B1B78032B13D1394F87
:100CA800394E3A78394836F812E00368511C01F099
:100CB8000F01A3EB0E0339700027354926F812708F
:100CC8001A0903600A8001210D20FFF73DFC34203A
:100CD80023F0A0F8072385F85A30CBE6FB20FFF76E
:100CE800CDFC00F07F00132826D8EA6D42F22833A5
:100CF80003FB02F30024B7E6362023F08BF825F037
:100D0800D5F93A2023F086F81B4B186803F0CAF887
:100D1800362023F07FF895F86C101E480131C9B2CF
:100D2800FFF7C4FC1C4A0823166085F85A300224D1
:100D3800A0E603F0B2F8AEE714213846FFF7E0FC6E
:100D480097F91330002BD0DA97F800A000244FF061
:100D5800010BBAF1110F2C66C5F85CB046D042F20F
:100D6800283381E6581D0020801E00209C55002055
:100D7800B81F0020691E0020281F0020C01E002068
:100D880012390020133900201839002014390020A6
:100D9800343F0020C41D0020641E00202B6E012B50
:100DA80010D995F8823013F0010F544B186810D001
:100DB80003F078F895F882202B6E0132642B85F8C1
:100DC800822009D801210B4408462B66FFF7BCFB9B
:100DD8007DE703F062F8EDE7494A12783221032AE9
:100DE800E965EFD1474A00211180EBE7DFF82C9144
:100DF8007A7899F801309A42B1D1BA7899F80230E4
:100E08009A42ACD1404B186803F04CF85946584602
:100E1800FFF79AFBFB7803F00303022B0ED0342074
:100E280022F0F8FF072385F85A30EA6DC8F8006009
:100E380042F2283303FB02F3022415E606F0D8FA3F
:100E48006866B87C32F0B8FE304A314B107B517C72
:100E580033F810202F4833F811303979078895F87E
:100E6800800099F8014085F87170C3F30B1388422C
:100E780085F87030C2F30B120EBF95F8443095F820
:100E8800813085F8443085F86F2008BF85F88130B7
:100E980099F8022085F86D404B1C03F01F0385F874
:100EA8006E20AC7895F844201B4F85F8803085F883
:100EB800681085F86CA0002302F10109944205EB43
:100EC800020C07EB030ED8B209F03F0203F101034D
:100ED80009D09CF804008EF808000A2BECD185F89C
:100EE8004420184601E085F84440092385F872003B
:100EF80085F8731085F85A3097E700BF341F002033
:100F080012390020343F0020C01E00201455002054
:100F180034550020061F0020C41D0020881E002014
:100F2800F8B584894FF6FF764FF47A742BB311B372
:100F38000F78013101E0B44217D00589013CAD07B3
:100F4800A4B2F8D507734FF47A7402E0BCB2B44285
:100F58000BD00589ED0704F1FF37F7D5057BEDB216
:100F68000AB115700132013BE0E703F0DFFC003005
:100F780018BF0120F8BDFF27DFE70120F8BD00BF3B
:100F8800F0B55B4B5B4A97B01968914200AF00F02F
:100F9800A3805949594A00234FF47000C1F88800CA
:100FA8003B607B60136843F48033136003E03B6865
:100FB800B3F5A04F09D0136803F400337B603B6896
:100FC80001333B607B68002BF1D04C4B1B6813F45A
:100FD800003318BF01237B607B68012B52D0464C3D
:100FE800464B474AE260474A596A11605A6A42F0DA
:100FF80080725A625A6942F4FC025A61002503223F
:1010080007F10801012341F6FF764FF09040FD609B
:10101800BE603A73BB7329F06FFA4FF6FF7307F19E
:1010280008013948BB6029F067FA07F10801374819
:10103800374E29F061FA07F10801364829F05CFAC1
:1010480007F10801344829F057FA07F10801334835
:1010580029F052FA07F1080029F0A8FABB683049CC
:10106800304AA1FB031330499B0CF0204FF0070EC8
:101078005C370B60566084F823009560C2F800E086
:10108800BD46F0BD294A1D4B122111605A685A60AD
:101098005A685A605A6842F480625A605A6822F460
:1010A8007C125A605A6842F4E8125A601A6842F090
:1010B80080721A601A689201FCD559680F4A21F0AB
:1010C80003015960596841F002015960536803F0FF
:1010D8000C03082BFAD182E700221A6062B6144B7F
:1010E8001B6883F30888134B1B689847FEE700BF0B
:1010F800FC9F0020EFBEADDE00ED00E000100240D6
:101108000005FA058C5B0020000400480008004830
:101118003F190100000C0048001000480014004866
:1011280083DE1B4310E000E0A055002000200240B1
:1011380000D8FF1F04D8FF1F064A002351688142C8
:1011480002F11C0204D001330C2BF7D100207047A8
:10115800D8B27047E000002070B50F4C0F4DC0EBBF
:10116800C00004EB8004686926693043686182B076
:101178009209667BA1600025012101A863618DF8B1
:1011880004608DF805208DF806508DF8071029F0B9
:101198007DF902B070BD00BFE000002000100240E1
:1011A800074BC0EBC00030B403EB8000054C056969
:1011B80063692B4363610176427630BC704700BF98
:1011C800E0000020001002402DE9F04F554C54F883
:1011D800204083B0002C60D0A56D1F469046524B2E
:1011E8006A682265A160236004F15E014FF4807390
:1011F80004F5AF726161A261E36023610646287E4F
:1012080027F02EFEE86858B1FFF796FF721CD2B29D
:101218000C21FFF7C5FF236DEA6862632433E3649A
:10122800A86890B1FFF788FF721C8146D2B20B21E3
:10123800FFF7B6FF2346EA7E3C494846FFF78CFF96
:10124800236DAA68A2632833A36494F85D0002F0B2
:10125800D4F9814694F85C0002F0CFF93A07824647
:1012680095F819B01DD5B9F1000F1AD017F0110F64
:101278004FF00B0306F1010614BF4E213E2189F8F9
:10128800063089F807605A46484602F079FAFB07A3
:1012980043D5636B6BB3A36B5BB3204603B0BDE868
:1012A800F08F17F0010F0CBF2E274E2718F0020FF2
:1012B8000DD0B9F1000F0AD00B22731C89F8062053
:1012C80089F8073048465A46394602F059FA18F064
:1012D800010FDED0BAF1000FDBD001360C238AF8FB
:1012E80007605A4639468AF80630504602F048FAEE
:1012F800CFE72B7FAA7E8DF804209B0900210122CD
:1013080001A88DF805308DF806108DF8072029F012
:10131800BDF8204603B0BDE8F08F484602F0BDFD99
:10132800B7E700BF142C0020D050030809040008B8
:1013380000B97047F0B595B0054628F0B3F96C4E82
:10134800C368026832600446002B00F0C480284657
:1013580002F053F9674BC3F8840018B1292200231F
:101368008271C371227A644D2E2102F009FA306825
:1013780005F0CEFE27F074FD3068604A038823F03C
:1013880001031B041B0C038014A91E232B800127B7
:101398000F230025138021F84C7D2D230293ADF8EF
:1013A8000C50ADF80650ADF80E5028F029F9E37945
:1013B800ADF8145060229907ADF816500695ADF8AF
:1013C8001C50ADF81E50ADF82050ADF822500492D4
:1013D80000F1838013F0010F0CBF002202224FF4AA
:1013E8008073ADF81470ADF81C20ADF820300023E0
:1013F80004AA61793068069305F0EEFA61793068DD
:101408003F4F28F0DDF833685A6C42F400425A64C2
:101418001A8892B242F080021A80E2796079196AD9
:1014280092074CBF04220122824021EA020119627C
:10143800196A0A431A621A8892B242F001021A80A3
:10144800207C00222921FFF7ABFE2E49207C0023B7
:101458006022FFF781FEE068386028F083FF386873
:1014680003684FF6FE721340036028F07BFF09A85B
:1014780028F04AFF33686279234938680A9134337F
:101488001344099380221023002509A940F22A3E1B
:101498000E920B934FF400724FF400530D95109574
:1014A800139511950F921293ADF830E028F03AFF9A
:1014B800627933680C2A98BF1449D86898BF31F804
:1014C80012503A6812490543DD601368012043F061
:1014D80002031360087015B0F0BD13F0010F0CBFC4
:1014E8002A4608220423ADF81E20ADF816307EE700
:1014F80008540020581D0020FE530020FC530020F3
:1015080004540020D9030008F44000208473030821
:10151800005400200348D0F83C3113B100F59A700C
:1015280018477047E00000200348D0F8203113B175
:1015380000F58C7018477047E00000200348D0F889
:1015480004310BB1FC301847704700BFE0000020A1
:101558000348D0F8E8300BB1E0301847704700BFB7
:10156800E00000200348D0F8CC300BB1C430184755
:10157800704700BFE00000200348D0F8B0300BB13E
:10158800A8301847704700BFE00000200348D0F893
:1015980094300BB18C301847704700BFE000002032
:1015A8000248836F0BB1703018477047E000002085
:1015B8000248C36D0BB1543018477047E000002053
:1015C8000248036C0BB1383018477047E000002020
:1015D8000248436A0BB11C3018477047E0000020EE
:1015E8000248836803B11847704700BFE000002035
:1015F800028822F040021204120C0280028822F0B3
:1016080038031B041B0C59B141F48071002991FA6D
:10161800A1F2B2FA82F108BF4FF0FF310139C900D7
:101628000B439BB2038003889BB243F040030380C3
:10163800704700BFF8B505015D4C5E4A6359934297
:10164800064604EB050100F085805B4A934200F0F2
:1016580081806719387A27F003FC3B7A03F01F0171
:101668005B090122022B02FA01F276D0032B79D012
:10167800012B67D063190136187901F0BEFFF6B265
:10168800074610B11223C67183716319587901F0A6
:10169800B4FF10B11323C67183716319987901F0EF
:1016A800ACFF10B11423C671837166190E21F2794B
:1016B800384602F065F8707901F09FFFF2790E2143
:1016C80002F05EF8B07901F098FFF2790E2102F08D
:1016D80057F86359384A934254D0364A93425CD0FB
:1016E800364A934243D02C44227B002A2FD1012032
:1016F80002249A8822F480521204120C9A80998843
:1017080089B241F4805199801A8802F4415242F416
:101718004572024322431A809A8822F470621204A6
:10172800120C42F4E0629A809A8B22F4006212044E
:10173800120C07219A8319821A8892B242F0400249
:101748001A80F8BD1E4B996A0A439A6292E70020F4
:101758000446CEE701230B737BE7194BD9680A438C
:10176800DA6087E7164B19690A431A6182E702F5BE
:10177800EA32116941F400411161116921F4004113
:101788001161B0E702F56042D16841F48051D1603F
:10179800D16821F48051D160A5E702F5EC321169D6
:1017A80041F480411161116921F4804111619AE786
:1017B800382C00200038004000300140003C004038
:1017C80000100240F0B5424C059D00EB800004EB90
:1017D80080046468002C79D03E4E49004FF42040C4
:1017E800CFB2C6F88800A169090459D46068DFF847
:1017F800F0E047F4903100EA0E0001434FF4204036
:101808006160C6F8880003E0411E00284CD00846F5
:10181800A1698907F8D54FF42040A262C6F888006C
:1018280003E0421E00283FD01046A2695206F8D5B0
:10183800294A6168DFF8A8E0C6F8880042EA03424E
:10184800174301EA0E0217436760C3B1013BDBB2DD
:1018580001332B44A0694FF4204210F0040002F138
:10186800FF3207D1511C29D0A06910F0040002F101
:10187800FF32F7D0626A05F8012B9D42EAD14FF496
:101888002040C6F8880002E0431E68B11846A369E4
:101898009B06F9D52023C6F88800E3610120F0BD36
:1018A800411E08B108469EE70C4A138801339BB2D3
:1018B8004FF0FF311380C6F88810F0BD0749C6F80D
:1018C80088200B8801339BB20B80F0BD2046F0BD09
:1018D8003C550020581D002000240002082D00203F
:1018E800009800FCF0B5037C012B85B0044663D05A
:1018F800022B67D1836913B11A689B8813856069C5
:1019080040F2E93301E0002B6CD00289013B12F070
:10191800020F9BB2F7D0C323037340F2E93301E00F
:10192800002B5FD00289013B12F0010F9BB2F7D068
:10193800037B60694FF0060E838902AE4FF47A7319
:101948004FF6FF71FF2703E0013B9BB28B423CD06F
:1019580002899507F8D507734FF47A7302E0ABB2A2
:101968008B4232D00289D20703F1FF35F7D5027BCB
:10197800D2B20EB132700136BEF1010EE8D1A369C0
:1019880013B11A689B8893619DF80C009DF8086054
:101998009DF809109DF80A509DF80B209DF80D3010
:1019A80041EA062143EA002342EA05220120218771
:1019B8006287A38705B0F0BD90F91400431C01D0DD
:1019C800022805DD002005B0F0BD02F0AFFFD6E724
:1019D80002AB617D009343220623FFF7F3FE002844
:1019E800D2D1EFE702F0A2FFA3E700BFF0B5037A78
:1019F800012B85B0044663D0022B67D1036913B16C
:101A08001A689B881385E06840F2E93301E0002BEF
:101A18006CD00289013B12F0020F9BB2F7D0BB23B6
:101A2800037340F2E93301E0002B5FD00289013BE8
:101A380012F0010F9BB2F7D0037BE0684FF0060E5F
:101A4800838902AE4FF47A734FF6FF71FF2703E0E4
:101A5800013B9BB28B423CD002899507F8D50773AE
:101A68004FF47A7302E0ABB28B4232D00289D207CC
:101A780003F1FF35F7D5027BD2B20EB132700136D1
:101A8800BEF1010EE8D1236913B11A689B889361EE
:101A98009DF80C009DF808609DF809109DF80A5003
:101AA8009DF80B209DF80D3041EA062143EA0023FA
:101AB80042EA05220120E1822283638305B0F0BD5A
:101AC80090F90C00431C01D0022805DD002005B068
:101AD800F0BD02F02BFFD6E702AB617B00933B22FF
:101AE8000623FFF76FFE0028D2D1EFE702F01EFFB2
:101AF800A3E700BFB0F1FF3F5CD002285ADCF0B486
:101B0800364C00EB800004EB80004468002C62D067
:101B1800334E49004FF42040CDB2C6F88800A16981
:101B2800090449D460682F4F45F08071384041F46A
:101B3800903101434FF420406160C6F8880003E00B
:101B4800411E00283CD00846A1698F07F8D54FF4FC
:101B58002040A262C6F8880002E0421E80B3104608
:101B6800A2691106F9D562681E4945F0007545F469
:101B780080350A4015434FF420406560C6F8880058
:101B880002E0421EE0B11046A2699207F9D54FF46F
:101B98002040A362C6F8880002E0431E80B11846C0
:101BA800A3699B06F9D52023C6F88800E3610120C4
:101BB800F0BC704700207047411E08B10846AEE7E8
:101BC800094A138801339BB24FF0FF311380C6F8DE
:101BD8008810F0BC70472046FBE700BF3C5500204A
:101BE800581D0020009800FC082D00202DE9F04F1A
:101BF80087B090F855300190002B40F0E483019AAB
:101C0800137C012B00F07B84022B44D1936913B120
:101C18001A689B881385019B586940F2E93302E0F2
:101C2800002B00F0E2840289013B12F0020F9BB204
:101C3800F6D06B23037340F2E93302E0002B00F087
:101C4800D4840289013B12F0010F9BB2F6D0037BCA
:101C5800019B586940F2E93302E0002B00F0C1848F
:101C68000289013B12F0020F9BB2F6D08023037366
:101C780040F2E93302E0002B00F0B3840289013B13
:101C880012F0010F9BB2F6D0037B019B9B6913B145
:101C98001A689B8893616423A94CAA4DDFF8ACA20B
:101CA800A948DFF8ACC24FF010084FF47A779E4687
:101CB800DAF80430C3F30803002B40F04E82EFF348
:101CC8001183002B40F049822168826800BF236895
:101CD8009942F9D12E6807FB06F39B1AB3FBF6F37A
:101CE80007FB013101260091DAF80430C3F3080339
:101CF800002B40F01582EFF31183002B40F0108287
:101D08002368816800BF22689342F9D1D5F800B0F2
:101D180007FB0BF2521AB2FBFBF207FB0323009AF4
:101D28009B1AB3F57A7FDFD3BEF1010EC0D1019AB9
:101D3800137C012B51D0022B58D1936913B11A6827
:101D48009B881385019B586940F2E93302E0002B18
:101D580000F060840289013B12F0020F9BB2F6D0BA
:101D68006B23037340F2E93302E0002B00F0528446
:101D78000289013B12F0010F9BB2F6D0037B019B55
:101D8800586940F2E93302E0002B00F032840289FE
:101D9800013B12F0020F9BB2F6D00323037340F20B
:101DA800E93302E0002B00F024840289013B12F0A1
:101DB800010F9BB2F6D0037B01988269002A00F0DC
:101DC8001F84136892889A61017C90F850700129E9
:101DD80000F0DF81022955D114E0164603236B2257
:101DE800717D96F91400FFF785FE337C0199012B6C
:101DF80091F8507000F0CD81022B43D18A6912B15D
:101E0800136892881A85019B40F2E932586902E00A
:101E1800002A00F019840389013A13F0020F92B2E4
:101E2800F6D01923037340F2E93202E0002A00F0E9
:101E38000B840389013A13F0010F92B2F6D0037BA9
:101E4800019B40F2E932586902E0002A00F0F98368
:101E58000389013A13F0020F92B2F6D0077340F2E9
:101E6800E93302E0002B00F0EC830289013B12F019
:101E7800010F9BB2F6D0037B019B9B6913B11A68D3
:101E88009B8893610F23DFF8C4A02F48DFF8C0C0F8
:101E98004FF010084FF47A779E46DAF80430C3F30F
:101EA8000803002B40F07382EFF31183002B40F0FE
:101EB8006E822168826800BF23689942F9D12E6832
:101EC80007FB06F39B1AB3FBF6F307FB0131012668
:101ED8000091DAF80430C3F30803002B40F03A828B
:101EE800EFF31183002B40F035822368816800BF2F
:101EF80022689342F9D1D5F800B007FB0BF2521AC9
:101F0800B2FBFBF207FB0323009A9B1AB3F57A7F17
:101F1800DFD3BEF1010EC0D101990A7C91F84E4081
:101F2800012A00F09F81022A40F0A5818B6913B134
:101F38001A689B881385019B40F2E93258690CE0C6
:101F48009C550020A055002010E000E000ED00E0C6
:101F580098550020002A00F071830389013A13F094
:101F6800020F92B2F6D01A23037340F2E93202E06C
:101F7800002A00F063830389013A13F0010F92B23B
:101F8800F6D0037B019B40F2E932586902E0002A4F
:101F980000F044830389013A13F0020F92B2F6D09D
:101FA800047340F2E93302E0002B00F03783028922
:101FB800013B12F0010F9BB2F6D0037B01988269B6
:101FC800002A00F03283136891889961027C012A03
:101FD80000F09F82022A00F05981012A00F0E28075
:101FE800022A40F0E880019B9A691AB11368918827
:101FF8001985019B586940F2E93302E0002B00F093
:10200800ED820289013B12F0020F9BB2F6D01C232D
:10201800037340F2E93302E0002B00F0DF8202890B
:10202800013B12F0010F9BB2F6D0037B019B58696C
:1020380040F2E93302E0002B00F0C0820289013B44
:1020480012F0020F9BB2F6D01823037340F2E93363
:1020580002E0002B00F0B2820289013B12F0010F6E
:102068009BB2F6D0037B01988269002A00F0AD820A
:10207800136891889961027C012A00F05481022A30
:1020880000F0A480012A00F05A81022A45D1019B60
:102098009A6912B1136892881A85019B586940F2AF
:1020A800E93302E0002B00F086820289013B12F03E
:1020B800020F9BB2F6D03823037340F2E93302E0F3
:1020C800002B00F078820289013B12F0010F9BB2CD
:1020D800F6D0037B019B586940F2E93302E0002BFC
:1020E80000F066820289013B12F0020F9BB2F6D023
:1020F8000123037340F2E93302E0002B00F0588219
:102108000289013B12F0010F9BB2F6D0037B019BC1
:102118009B6913B11A689B88936107B0BDE8F08F7B
:10212800EFF3118988F3128881680368DB0344BFE1
:10213800CCF8006081682368DCF800205FFA89F930
:1021480089F31188D5F800901A4407FB09F35B1A44
:10215800B3FBF9F307FB0233E1E5EFF3118288F3F0
:10216800128886680368D90303D50123CCF80030A8
:1021780086682368DCF80010D2B282F311882A68D6
:10218800194407FB02F39B1BB3FBF2F307FB013176
:10219800A8E501983B46417D90F914001922FFF704
:1021A800A9FC6FE6019C1C221823617D94F9140098
:1021B800FFF7A0FC227C012A00F0B580022A7FF4F8
:1021C80061AF019B9A691AB1136891881985019BBF
:1021D800586940F2E93302E0002B00F0E6810289F9
:1021E800013B12F0020F9BB2F6D03723037340F283
:1021F800E93302E0002B00F0D8810289013B12F09C
:10220800010F9BB2F6D0037B019B586940F2E9337A
:1022180002E0002B00F0B8810289013B12F0020FA6
:102228009BB2F6D00223037340F2E93302E0002B9D
:1022380000F0AA810289013B12F0010F9BB2F6D08F
:102248000199037B8A69002A00F0A58113689288A6
:102258009A61097C012972D002293FF41DAF07B0A9
:10226800BDE8F08F2346019C1A22617D94F9140081
:10227800FFF740FC227C012A00F04B81022A7FF400
:10228800ACAE019B9A691AB1136891881985019BB4
:10229800586940F2E93302E0002B00F072810289AC
:1022A800013B12F0020F9BB2F6D01B23037340F2DE
:1022B800E93302E0002B00F064810289013B12F04F
:1022C800010F9BB2F6D0037B019B586940F2E933BA
:1022D80002E0002B00F045810289013B12F0020F59
:1022E8009BB2F6D01823037340F2E93302E0002BC7
:1022F80000F037810289013B12F0010F9BB2F6D042
:10230800037B01988269002A00F032811368918862
:102318009961027C012A3FF445AF022A3FF468AE76
:10232800012A7FF44BAF019C37220223617D94F987
:102338001400FFF7DFFB227C012A7FF4A6AE019888
:102348000123417D90F914003822FFF7D3FB07B031
:10235800BDE8F08FEFF3118988F31288816803686C
:10236800DB0344BFCCF8006081682368DCF80020F8
:102378005FFA89F989F31188D5F800901A4407FBA8
:1023880009F35B1AB3FBF9F307FB0233BCE5EFF380
:10239800118288F3128886680368D90303D501235C
:1023A800CCF8003086682368DCF80010D2B282F3DB
:1023B80011882A68194407FB02F39B1BB3FBF2F34D
:1023C80007FB013183E51D09013D052D03F00F03CE
:1023D80000F2C280A34A32F8150040FA03F2D4078B
:1023E80040F1BA80012404FA03F3013B184031F0AC
:1023F80029FA9D4BDFF88C825F5D074418EBC7050F
:1024080000F0AA8020220023AA71EB7158F8370047
:10241800964A00F138439B0AD25C02F01F03520926
:10242800022A04FA03F300F01881032A00F010814D
:10243800A24200F08C80AB88049304A90024059480
:1024480028F05AF8AB88019E894AF260B3FA83F201
:10245800C2F11F02511C3FD0D1B201F0FC0303F1BD
:10246800804303F5803301F00301D3F808E08800C6
:102478004FF00F0C58F83710DFF80C820CFA00F701
:102488002EEA070706F10C0E48F822E09F60D3F801
:1024980008C0784FDFF8F4E1C1F38721814041EAB1
:1024A8000C014FF00109996009FA02FCB918CEF83D
:1024B80000C0082304A8049291F828808DF81530EC
:1024C8008DF816908DF8144023F07EFD6A4A12F8B4
:1024D8000830F02B27DCAB88B3FA83F3C3F11F0372
:1024E800581C3FF48CAB012202FA03F363490A68D3
:1024F8001343019A0B60137C012B7FF485AB1046C4
:102508008023417D90F914006B22FFF7F3FAFFF75F
:10251800C2BB019C1B221823617D94F91400FFF7AC
:10252800E9FA227C59E507EB0803F02193F83830E3
:102538008DF80C3003A803238DF80E408DF80F900A
:1025480002F808108DF80D3027F0A0FFC3E74C4AB9
:1025580051690B4353616EE7019A454BD3600123E0
:10256800C4E702F0E3F901988269002A7FF4CEAE4D
:10257800027C012A03463FF415AE022A3FF43AAD25
:1025880019E602F0D3F99FE602F0D0F901998A69B9
:10259800002A7FF45BAE0B7C012B3FF4D0AE022BFC
:1025A8003FF47BAD07B0BDE8F08F02F0BFF92BE632
:1025B80002F0BCF9ABE502F0B9F98BE502F0B6F927
:1025C80001988269002A7FF453AD027C012A0346F0
:1025D8003FF4A9AE022A3FF4FBAD53E502F0A6F999
:1025E80024E502F0A3F9FFF750BB02F09FF9FFF7CB
:1025F8002FBB02F09BF901988269002A7FF4E1ABB6
:10260800037C90F85070012B3FF4C3AD022B3FF4CC
:10261800FAAB37E402F08AF9FFF7B1BB02F086F9AA
:1026280001988269002A7FF4CEAC027C012A034615
:102638003FF46FAF022A3FF42BAECEE402F076F9F6
:10264800A0E402F073F917E402F070F9FFF7F8BBA1
:102658000B4AD1690B43D361EDE6094A91690B43F3
:102668009361E8E6186F0308246F03084C720308A7
:102678003D030008D0500308781F002000040140E3
:1026880000100240DC500020381F002014040140D4
:102698001749184B184A194810B4D1F8884044F41F
:1026A8007004C1F888401C6844F001041C605C6830
:1026B80022405A601A6822F0847222F480321A602A
:1026C8001A6822F480221A605A6822F4FE025A60BC
:1026D800DA6A22F00F02DA621A6B002410404FF017
:1026E800006218639C608A605DF8044B704700BF05
:1026F80000ED00E0001002400CC07FF8CCFC00FFA9
:102708001A232422837219230370C27200232322FE
:10271800037542704375704703682DE9F041DF691E
:102728001FB13B46BDE8F0411847002A164611DDA7
:1027380004460D460E4400E023689B6820469847EF
:102748000028F9D0236815F8011B1B682046984714
:10275800AE42F1D1BDE8F08100232522027043701A
:102768008370C3707047152303701623C370172333
:1027780083712D2343702E2303712F23C371704758
:10278800002870B51EDB0928044620DD012303EB71
:1027980083035B00B0FBF3F2092AF8D87BB10E4E35
:1027A800B4FBF3F00928CCBF57223022A6FB03E57F
:1027B800024403FB1044EB0801F8012BF0D100237D
:1027C8000B7070BD2D230B7040420131DBE73030B8
:1027D80001F8010BF3E700BFCDCCCCCC884230B474
:1027E8004FF001042ED301FB04F4B0FBF4F58D4245
:1027F800F9D284B1AAB901E0B0FBF4F5092DCCBF38
:10280800572230222A4404FB150003F8012BB4FB9D
:10281800F1F4002CF0D100221A7030BC7047B0FBE4
:10282800F4F5092DCCBF372230222A4404FB1500C9
:1028380003F8012BB4FBF1F4002CF0D100221A703C
:1028480030BC70470546002AEBD1D7E703685A1C0D
:102858000260197070472DE9F047089C2578002B15
:10286800804689460CBF4FF0200A4FF0300A661C9C
:1028780035B3002A29DD334601E0024698B113F842
:10288800011B501E0029F8D1971E60B13D46013D3D
:1028980051464046C8476B1C002BF8DC257827EAD0
:1028A800E770013055B1041B29464046C847301926
:1028B80016F8015B002DF7D1BDE8F087BDE8F08779
:1028C800002A04DC2846BDE8F0870020EBE7571E05
:1028D800DCE783684268D0ED037A00EB83010133BB
:1028E800934281ED040A836004BF0023836000EBF8
:1028F800830393ED047A036870EE277A9A42C0ED59
:10290800037A77EEC77AC0ED037A0CDA013307EE63
:10291800103AF8EEC76AB7EE007A87EEA60A0360A7
:1029280030EE070A704707EE102AB8EEC77A87EE2E
:10293800870A704790ED057A90ED004AD0ED066A57
:10294800D0ED014AD0ED047A90ED035AD0ED025A49
:10295800A4EE007AB0EE406AB0EE470AB0EE667AAE
:10296800A6EE247A67EEC07AA0EE457AE6EE257ADE
:1029780080ED057AC0ED067A7047D0ED057A90EDC6
:10298800013AD0ED003AD0ED064A90ED024A90EDBA
:10299800077A90ED035A90ED086AD0ED045AC0ED1D
:1029A800067AF0EE406A27EE830AC0ED056AA3EEC8
:1029B800A60A80ED087AA4EE240AA5EE470AA5EE39
:1029C800C60A80ED070A7047D0ED007A90ED017ACB
:1029D80030EE670AE7EE007AB0EE670AC0ED007ADB
:1029E800704770470A44914214D030B40139551EDB
:1029F80041F2210211F8014F082380EA042004045F
:102A08004CBF82EA40004000013B80B2F7D18D42C2
:102A1800F0D130BC704701207047F0B58F7A91F83B
:102A280009E04D7B0C7CCA7C324E3B0203F4706398
:102A38004EEA030391F80BE085B03F0947EA0E1709
:102A48004FEA052CADF802708F7BADF800300CF41E
:102A5800706E2D0991F80CC045EA071527024CEA5B
:102A68000E0C07F4706ECF7BADF804C047EA0E0772
:102A780091F811C091F814E0ADF806508D7CADF8CE
:102A880008701102240901F470611209294344EA0B
:102A98000C1442EA0E12ADF80A40ADF80C10ADF86D
:102AA8000E206C46002140F2765502E034F8023FD1
:102AB8000131B3F5006FA3F5006224BF93B2238000
:102AC800A3F140034FEA430286FB02E3A3EBE27360
:102AD8009BB203F13B022CBF0827002792B2AA42FF
:102AE8000F449CBF03F5577320F817300729DDD131
:102AF80005B0F0BD56555555F0B4184C23785A1CFE
:102B080002F03F02E118531C22441B257E2603F0E5
:102B18003F030E71237015717D27C51D07E0E1186D
:102B2800A84203F101030A7103F03F0313D010F820
:102B3800012BA2F17D010129F1D8591C01F03F01B7
:102B48002344661882F020020131A8421F7101F067
:102B58003F033271EBD12370F0BC70471C1E00207C
:102B680030B50446006D61710368A26823F0010363
:102B7800036087B0A379009213F004023DD04FF4AC
:102B8800805213F00203019244D102934FF4806300
:102B98000022039311F00103059237D1049308230F
:102BA8008D07694648BF049327F0F0FE6079236DCE
:102BB800A17900F00202002A15BF4FF440324FF409
:102BC80080324FF40034002410F0010F586808BF19
:102BD8002246CC074CBF024320EA02025A609A6898
:102BE80009074CBF42F0080222F008029A601A68EE
:102BF80042F001021A6007B030BD13F002030192DF
:102C08000BD04FF4005513460295C1E704230493F3
:102C18000C23C5E74FF40053B7E70293B8E710B5A4
:102C28000446006DA160036823F001030360A379E3
:102C380086B013F00402009141D04FF4805213F093
:102C48000203019244D102934FF4806362790393A3
:102C5800D1074FF000030493059345BF0423049361
:102C680008230C236946920748BF049327F08EFE79
:102C78006079236DA17900F00202002A15BF4FF494
:102C880040324FF480324FF40034002410F0010F2A
:102C9800586808BF2246CC074CBF024320EA02020C
:102CA8005A609A6809074CBF42F0080222F00802ED
:102CB8009A601A6842F001021A6006B010BD13F05B
:102CC8000203019207D04FF4005113460291BDE769
:102CD8004FF40053B7E70293B8E700231F220360BD
:102CE80002701E2282700122436002718371704754
:102CF8002DE9F341056906460F467DBBD0F80080F3
:102D0800C8F30A0323B30023D6F80080019323F005
:102D1800D1F9042819D1224C236943F00103236116
:102D2800BBB2A8F8003023F0C5F904282ED108F169
:102D380002030193019B3F0C1F8023F0BBF9236919
:102D4800042823F00103236125D06FF0010505E075
:102D580023F0B0F9042805D04FF0FF35284602B01B
:102D6800BDE8F0810E4C236943F002032361C4F8E7
:102D78001480236943F04003236123F09BF92369FE
:102D8800042823F002032361BDD0E5E7236923F07B
:102D980001032361D9E7336804333360DEE700BFFA
:102DA80000200240F8B504460D468E180027B542AB
:102DB80001D12069F8BDE368591CE160234415F886
:102DC800012B1A720429F2D1A1682046FFF790FF5F
:102DD800E7602061EBE708B510230B70FDF722FBD5
:102DE800084B1A784AB9084A0849116002221A7031
:102DF800074B012283F8442008BD054B002283F8C5
:102E0800442008BD1F40002050450020012B000829
:102E18001C1E0020082370B50B70FDF703FB074B41
:102E2800074D084C0849094E1A7809482E600025B4
:102E3800A56408600AB903221A7070BD123900200F
:102E4800902400201C1E0020404900202D0300086B
:102E58001503000803685B6A03B1184770470368E5
:102E68001B6A03B11847704703682DE9F041DF6911
:102E78001FB13B46BDE8F0411847002A164611DD50
:102E880004460D460E4400E023689B682046984798
:102E98000028F9D0236815F8011B1B6820469847BD
:102EA800AE42F1D1BDE8F08103689B691847036819
:102EB8005B6918470368DB68184703689B6818470D
:102EC80003685B68184703681B681847014B186854
:102ED800F9E700BFE41F0020054B53F8203033B159
:102EE8001A689B88918A0B4218BF1B04936170472C
:102EF8006855002003682DE9F04F03F13845644E0A
:102F0800AD0A0124755D05F01F066D09022D04FA4E
:102F180006F400F0A280032D00F0A480012D52D009
:102F28008088B0FA80F4C4F11F04A4B2E50803EB6A
:102F3800850504F007042E6AA4000F27A74026EA97
:102F480007062E622E6A01F0030702FA04F47A1EBD
:102F58003443012AC1F3810CC1F300182C62C1F378
:102F6800411135D9C60700F19780850700F1A38084
:102F7800440700F1B180020700F1BF80C60600F1E6
:102F8800CD80850600F1DB80440600F1E980020669
:102F980000F1F780C60500F10581850500F1138170
:102FA800440500F12181020500F12F81C60400F1DA
:102FB8003D81850400F14B81440400F159810204EC
:102FC80055D4BDE8F08F334D6E6934436C61A7E783
:102FD800002422464FF0010E4FF0030904E00132AD
:102FE800102A04F10204ECD00EFA02F636EA0005C3
:102FF800F5D1D3F808A009FA04F5ED430AEA050A61
:10300800C3F808A0D3F808B00CFA04FA4AEA0B0A85
:10301800C3F808A0B3F804A01FFA8AFA2AEA060639
:103028009E80B3F804A008FA02F646EA0A06B6B289
:103038009E801E682E401E60D3F800A007FA04F692
:1030480046EA0A061E60D3F80CA001FA04F605EA5F
:103058000A0A46EA0A05DD60C1E70E4DAE69344347
:10306800AC615DE70B4DEE693443EC6158E71A68D3
:1030780022F040421A601A6842EA87771F60DA68CD
:1030880022F0404242EA8171D960BDE8F08F00BF6A
:103098004C720308001002401A6822F003021A60FA
:1030A8001A683A431A60DA6822F003020A4385076D
:1030B800DA607FF55DAF1A6822F00C021A601A68B0
:1030C80042EA87021A60DA6822F00C0242EA8102B8
:1030D8004407DA607FF54FAF1A6822F030021A60B1
:1030E8001A6842EA07121A60DA6822F0300242EAE5
:1030F8000112DA6002077FF541AF1A6822F0C002B8
:103108001A601A6842EA87121A60DA6822F0C00266
:1031180042EA8112C606DA607FF533AF1A6822F4F4
:1031280040721A601A6842EA07221A60DA6822F4C2
:10313800407242EA01228506DA607FF525AF1A68F7
:1031480022F440621A601A6842EA87221A60DA6832
:1031580022F4406242EA81224406DA607FF517AF22
:103168001A6822F440521A601A6842EA07321A6052
:10317800DA6822F4405242EA0132DA6002067FF548
:1031880009AF1A6822F440421A601A6842EA873284
:103198001A60DA6822F4404242EA8132C605DA60EF
:1031A8007FF5FBAE1A6822F440321A601A6842EAC8
:1031B80007421A60DA6822F4403242EA0142850581
:1031C800DA607FF5EDAE1A6822F440221A601A68B8
:1031D80042EA87421A60DA6822F4402242EA8142CF
:1031E8004405DA607FF5DFAE1A6822F440121A60EF
:1031F8001A6842EA07521A60DA6822F4401242EA70
:103208000152DA6002057FF5D1AE1A6822F4400255
:103218001A601A6842EA87521A60DA6822F4400291
:1032280042EA8152C604DA607FF5C3AE1A6822F01A
:1032380040721A601A6842EA07621A60DA6822F075
:10324800407242EA01628504DA607FF5B5AE1A6819
:1032580022F040621A601A6842EA87621A60DA68E5
:1032680022F0406242EA81624404DA607FF5A7AE48
:103278001A6822F040521A601A6842EA07721A6005
:10328800DA6822F0405242EA0172DA6097E603688F
:1032980003F138422DE9F04F920A584DAA5C02F02A
:1032A8001F0552090124022A04FA05F400F08C8053
:1032B800032A00F08E80012A3CD001F003077A1E11
:1032C800012AC1F3810CC1F300188088C1F34111B0
:1032D80035D9C60700F19680850700F1A28044071A
:1032E80000F1B080020700F1BE80C60600F1CC8074
:1032F800850600F1DA80440600F1E880020600F154
:10330800F680C60500F10481850500F112814405A7
:1033180000F12081020500F12E81C60400F13C81F4
:10332800850400F14A81440400F15881020455D40F
:10333800BDE8F08F324A55692C435461BDE700243B
:1033480022464FF0010E4FF0030904E00132102A23
:1033580004F10204ECD00EFA02F636EA0005F5D1C3
:10336800D3F808A009FA04F5ED430AEA050AC3F8F8
:1033780008A0D3F808B00CFA04FA4AEA0B0AC3F812
:1033880008A0B3F804A01FFA8AFA2AEA06069E8063
:10339800B3F804A008FA02F646EA0A06B6B29E8016
:1033A8001E682E401E60D3F800A007FA04F646EA0D
:1033B8000A061E60D3F80CA001FA04F605EA0A0A08
:1033C80046EA0A05DD60C1E70D4A95692C43946118
:1033D80073E70B4AD5692C43D4616EE71A6822F06B
:1033E80040421A601A6842EA87771F60DA6822F05A
:1033F800404242EA8171D960BDE8F08F4C720308FF
:10340800001002401A6822F003021A601A683A4350
:103418001A60DA6822F003020A438507DA607FF54A
:103428005EAF1A6822F00C021A601A6842EA870234
:103438001A60DA6822F00C0242EA81024407DA6074
:103448007FF550AF1A6822F030021A601A6842EA13
:1034580007121A60DA6822F0300242EA0112DA60D2
:1034680002077FF542AF1A6822F0C0021A601A6894
:1034780042EA87121A60DA6822F0C00242EA811230
:10348800C606DA607FF534AF1A6822F440721A6013
:103498001A6842EA07221A60DA6822F4407242EA9D
:1034A80001228506DA607FF526AF1A6822F44062A9
:1034B8001A601A6842EA87221A60DA6822F44062BF
:1034C80042EA81224406DA607FF518AF1A6822F4CE
:1034D80040521A601A6842EA07321A60DA6822F41F
:1034E800405242EA0132DA6002067FF50AAF1A68F2
:1034F80022F440421A601A6842EA87321A60DA688F
:1035080022F4404242EA8132C605DA607FF5FCAE19
:103518001A6822F440321A601A6842EA07421A60AE
:10352800DA6822F4403242EA01428505DA607FF522
:10353800EEAE1A6822F440221A601A6842EA8742FC
:103548001A60DA6822F4402242EA81424405DA60CD
:103558007FF5E0AE1A6822F440121A601A6842EA4F
:1035680007521A60DA6822F4401242EA0152DA601D
:1035780002057FF5D2AE1A6822F440021A601A6872
:1035880042EA87521A60DA6822F4400242EA81521B
:10359800C604DA607FF5C4AE1A6822F040721A6079
:1035A8001A6842EA07621A60DA6822F0407242EA50
:1035B80001628504DA607FF5B6AE1A6822F04062CF
:1035C8001A601A6842EA87621A60DA6822F0406272
:1035D80042EA81624404DA607FF5A8AE1A6822F0F4
:1035E80040521A601A6842EA07721A60DA6822F0D2
:1035F800405242EA0172DA6098E610B50409013CCB
:10360800052C17D80C4B33F8142000F00F0042FAA1
:1036180000F313F001030DD0012303FA00F0013881
:10362800104030F00FF9054A054B125D104403EBCA
:10363800C00010BD002010BD186F0308246F0308D8
:10364800DC5000202DE9F04F4A484B4B4B4C4FF0D3
:1036580090414FF0010A4FF002094FF004084FF073
:10366800080C4FF0100E20274026802530F8022B3A
:1036780012F0010F03D01960A3F804A0083312F068
:10368800020F03D01960A3F80490083312F0040F56
:1036980003D01960A3F80480083312F0080F03D090
:1036A8001960A3F804C0083312F0100F03D0196092
:1036B800A3F804E0083312F0200F02D019609F80AD
:1036C800083312F0400F02D019609E80083312F0C0
:1036D800800F02D019609D80083312F4807F05D0D6
:1036E8004FF4807B1960A3F804B0083312F4007F0C
:1036F80005D04FF4007B1960A3F804B0083312F426
:10370800806F05D04FF4806B1960A3F804B00833BC
:1037180012F4006F05D04FF4006B1960A3F804B0E1
:10372800083312F4805F05D04FF4805B1960A3F86A
:1037380004B0083312F4005F05D04FF4005B196041
:10374800A3F804B0083312F4804F05D04FF4804B2F
:103758001960A3F804B00833D20B04D04FF4004228
:1037680019609A80083301F58061A1427FF47EAF29
:10377800BDE8F08F186F0308DC50002000180048DF
:10378800002867D003682DE9F04F03F138445C4EF8
:10379800A40A0125345D04F01F066409022C05FA09
:1037A80006F558D0032C00F0A580012C58D080884D
:1037B800B0FA80F4C4F11F04A4B2E50803EB850550
:1037C80004F007042E6AA4000F27A74026EA07067C
:1037D8002E622E6A01F00307A2407C1E3243012CA0
:1037E800C1F3810CC1F300182A62C1F341113CD91D
:1037F800C60700F18980850700F19580440700F12C
:10380800A380020700F1B180C60600F1BF808506DB
:1038180000F1CD80440600F1DB80020600F1E9806A
:10382800C60500F1F780850500F10581440500F122
:103838001381020500F12181C60400F12F8185045E
:1038480000F13D81440400F14B81020400F15981EB
:10385800BDE8F08F70472B4CA6693543A561A6E7F4
:10386800284C666935436561A1E7002422464FF07C
:10387800010E4FF0030904E00132102A04F102049A
:10388800E6D00EFA02F636EA0005F5D1D3F808A01C
:1038980009FA04F5ED430AEA050AC3F808A0D3F8C3
:1038A80008B00CFA04FA4AEA0B0AC3F808A0B3F8FD
:1038B80004A01FFA8AFA2AEA06069E80B3F804A032
:1038C80008FA02F646EA0A06B6B29E801E682E403C
:1038D8001E60D3F800A007FA04F646EA0A061E603E
:1038E800D3F80CA001FA04F605EA0A0A46EA0A0522
:1038F800DD60C1E7034CE6693543E56157E700BF82
:103908004C720308001002401A6822F003021A6081
:103918001A683A431A60DA6822F003020A438507F4
:10392800DA607FF56BAF1A6822F00C021A601A6829
:1039380042EA87021A60DA6822F00C0242EA81023F
:103948004407DA607FF55DAF1A6822F030021A602A
:103958001A6842EA07121A60DA6822F0300242EA6C
:103968000112DA6002077FF54FAF1A6822F0C00231
:103978001A601A6842EA87121A60DA6822F0C002EE
:1039880042EA8112C606DA607FF541AF1A6822F46E
:1039980040721A601A6842EA07221A60DA6822F44A
:1039A800407242EA01228506DA607FF533AF1A6871
:1039B80022F440621A601A6842EA87221A60DA68BA
:1039C80022F4406242EA81224406DA607FF525AF9C
:1039D8001A6822F440521A601A6842EA07321A60DA
:1039E800DA6822F4405242EA0132DA6002067FF5D0
:1039F80017AF1A6822F440421A601A6842EA8732FE
:103A08001A60DA6822F4404242EA8132C605DA6076
:103A18007FF509AF1A6822F440321A601A6842EA40
:103A280007421A60DA6822F4403242EA0142850508
:103A3800DA607FF5FBAE1A6822F440221A601A6831
:103A480042EA87421A60DA6822F4402242EA814256
:103A58004405DA607FF5EDAE1A6822F440121A6068
:103A68001A6842EA07521A60DA6822F4401242EAF7
:103A78000152DA6002057FF5DFAE1A6822F44002CF
:103A88001A601A6842EA87521A60DA6822F4400219
:103A980042EA8152C604DA607FF5D1AE1A6822F094
:103AA80040721A601A6842EA07621A60DA6822F0FD
:103AB800407242EA01628504DA607FF5C3AE1A6893
:103AC80022F040621A601A6842EA87621A60DA686D
:103AD80022F0406242EA81624404DA607FF5B5AEC2
:103AE8001A6822F040521A601A6842EA07721A608D
:103AF800DA6822F0405242EA0172DA6002047FF585
:103B0800A7AE1A6822F040421A601A6842EA87771C
:103B18001F60DA6822F0404242EA8171D960BDE84C
:103B2800F08F002852D0036803F138422DE9F04F96
:103B3800920A514DAA5C02F01F0552090124022A7B
:103B480004FA05F443D0032A00F09080012A43D0F8
:103B580001F003077A1E012AC1F3810CC1F3001892
:103B68008088C1F341113CD9C60700F189808507D7
:103B780000F19580440700F1A380020700F1B180AD
:103B8800C60600F1BF80850600F1CD80440600F12D
:103B9800DB80020600F1E980C60500F1F7808505A3
:103BA80000F10581440500F11381020500F121812E
:103BB800C60400F12F81850400F13D81440400F121
:103BC8004B81020400F15981BDE8F08F70472B4A00
:103BD80095692C439461BBE7284A55692C43546185
:103BE800B6E7002422464FF0010E4FF0030904E027
:103BF8000132102A04F10204E6D00EFA02F636EA7F
:103C08000005F5D1D3F808A009FA04F5ED430AEA4E
:103C1800050AC3F808A0D3F808B00CFA04FA4AEA6F
:103C28000B0AC3F808A0B3F804A01FFA8AFA2AEA14
:103C380006069E80B3F804A008FA02F646EA0A06C9
:103C4800B6B29E801E682E401E60D3F800A007FA08
:103C580004F646EA0A061E60D3F80CA001FA04F638
:103C680005EA0A0A46EA0A05DD60C1E7034AD5699A
:103C78002C43D4616CE700BF4C720308001002406B
:103C88001A6822F003021A601A683A431A60DA685E
:103C980022F003020A438507DA607FF56BAF1A68E2
:103CA80022F00C021A601A6842EA87021A60DA687F
:103CB80022F00C0242EA81024407DA607FF55DAF28
:103CC8001A6822F030021A601A6842EA07121A606B
:103CD800DA6822F0300242EA0112DA6002077FF560
:103CE8004FAF1A6822F0C0021A601A6842EA8712B7
:103CF8001A60DA6822F0C00242EA8112C606DA6067
:103D08007FF541AF1A6822F440721A601A6842EAD5
:103D180007221A60DA6822F4407242EA0122850614
:103D2800DA607FF533AF1A6822F440621A601A68C5
:103D380042EA87221A60DA6822F4406242EA812263
:103D48004406DA607FF525AF1A6822F440521A60FB
:103D58001A6842EA07321A60DA6822F4405242EAE4
:103D68000132DA6002067FF517AF1A6822F4404282
:103D78001A601A6842EA87321A60DA6822F4404206
:103D880042EA8132C605DA607FF509AF1A6822F483
:103D980040321A601A6842EA07421A60DA6822F466
:103DA800403242EA01428505DA607FF5FBAE1A68C7
:103DB80022F440221A601A6842EA87421A60DA68D6
:103DC80022F4402242EA81424405DA607FF5EDAEF2
:103DD8001A6822F440121A601A6842EA07521A60F6
:103DE800DA6822F4401242EA0152DA6002057FF5ED
:103DF800DFAE1A6822F440021A601A6842EA875253
:103E08001A60DA6822F4400242EA8152C604DA6093
:103E18007FF5D1AE1A6822F040721A601A6842EA39
:103E280007621A60DA6822F0407242EA0162850489
:103E3800DA607FF5C3AE1A6822F040621A601A6829
:103E480042EA87621A60DA6822F0406242EA8162D6
:103E58004404DA607FF5B5AE1A6822F040521A6061
:103E68001A6842EA07721A60DA6822F0405242EA97
:103E78000172DA6002047FF5A7AE1A6822F04042A8
:103E88001A601A6842EA87771F60DA6822F04042AF
:103E980042EA8171D960BDE8F08F10B10368828869
:103EA8001A85704710B1036882889A61704738B1E3
:103EB80000298388026814BF002110218B40936178
:103EC800704710B40A4B0B4A1C78012383402340E7
:103ED80052F8200029B9B3FA83F149095DF8044B77
:103EE800E5E7191C18BF01215DF8044BDFE700BFA7
:103EF800645500206855002030B1036882881B8A09
:103F08001A4214BF0120002070472DE9F047A04D48
:103F180095F84C3082B006460A2B58D8DFE803F0F3
:103F280052C5C5C5C5C5CD06185B870003F060FA44
:103F380000242865082241F2B443204685F85440FD
:103F480085F84C20AB65FCF7DBFA002840F01781B8
:103F5800686EFFF7D1FF20B195F85430002B00F0C0
:103F6800D88195F8A830002B40F0BB8003F040FAC8
:103F78002B6DE96D42F22832C01A02FB01F282422F
:103F880025DA95F80931D5F8A4005A1C85F80921D5
:103F9800DA0740F1F180FFF780FF7E4B1B78032B97
:103FA80002D17D4B00221A8000210120FCF7CCFAB7
:103FB80034201FF02FFF0723002085F84C3002B073
:103FC800BDE8F087754B1B680A2B00F2F1800020D2
:103FD80002B0BDE8F087AB6D03F28F1403F008FA66
:103FE8002B6DC01A8442F2DA36201FF013FF22F03C
:103FF8005DF83A201FF00EFF1E2003F045FAD5F8B1
:104008000C01FFF74FFF36201FF004FF95F8D4107E
:1040180063480131C9B2FCF749FB95F84430002BDD
:1040280040F025820A2385F84C300220D0E703F0BF
:10403800DFF92B6DAA6DC01A02F674628242C6DAE5
:1040480003F0D6F9DFF864812865002141F2B44312
:1040580098F8010085F85410AB65FCF775FA342020
:104068001FF0D8FED5F80C01FFF717FF296E0129BC
:1040780040F2128295F81541D5F81801E30740F18E
:104088001282FFF70FFF0134642985F8154140F2C9
:1040980003823221012200200723E96588F80020E5
:1040A80085F8A80085F84C3092E701461846FCF7D9
:1040B8004DFB002002B0BDE8F0872F23002085F8D3
:1040C8004D30FCF779FA07230021012085F84C30A0
:1040D800FCF73AFA34201FF09DFE012002B0BDE83B
:1040E800F08703F085F92B6DAA6DC01A8242BFF6DE
:1040F8003DAF0E2195F86D2095F86E3085F8D410F7
:1041080085F8D63085F8D52095F8E810F27885F846
:10411800D720092385F84C30002900F0568295F8FD
:10412800EA3063F07F03DBB285F8D830737D81F025
:10413800010185F8E810190740F1FE810021882364
:1041480085F8EC1085F8D9301648174C00F10906A7
:10415800002101E010F8012F82EA1122864234F88A
:10416800123083EA01231BB299B2F3D1090A85F808
:10417800E11085F8E230F9E6FFF794FE0DE7322307
:104188002C652C6685F84C402046EB6520E700BF7F
:104198001C1E002012390020343F00209C550020AE
:1041A800F01E0020F31E002010510308000000201C
:1041B800FCF742FA01210220FCF7C4F90C21172070
:1041C800FCF7C0F918210846FCF7BCF91E210620A7
:1041D800FCF7B8F904210720FCF7B4F901210820FD
:1041E800FCF7B0F9FF213E20FCF7ACF90A210B20BF
:1041F800FCF7A8F900210C20FCF7A4F95C210D209C
:10420800FCF7A0F976210E20FCF79CF927210F2056
:10421800FCF798F97B211020FCF794F96121112013
:10422800FCF790F913211220FCF78CF923211320B5
:10423800FCF788F97A211420FCF784F9512115201C
:10424800FCF780F916211920FCF77CF96C211A205B
:10425800FCF778F903211B20FCF774F940211C2096
:10426800FCF770F991211D20FCF76CF956212120EB
:10427800FCF768F910212220FCF764F9A921232012
:10428800FCF760F90A212420FCF75CF900212520BD
:10429800FCF758F911212620FCF754F95921292057
:1042A800FCF750F988212C20FCF74CF931212D20FE
:1042B800FCF748F90B212E20FCF744F907210320CD
:1042C800FCF740F900210920FCF73CF936201FF0E3
:1042D800A1FD002436201FF09DFDE1B20A20FCF765
:1042E80031F933201FF096FD4FF4617003F0CCF8DC
:1042F8002320FCF7C3F92420FCF7C0F9013425205A
:10430800FCF7BCF9FF2CE5D1012385F84C300020DF
:104318005EE6FB20FCF7B2F900F07F03FB2085F88E
:104328006830FCF7ABF900F07F01202985F86810A8
:1043380040F2BC80202185F868103046FCF7E0F98F
:1043480095F868C0BCF1070F06F1030000F05F8123
:10435800ACF1080E5FFA8EFE0EF1040ED14CB64495
:10436800002110F8012B82EA1122704534F812302E
:1043780083EA012399B2F4D10B0A06EB0C0414F872
:10438800042C9A427FF4EDAD14F8032CCBB29A4278
:104398007FF4E7AD33781D2B7FF4E3AD727895F8A1
:1043A8006D309A427FF4DDADB27895F86E309A425E
:1043B8007FF4D7ADB27995F8A2309A427FF4D1ADA7
:1043C800DFF80483D5F8A400002301222B66AB652F
:1043D800EA65FFF767FD98F80030BBB1737931796A
:1043E80095F84D209B00DBB2914288F8013007D345
:1043F80002F13F008842C0F20D81013388F8013094
:104408000122002385F8A82088F8003014F8020C4F
:104418002FF0D2FB727DA44995F8C9E002F003029F
:104428003446C2EBC20354F8160FC850C818E9182E
:104438000EF10103A488848003F003030124002003
:104448009A4281F8B24085F8C80000F0FB801C460B
:10445800C4EBC401294404F1010C91F8B20000280E
:1044680000F0E0800CF00304A242F1D1EAE08F4AA8
:10447800D5F810311268D31A0020182B8DF80700D0
:1044880018D902AE012306F8013DC5F810213146BE
:1044980000221CF01BFBC5E501310823296685F8BD
:1044A8004C30002094E5FFF7F8FCECE500293FF4D8
:1044B80058AD42E795F8D0807D4F08F1010808F023
:1044C80003084FEAC80982460DF10706A9EB08045C
:1044D8002C4494F8B230002BD9D00028D7D194F8C6
:1044E800AC2095F814319A4202D813E00028EDD197
:1044F800E2183146002392F8AD003A461CF068FDF8
:1045080095F8143194F8AC200133DBB29A4285F85F
:104518001431EBD89A42D9D1A9EB08032B4408F1FE
:10452800010285F8D08002F0030883F8B2A085F86C
:1045380014A14FEAC809C9E713F040014DD1C3F3EC
:104548000113013395F8EC0003F0030398423FF49C
:10455800FBAD95F8C86095F8082195F800E0554C32
:1045680006F0F00660F301060B4685F8D96072453F
:10457800DFB205EB020602F1010103F1010343D0AA
:10458800327904F8012B052B01F03F02EFD185F8B1
:1045980008211F46484C85F8DA702646431C00EB74
:1045A8004001584256F8167D95F8D720B6884FEA4C
:1045B800410100F0030003F0030358BF43426018B1
:1045C800675085F8EC308680BEE53C483C4B007B64
:1045D80033F81030C3F34613A6E53A4C95F8C810E3
:1045E800C3F3011303EB430604F1160000EB460086
:1045F80001F0F00163F3010186880368A68085F85D
:10460800D910C5F8DA309FE585F80821C2E70023FC
:104618001946B2E602F17F00814223DC023388F8B2
:104628000130EDE695F8C820D5F8CC1064F30512F2
:10463800D2B242F040020131540685F8C820C5F8CC
:10464800CC1016D40022C5F8CC20C3EBC3022A44F0
:10465800591C92F8B220CAB3734537D01F4601F0EF
:104668000303F2E7BF329142DCBF033388F801301D
:10467800C6E604290ED9032385F8B20085F8B900E7
:1046880085F8C00085F8C700C5F8CC0085F8D0309B
:1046980085F8C93002F0ACFE0123286585F854304E
:1046A8005FE400BF10510308C81E00209C5500207D
:1046B8001F2A0008F71E00200C1F00201455002098
:1046C80034550020F61E00200000002095F8C83060
:1046D80085F8C97067F3051385F8C830DAE72DE95E
:1046E800F0410C4E356873691D4011D0DFF8288001
:1046F8000127B5FA85F4C4F11F0408EB840307FA0F
:1047080004F4D3F81C0103689847A5437461F0D1F9
:10471800BDE8F081000401401C1E00202DE9F04195
:104728000C4E356873691D4011D0DFF82C800127C5
:10473800B5FA85F4C4F11F0408EB840307FA04F4FE
:10474800D3F81C0103689847A5437461F0D1BDE80C
:10475800F08100BF000401401C1E00202DE9F0413B
:104768000C4E356873691D4011D0DFF82C80012785
:10477800B5FA85F4C4F11F0408EB840307FA04F4BE
:10478800D3F81C0103689847A5437461F0D1BDE8CC
:10479800F08100BF000401401C1E00202DE9F041FB
:1047A8000C4E356873691D4011D0DFF82C80012745
:1047B800B5FA85F4C4F11F0408EB840307FA04F47E
:1047C800D3F81C0103689847A5437461F0D1BDE88C
:1047D800F08100BF000401401C1E00202DE9F041BB
:1047E8000C4E356873691D4011D0DFF82C80012705
:1047F800B5FA85F4C4F11F0408EB840307FA04F43E
:10480800D3F81C0103689847A5437461F0D1BDE84B
:10481800F08100BF000401401C1E00202DE9F0417A
:104828000C4E356873691D4011D0DFF82C800127C4
:10483800B5FA85F4C4F11F0408EB840307FA04F4FD
:10484800D3F81C0103689847A5437461F0D1BDE80B
:10485800F08100BF000401401C1E00202DE9F0413A
:104868000C4E356873691D4011D0DFF82C80012784
:10487800B5FA85F4C4F11F0408EB840307FA04F4BD
:10488800D3F81C0103689847A5437461F0D1BDE8CB
:10489800F08100BF000401401C1E0020094A9369F2
:1048A80010B5094C43F00103936104F58E70402262
:1048B800002130F09AFB4FF0FF33C4F85C31C4F8A4
:1048C8005F3110BD001002401C1E00202DE9F04190
:1048D800044618460D46164698462EF0B9FA27683B
:1048E800E6722844A07229467D694346324620462E
:1048F800AC46BDE8F0416047036810B504461B6844
:104908009847236820469B689847A37B0133A37385
:1049180010BD08B5FEF771FE38B12D228271002254
:10492800C271BDE8084024F015BB08BD0B4B984286
:1049380006D0A3F5784398420DD04FF0FF3070476A
:104948000022074B03EB02135A89013292B25A81B3
:10495800588980B270470122F3E700BF0030014058
:10496800382C0020F0B50D460178012983B00446A3
:10497800164618D0022902D0002003B0F0BD806886
:104988001F46FFF78AFA45F080016068FBF736FE9C
:104998003B46324600216068FCF7C2FAA068FFF780
:1049A80081FA0120E9E790F90400421CE4D00228CA
:1049B800E2DC617900962A46FCF704FFDDE7427ADB
:1049C80002B9704710B504460368406804F10A014B
:1049D80098470023637210BD437A5A1C0344D2B22D
:1049E80042729972037A934200D802B9704710B59F
:1049F80004460368406804F10A019847002363727B
:104A080010BD98B10B4B012210B402FA01F103F169
:104A1800750402E00333A34209D01A788242F9D11F
:104A28005A780A42F6D001205DF8044B70470020FE
:104A3800FAE700BF1053030830B40A4D002305F508
:104A4800007401E0272B0AD003EB43020133A15C79
:104A58008142F7D12A4430BC92F802027047002004
:104A680030BC70471051030870B5448806460D469F
:104A7800C4F30B0422460021284630F0B6FA336905
:104A8800094A934209D3094A934206D22246284644
:104A98001946BDE870402FF0ADB923B1214628462C
:104AA800BDE87040184770BDCCB10308F2B20308E6
:104AB800064B07498B4202D30023184670471A88D1
:104AC800C2F30B029042F8D01433F3E758AD030851
:104AD800CCB10308024A136823EA0000106070474B
:104AE800EC530020F8B5174D2B78A52B28D16B78FF
:104AF800BE2B25D1022229464FF6FF70FDF772FF23
:104B0800114FAC1C22884AB1A618BE4218D2052AF9
:104B180016D92146FDF766FF3446F3E721460222FF
:104B2800FDF760FF0222A118FDF75CFF0634074B72
:104B3800641B1C8041F60F53C31A58425841F8BDF4
:104B48000020F8BD00F00308000004080A2D00202A
:104B58002DE9F04FDFF848914C4F8BB00326A7EBB7
:104B680009071822002104A830F03FFA484BCDF875
:104B7800109005971A69120604D5464A5A6002F140
:104B880088325A6001228DF824203422DA60424BA0
:104B9800424C1B88ADF800300222694604A8FEF793
:104BA80001F9022269464FF6FF70FDF71BFFDFF897
:104BB800F4A080464FF0000B544536D30AAC0025CC
:104BC80024F8245D0222214604A8FEF7EBF802220D
:104BD80021464046FDF706FF40BAC043ADF808003D
:104BE800022202A904A8FEF7DDF8079860B106AB17
:104BF800C0F104022946184430F0F7F9069904A8D0
:104C0800FEF776F8079508909DF82430089A23B1A6
:104C18001F490B6943F080030B61013E2DD0002A28
:104C28009FD1FFF75FFF50B32CE065888DF80DB07A
:104C3800C5F30B05AB1DADF808302388C3F30B0291
:104C4800ADF80A201B0B062202A904A88DF80C3027
:104C5800FEF7A8F8062202A94046FDF7C3FE6168E0
:104C680080462A4604A8FEF79DF8616840462A4611
:104C7800FDF7B8FE143480469EE7002AD1D00520FF
:104C880001F0DAF80BB0BDE8F08F00BF00000408AF
:104C980000200240230167458553030858AD0308E7
:104CA80000F00308CCB103080378202B024600F17A
:104CB8000100F9D0092BF7D02D2B2CD02B2B03BFBB
:104CC8005378B7EE000A0246B7EE000AA3F13001A6
:104CD800C8B209289FED467A10D8F2EE046A07EEAA
:104CE800901AF8EEE77A12F8013FE7EE267AA3F178
:104CF8003001C8B20928B0EE677AF0D92E2B4CD013
:104D080003F0DF03452B0BD0F7EE007A67EE276A36
:104D180020EE260A70475378BFEE000A0246D5E710
:104D280010B451782D2959D02B290ABF9178501CDD
:104D3800901C0024A1F13003092B53D8002303EB66
:104D4800830301EB430310F8011FA1F13002092A84
:104D5800A3F13003F3D9B3F59A7F28BF4FF49A73C0
:104D6800072B42D9DFED236A1A46F7EE007A083A94
:104D7800072A67EEA67AFAD803F007032BB1F2EEFA
:104D8800046A013B67EEA67AFBD124B3C7EE276A13
:104D98005DF8044B20EE260A70475378A3F13001E2
:104DA800C8B2092802F10102AAD8F2EE046AF0EEAC
:104DB800665A07EE901AF8EEE77A12F8013F87EE86
:104DC800A66AA3F13001C8B2092866EEA56A37EED3
:104DD800067AEED994E767EE276AD9E7901C9178AE
:104DE8000124A7E7F7EE007ACFE7F7EE007AC5E7E8
:104DF8000000000020BCBE4CB5EEC00ADFED317AE1
:104E0800F1EE10FACCBF30EE270A30EE670ADFED7C
:104E18002E7A20EE270A30B5FDEEC07A87B017EE5D
:104E2800904A054684EAE470002303A9A0EBE470E5
:104E380001930093029326F0FDFE002CACBF2023C3
:104E48002D2303A88DF800302EF002F8012803A9BD
:104E580024D002282DD0032805BF30236846684691
:104E68008DF8013030F0C9F868462DF0F1FF0338AD
:104E7800C4B222466946284630F0F6F800232B557E
:104E880028462DF0E5FF2E22431C2A540DEB040181
:104E9800E81830F0CFF8284607B030BD3023684610
:104EA8008DF801308DF802308DF8033030F0A5F818
:104EB800DAE7302368468DF801308DF8023030F09B
:104EC8009CF8D1E76F12033A00007A442DE9F041CB
:104ED800064615460846B6FBF2F43CB905FB1464D1
:104EE800124B1B5D00F8013BBDE8F081B4FBF2F703
:104EF80067B90E4B05FB174705FB1464DA5D00F82C
:104F0800012B1B5D00F8013BBDE8F081B7FBF2F80F
:104F1800B8F1000F02D04046FFF7D8FF05FB18781C
:104F2800024B13F8082000F8012BE3E72C7C030858
:104F38002DE9F04714461D46064600234FF47A72C1
:104F4800204629462EF02EFCDFF848814B4A4C4F6C
:104F580088FB00310144C31782FB002EC3EB6111AB
:104F680088FB012887FB00278644464AC3EBEE2EC0
:104F7800C1EB011C82FB0E29A0EB8C0C0744424AB2
:104F880086F806C0C3EB27474FEAEE7C08EB010A18
:104F9800CCEBA90C82FB07824FEAE1780CEB4C0CB6
:104FA800C8EB6A18AEEBCC0EC8EB0818DFF8E8C0FF
:104FB80086F804E0A1EB880171718CFB0010F917E9
:104FC800C1EBE21240F2B55101FB1272C3EBE050A3
:104FD800B2F5896F4FEA800740DA40F2DA239A4245
:104FE80044DCB2F5B77FB4BF4FF0000C4FF0010CB2
:104FF8004FEA4C08254B08EB0C0103EBC1031FFAE1
:105008008CFEB3F88E02224908EB0C0301EBC301B6
:1050180016310B2301E031F8020D82421BDA013B05
:10502800F9D11A4BC44403EBCC0C0123BCF8780229
:10503800B37007F2B2770132121ABE44F270A6F8C2
:1050480000E0204629464FF47A7200232EF0AAFB8E
:105058003281BDE8F0870133DBB2E9E74FF0030E98
:10506800F44640F296504FF00608CCE74FF0020E97
:10507800F44640F229404FF00408C4E7C5B3A291B2
:1050880007452EC2ABAAAA2A73B06D1610510308A1
:105098008853030889888888792D0311104B2DE9D6
:1050A8003048D3E9004554EA05020BD103460122F2
:1050B80000201871587198719A70DA7018801881E8
:1050C800BDE83088074B1A6814EB020B45F1000C59
:1050D8005A466346FFF72CFF0120BDE8308800BF21
:1050E800402300209C550020F0B402888578164F94
:1050F800C37804794179A2F2B27202F0030606EB92
:105108004606013D05EB860507EB4505013BB5F86D
:1051180078628579008940F2B557920807FB023218
:10512800931903EB430304EBC303C3EB031301EB32
:105138008303C3EB031305EB830300214FF47A7257
:10514800C2FB0301F0BC704710510308FAB170B4F8
:105158008E18044603E0101A14D1B14214D014F882
:10516800012BA2F14103192B11F8013BA3F14105D1
:1051780098BF2032192D03F12000ECD9D01A01D1A3
:10518800002BEAD170BC7047002070BC70471046F5
:1051980070474FF0FF32FFF7D9BFA0F16103192B19
:1051A80098BF20387047A0F14103192B98BF2030D1
:1051B8007047202805D0093804288CBF002001201A
:1051C800704701207047613819288CBF00200120E2
:1051D8007047413819288CBF0020012070473038AB
:1051E80009288CBF002001207047A0F13003092B4B
:1051F80007D920F02000413819288CBF0020012051
:1052080070470120704730B402681146531C036090
:1052180011F8024B0160D31C517803609378151D77
:1052280005601B0443EA0123D078234343EA006066
:1052380030BC70470368591C1A46016012F8021BFB
:105248000260587841EA0020704703685A1C0260DF
:105258001878704738B50446006815462EF0CAFD20
:1052680022682A44226038BD036810B40A0A5C1C0C
:1052780004601A7003685A1C026019705DF8044BC8
:10528800704703685A1C026010B4197003680A0A50
:105298005C1C04601A7003680A0C5C1C04601A70B9
:1052A8000368090E5A1C026019705DF8044B7047B8
:1052B80003685A1C026019700368090A5A1C0260C4
:1052C800197070472DE9F047002488B080460F46D2
:1052D8001E46A14605AD531C0393117839B3252901
:1052E80033D1931CCDF810900393507830284ED0CA
:1052F8004FF0000AA0F13003DBB2092B42D96C2829
:1053080019D0642800F0938024D825281CD063D9AC
:10531800582876D063281BD131784046B847039A7D
:10532800531C03931178043601340029D7D1204641
:1053380008B0BDE8F087039B5A1C03921B78642BC6
:105348007CD02AD8252B54D1252140460134B84792
:10535800039AC0E7732833D044D975284FD106F192
:10536800040E30682B4600220A217646FDF736FAED
:10537800049A0095534639464046FDF76CFA039A5D
:105388000444A8E704AA03A926F09AFBB7E7D31CAC
:10539800039390784FF0010AACE7732B10D05BD9D8
:1053A800752B3AD0782B96D1A3F15802B2FA82F233
:1053B800306852092B4610210436FDF70FFAD7E75B
:1053C8003368049A0093394600234046FDF743FAB0
:1053D80004360444039A7EE70028B9D1204608B071
:1053E800BDE8F0876E28B3D1039A336804361C6091
:1053F80071E72AD9582BD7D0632B8DD06BE7782843
:10540800A6D1A0F15802B2FA82F2306852092B46AE
:105418001021FDF7E3F90436AAE706F1040E306817
:105428002B4600220A217646FDF7D8F9A0E7331D5E
:10543800306829461E46FDF7A3F999E7331D306801
:1054480029461E46FDF79CF992E7002B7FF443AFEF
:10545800204608B0BDE8F0876E2BC6D03BE70EB4F7
:1054680000B584B005AB019053F8042B06490393AB
:1054780001A8FFF727FF019B00221A7004B05DF80E
:1054880004EB03B0704700BF552800080FB430B5CF
:1054980083B006AB0A490B4853F8042B0968006827
:1054A8000193FFF70FFF084C05462068FDF7FFFC46
:1054B8000028FAD0284603B0BDE8304004B0704751
:1054C800082C00200C2C0020E41F0020DFED2B7A94
:1054D800B4EEE70AF1EE10FA4ADDDFED296A9FED36
:1054E800297A01E0B0EE670AB4EEC70AF1EE10FAC5
:1054F80070EE667AF6DC9FED247AF4EEC77AF1EE68
:1055080010FA38D5DFED1E6A9FED207A01E0F0EE43
:10551800407AF4EEC77AF1EE10FA37EEA60AF6D41E
:10552800DFED1B7AB4EEE70AF1EE10FA14DDDFEDD9
:10553800137A37EEC00A60EE006A9FED166A9FED97
:10554800167ADFED167AA6EE867A20EE266AE6EE61
:10555800877AA6EE270A7047DFED117AB4EEE70ADC
:10556800F1EE10FA44BFDFED087A37EEC00AE2E741
:10557800F0EE407ABFE7B0EE670AD1E7DB0F4940AB
:10558800DB0FC940E4CB1641DB0F49C0E4CB16C1A1
:10559800DB0FC93F92E741B99730083C15A82ABEEE
:1055A800DB0FC9BF09B909E0194690FBF1F301FB0C
:1055B80013030846002BF7D1084670470146FBE75E
:1055C80007EE901AF8EE677A9FED837A27EE800A45
:1055D80020EE070AFDEEC07A17EE903A2033402BF2
:1055E80000F28C80DFED7D7AB4EEE70AF1EE10FA76
:1055F80040F3E880B0EE407A9FED796ADFED796A92
:1056080001E0B0EE677AB4EEE67AF1EE10FA77EEE2
:10561800467AF6DC9FED747AF4EEC77AF1EE10FA6A
:1056280040F1CD809FED6E6ADFED706A01E0F0EE2B
:10563800477AF4EEE67AF1EE10FA37EE867AF6D487
:10564800DFED6B7AB4EEE77AF1EE10FA51DCDFEDBC
:10565800697AB4EEE77AF1EE10FA44BFDFED627AC8
:1056680037EEC77A27EE076ADFED635ADFED637A14
:10567800DFED636A9FED635AE6EE257A67EE065A18
:10568800E6EE276AF7EE007AA5EEA67AF0EE675AFC
:10569800E7EE055AE7EE457A87EEA55ADFED547A2C
:1056A80030EE277AFDEEC76A16EE903A2033402B8B
:1056B80029D99FED557AF6EE006AB7EE006AF7EE43
:1056C800004AC4EEA57A0023836143610362C36183
:1056D80080ED045A67EEA66A27EE866A27EE877A77
:1056E800C0ED006AC0ED026A80ED016A80ED037AC0
:1056F8007047DFED3A7A37EEC77AB3E7B7EE005A6C
:10570800F0EE455ACAE7B4EEE70AF1EE10FA5FDDAB
:105718009FED336ADFED336A01E0B0EE677AB4EEED
:10572800E67AF1EE10FA77EE467AF6DC9FED2E7AFD
:10573800F4EEC77AF1EE10FA47D59FED296ADFED4E
:105748002B6A01E0F0EE477AF4EEE67AF1EE10FA11
:1057580037EE867AF6D4DFED267AB4EEE77AF1EE04
:1057680010FA27DCDFED237AB4EEE77AF1EE10FACF
:1057780044BFDFED1D7A37EEC77A27EE076ADFED03
:105788001E4ADFED1E6ADFED1E7AE6EE246A67EE3A
:10579800064AE6EE267AB7EE006AA4EEA77AF6EE97
:1057A800006A36EE476AF8EE007A27EE277A66EE48
:1057B800266A84E7DFED097A37EEC77ADDE7B0EECF
:1057C800677A3DE7F0EE407A24E7B0EE677AC2E701
:1057D800F0EE477AAAE700BF27D4D236DB0F49405C
:1057E800DB0FC940E4CB1641DB0F49C0E4CB16C13F
:1057F800DB0FC93FDB0FC9BF92E741B99730083CBF
:1058080015A82ABEF304353F0000008070B406686E
:105818008E4217D90139751E002311F8014F08224D
:10582800634013F0800F4FEA430318BF83F0D5039A
:10583800013ADBB2F5D18D42EFD1721C02603370B0
:1058480070BC70470023F8E710B44C09012250F8E7
:10585800243001F01F0102FA01F10B4340F8243013
:105868005DF8044B70474B0901F01F0150F82320E5
:10587800012303FA01F1114214BF184600207047B2
:1058880038B50B4C23688BB15A68821A002A054632
:1058980004DA0CE05A68AA1A002A07DB9A68226020
:1058A80018461A6890472368002BF3D138BD38BDD5
:1058B800C43300200D4B04210022890710B4027262
:1058C80003F1640402D51979815401329C4203F131
:1058D800140308D0072A06DC99798907F3D49C4277
:1058E80003F11403F6D15DF8044B704754720308B2
:1058F80010B4104C0423214613F001034FF00002AA
:1059080001F1140108D10132062A0ED08B7913F067
:10591800010301F11401F6D002EB820204EB8202CA
:105928005DF8044B13790370704703705DF8044BFE
:10593800704700BF54720308012310B400221024DA
:105948001121447041710372037083710371837074
:10595800C271C2705DF8044B704700BF436A826928
:10596800D154436A0169826B01338B4228BF0023FB
:105978004362002A2FD0EFF31181502383F312885A
:10598800836B1A68D2072CD470B45E686EB9456A06
:10599800826A954217D084691444DC600ED9AA1A29
:1059A8005A608562002280F854201A6842F0010289
:1059B800C9B21A6081F3118870BC70470469A21AD1
:1059C8005A608662EEE7012380F85430C9B281F349
:1059D800118870BC7047026D136843F08003136030
:1059E8007047C9B281F31188704700BF426B10B489
:1059F80062B1436CC2684469D11A013B615C5DF8CD
:105A0800044B08BF13464364C8B27047016A436930
:105A1800C4685B5C0131A14228BF114601625DF890
:105A2800044BD8B2704700BF836B13B190F8540091
:105A38007047836A406A181AB0FA80F040097047C4
:105A4800416A836A99420AD3CB1A816B026961B1B0
:105A58004968501E0B4483420AD2C01A7047026933
:105A68001144CB1A816B0029F2D1501EC01A70471D
:105A780000207047436B43B1426C5B6893422FBF71
:105A8800981AC0689B1AC0187047C269036A9A427C
:105A98002FBFD01AC0688018C01A70472DE9F04788
:105AA8008C4B1B78DB07074644D58B4B8B4D1C78FA
:105AB8008B4E012C59D01CD3022C07D189498A4A14
:105AC80009881288914201D901241C70EB7AE3B14C
:105AD8002B89D3B1854B1B78BBB10EF0E5FB0028B1
:105AE80000F09B802B7B83422CBF01210021317069
:105AF8000CE07C497E4A098810886A7B801A8842B3
:105B0800E2DAEB7A0024002BE2D131782A79632A91
:105B180006D8022C774E00F0BA803378002B5DD17E
:105B2800754AAB7A8C4238BF0C461470002B4CD1A6
:105B3800BDE8F0876B4B694D19885B88E878CB1A0C
:105B480083EAE3728142A2EBE3721DD32B788B4286
:105B58001AD3614B1C78E01E012861D9674909787E
:105B680002294FD0012C5E4EA5D15F4A5D491288AB
:105B7800687B0988121A914239DD5D4A12888A4287
:105B8800A4D200241C70A1E7B1EB400FE1DC524B1A
:105B98001C78E11E012940F29480022ADEDC574974
:105BA8004F4E0878DFF84481DFF844C1DFF838E168
:105BB80000210324022834701C7088F80010ACF807
:105BC8000010AEF8001081D11FE0012C71D0022C1A
:105BD8000BD10720BDE8F0472CF0CEBE7068381A0C
:105BE800474B984258DD72709AE7BDE8F087022467
:105BF8001C706BE7022AD2DD4049097802294FF070
:105C0800040464D13949364E09783E48022ACCBF8B
:105C180000220122C28081804BE70221317075E7A2
:105C2800022A9BDC95F800C091FBFCFC0CF1010CEE
:105C3800BCF1080FDFF8B4A0304EA87895F801E061
:105C480096F800802A4CDFF8A090254EA8BF4FF0A8
:105C5800080C8AF800C01FFA8CFA10FB0AF01EFB29
:105C68000AFE80B2DFF88CA02080A9F800E00024AA
:105C78004FF0640EB8F1020F34701C70CAF804407B
:105C88008AF801E07FF439AF0FFA8CF1BDE730787C
:105C9800A0B9012377603370C2F164021A4B00FB8C
:105CA80002F083FB0023C017A0EBA3506430707090
:105CB80036E70820BDE8F0472CF05EBE7368F81A96
:105CC8008EE7032C96D10D49097802299AD0044E03
:105CD800FCE600BFBF55002090260020B0480020F9
:105CE800A02600203846002094260020F2460020F6
:105CF8009226002098260020373F0020D446002016
:105D08007F969800D84600206BCA5F6B2DE9F04754
:105D18000569C3681D4028D00F4606464FF0004865
:105D28004FF00009B5FA85F328FA03F2D2431B3B7A
:105D380032611540042B16D8DFE803F03129211908
:105D480003007B6A002B32D003F1FF3A1FFA8AFA6C
:105D5800C7F824903C6A34B12368204651469847D6
:105D68006468002CF8D1002DDCD1BDE8F0873868D4
:105D7800716B036889B29847002DD3D1F5E778682D
:105D8800B16B036889B29847002DCBD1EDE7B868AD
:105D9800F16B036889B29847002DC3D1E5E7F8682D
:105DA800316C036889B29847002DBBD1DDE7F36AEF
:105DB8001FFA83FACEE700BF08B501210220FEF7DB
:105DC80080F8094B1B7803F00503052B08D0002148
:105DD8000120FEF776F800210846FEF772F8FEE784
:105DE8001EF042FFF3E700BF102C0020022828BF56
:105DF800022010B4084C094B207000EB8002C0EB65
:105E0800C20207495DF8044B013003EB4203C0B2FC
:105E18000B602CF097BE00BF844900209A520020E6
:105E28001849002008B513F0C3FEFEF791FEBDE83F
:105E3800084013F0A5BE00BF2DE9F04F013085B032
:105E4800C3B203938E4D8F4F8F4C904E0A2302930B
:105E58003220DFF8409223F0F1FD4FF4FA7A4FF048
:105E6800100C4FF47A70D9F80430C3F30803002BF0
:105E780040F0C880EFF31183002B40F0C3802968FD
:105E8800A26800BF2B689942F9D1D7F800E000FB5F
:105E98000EF39B1AB3FBFEF300FB01314FF0010E2A
:105EA8000191D9F80430C3F30803002B40F08E8029
:105EB800EFF31183002B40F089802B68A16800BFA5
:105EC8002A689342F9D1D7F800B000FB0BF2521AB6
:105ED800B2FBFBF200FB0323019A9B1AB3F57A7F0E
:105EE800DFD3BAF1010ABED1039B002B40F0C48076
:105EF8004FF47A7ADFF89C9150464FF0100CD9F89D
:105F08000430C3F30803002B40F09980EFF31183AA
:105F1800002B40F094802968A26800BF2B68994242
:105F2800F9D1D7F800E000FB0EF39B1AB3FBFEF3A0
:105F380000FB01314FF0010E0191D9F80430C3F391
:105F480008033BBBEFF3118323BB2B68A16800BF99
:105F58002A689342F9D1D7F800B000FB0BF2521A25
:105F6800B2FBFBF200FB0323019A9B1AB3F57A7F7D
:105F7800E3D3BAF1010AC2D1029B013B02937FF439
:105F880067AF4349434B4448444A0860DA6005B068
:105F9800BDE8F08FEFF311888CF31288A1682368AD
:105FA800DB0344BFC6F800E0A1682B6832685FFADB
:105FB80088F888F31188D7F800801A4400FB08F3A2
:105FC8005B1AB3FBF8F300FB0233CDE7EFF311885C
:105FD8008CF31288A1682368DB0344BFC6F800E08D
:105FE800A1682B6832685FFA88F888F31188D7F8B7
:105FF80000801A4400FB08F35B1AB3FBF8F300FBBC
:10600800023369E7EFF311828CF31288D4F808E0C1
:106018002368D90303D501233360D4F808E02B683B
:106028003168D2B282F311883A68194400FB02F34E
:10603800A3EB0E03B3FBF2F300FB01312EE7EFF302
:1060480011828CF31288D4F808E02368D90303D5A9
:1060580001233360D4F808E02B683168D2B282F3A8
:1060680011883A68194400FB02F3A3EB0E03B3FB53
:10607800F2F300FB01315DE7184623F04FFB37E7E9
:106088009C550020A055002010E000E09855002005
:10609800FC9F002000ED00E0EFBEADDE0400FA0535
:1060A80038B5434B5A899989914224BF00225A81B5
:1060B800198ADA89914224BF0022DA81DA788AB310
:1060C800072A2FD03B493C4D91F853000124002169
:1060D8000A282C709C70D9713DD00C2865D0DFED52
:1060E800377A8ABB364C9FED370AA278002918BF49
:1060F800F0EE407A062A04D8334901EB820191ED8B
:10610800000A217959B3013A032A4DD8F7EE007AEB
:1061180087EE800A2DF0AEFF2388984228BF1846E4
:10612800208038BDD97921B198780428B8BF0420D7
:106138009870204890F853000A280CD00C28CED12B
:10614800DFED227A002ACDD0072ACBD00A282CD11D
:10615800DFED1F7AC6E70A20DFED1E7AC1E79B78DC
:10616800154A07EE103A1178B8EEC77A27EE277A63
:1061780007EE901AF8EEE77A67EE877AB4EEE70A48
:10618800F1EE10FA10DDC0EE077AFDEEE77A17EEB1
:10619800903A102BA8BF1023012BB8BF0123DBB204
:1061A8008B4238BF0B46137038BDDFED0B7A99E789
:1061B800684D00207C4D0020683700206F1203399D
:1061C800205800206F120338E85303080AD7A33970
:1061D8000F506E3A5304E9386F12833A2DE9F047AD
:1061E800AE4FAF4E13F0E4FCBE421ED2DFF82C8354
:1061F800DFF82C934446258862197DB14A450DD2B3
:10620800052D0BD933886188C3F30B03994200F03D
:10621800E480144625886219002DEFD17168304654
:106228001436FEF721FCBE42E4D39E4A1378A3F14C
:10623800170102290FD99C4911F83300002840F0B2
:10624800F880D8000144497829B1984911F83330C9
:10625800002B00F01C81964B5A78022A40F2E3800A
:10626800002294495A701A789348022A016000F271
:10627800D68002EB8201914BC2EBC10203EB4203D1
:10628800998C5A8C8E4C9142236001D300225A84F7
:106298008C4B9A78042A00F0F18032B91A88B2F54A
:1062A800F07F84BF4FF4F0721A80874DFFF7F8FE35
:1062B8002B68864A1A40002A00F0EC80DE0700F1BD
:1062C800D880580400F1D080190700F1C8809A01DD
:1062D80000F1BF809B0400F1B58020F013F810B9DD
:1062E8007B480DF019FE4020FEF7F4FB8020FEF7F6
:1062F800F1FB4FF40070FEF7EDFB4FF48020FEF742
:10630800E9FB4FF40010FEF7E5FB4FF08060FEF765
:10631800E1FB4FF00060FEF7DDFB1FF0E3F9002121
:1063280030226C482EF061FE206827F03BF86A4B5B
:10633800276803F1500102E0043399426DD01A78BE
:10634800002AF9D19C78D8788442F5D26349644B05
:106358000D79644964480A70644E654C0460C8222B
:10636800642111FB0521002259609A60DA601A61E4
:106378005A619A61DA6183F8202083F82120376016
:1063880017F09AFE5B4B9FED5C5A1B885B4A9FEDAA
:106398005C6A50795B4906EE903AF8EEE66A138833
:1063A800C5EE265A07EE103A53881279C1ED005A05
:1063B80007EE903AB8EEC77A534BF8EEE77A1872C0
:1063C8005A7227EE067A67EE867ABDE8F04783EDC3
:1063D800017AC3ED007A13F0D3BB63799B077FF48E
:1063E80018AF716894F804A03046FEF73DFB338877
:1063F800BAEB133F04D01436BE42FFF4FBAE14E7E9
:1064080073887068AA1FC3F30B039A4204F106014C
:10641800A8BF1A462DF0EEFCEDE7012296E7002210
:106428001A70264B2CE7234902EB420201EB82014A
:1064380019E7D8000C186468002C7FF403AF172400
:106448001470FFE63148FEF745FB4020FEF742FB9B
:1064580043E746F20900FEF73DFB2B683AE72C4874
:10646800FEF738FB2B6832E72A48FEF733FB2B6828
:106478002AE72948FEF72EFB2B6822E79A8AB2F50D
:106488007A7FBFF412AF4FF47A729A820DE718231D
:106498001370E0E643F000732B600FE7CCB10308FC
:1064A80058AD0308EC39002068760308B073030878
:1064B80084490020904900201C4900209A5200205D
:1064C8001849002020580020EC53002009600002E1
:1064D8004C4D0020D020002028340020D44C00202F
:1064E8003C3F002074060020BC1F0020042100202F
:1064F8007A370020BC220020C0C9FB483423002082
:1065080017B7D138C0220020144C002009400002DF
:1065180001600002092000020860000202F003087E
:106528000000040808B513F043FBFEF711FB13F055
:1065380027FBFFF753FE0120BDE808402CF002BB03
:106548002DE9F047B54C82B063682046984700288B
:1065580000F0BF80B24B1B780122042B84F83C204A
:1065680000F0BA80B4F91610B4F91820B4F91A304A
:1065780021636263A363AB4B1B88002B69D0AA4DD0
:10658800D4ED0C7AD5ED004A95ED050A95ED015A42
:1065980095ED067AD5ED035A95ED026AF8EEE76AAD
:1065A800D5ED047AA4EEA60AA5EE267A67EEC07A9F
:1065B800A5EEC07AE6EE267A85ED057AC5ED067A6F
:1065C8002DF058FDD4ED0D6AD5ED094A95ED0E0A6A
:1065D80095ED0A5A95ED0F7AD5ED0D7AD5ED0C5A51
:1065E80095ED0B6A2063F8EEE66AA4EEA60AA5EE1E
:1065F800267A67EEC07AA5EEC07AE6EE267A85EDB1
:106608000E7AC5ED0F7A2DF035FDD4ED0E6AD5ED75
:10661800124A95ED170A95ED135A95ED187AD5EDAE
:10662800167AD5ED155A95ED146A6063F8EEE66AA8
:10663800A6EEA40AA6EE857A67EEC07AA0EE657A81
:10664800E6EE867A85ED177AC5ED187A2DF012FDFB
:10665800A063764FA17F764817F0B0FC3B88002BEB
:106668007CD1744E3568744B1B685B0742D4B5F90E
:106678000070216B636BA06B704A714E92ED026AD9
:10668800D2ED006AD2ED015AC91B2163B5F9027037
:10669800DB1B6363B5F904703568C01B07EE900A0D
:1066A800B8EEE75A07EE901AB8EEE77A07EE903A96
:1066B800F8EEE77A36EE056A36EE877A77EEA57A4F
:1066C8000135A06382ED026A82ED007AC2ED017A9B
:1066D800356002B0BDE8F0875A4BB4F91600B4F93A
:1066E8001810B4F91A2018802063598061639A80C1
:1066F800A26340E7544F3B88322B7ED0002B5BD1FE
:1067080052480378002BB2D0DFF848E1F169326AC9
:106718008EFB01730027C9170770C1EB23118EFB8D
:106728000203D217C2EB2312736A29806A80A08AF7
:1067380047498EFB03E2DB17C3EB22131B1AAB801E
:10674800CF6013F035FAFEF703FA13F019FAFFF7E2
:1067580045FD01202CF0F6F9356888E7354E226BA7
:106768003568B3F5C87F4FF0000323632B80398861
:1067780018BF7068B7F8008008BF0020B1F5C87F5F
:1067880018BFB368616B02440B440020B8F5C87F9A
:1067980060637260B36068803AD0D4F838E0F1681A
:1067A800A0637144B8F1010FA880F16054D008F1DA
:1067B800FF38A7F8008056E7F169226B00232363AE
:1067C8002B80B7F800E00A44BEF1320F616B6363B7
:1067D8006B80F261A26B6BD0706A0190306AA36320
:1067E8000144019831620244BEF1010FAB8072622C
:1067F80063D00EF1FF333B8082E7154B2988D868B8
:106808006A88AB883182B0617282B3820021D4E792
:10681800A36BF360A063A880C9E700BFCC48002041
:10682800D4460020343D0020383D0020F64C00209E
:10683800FC480020BC1F002004500020084C002009
:10684800044C0020D8460020CC200020C92000207D
:10685800743700201F85EB51DFF80CC1DFF8F8E032
:10686800C8328CFB02A9C833D217C2EBE9128CFBE1
:1068780003A9DB17C3EBE913C8316B802A808CFBB3
:10688800013CA28ACB17C3EBEC139B1AAB80CEF862
:106898000C0013F08DF9FEF75BF913F071F9FFF7AF
:1068A8009DFC40462CF04EF9B7F8008035687EE72D
:1068B800A36331627262AB809BE7234A2348126864
:1068C8002349037012F4003281F800E032D11346F4
:1068D8002049C85C0B2803F10C030ED00132182A9A
:1068E800F7D1338A2B80728A1B4B6A80B18AB269CE
:1068F800A980B7F800E0DA607BE71848D0F800C054
:106908005300BCF1000F09D003EB020E01EB8E0E11
:106918009CF801C09EF801E0E645E2D21344DFF896
:106928004CE00F4A01EB830100230160AEF8003010
:106938001360D6E70B4A1278032A01D01A46C7E734
:106948002BF0FEFF3568CCE7E82F0020CE20002092
:10695800C82000202C650308743700203822002046
:1069680024230020373F00201F85EB5120230020DF
:1069780038B50C4C0C4DAC4206D261682046143434
:10698800FEF772F8AC42F8D3084A094B094C146078
:10699800002209491A705A7008480860BDE8384052
:1069A80018F05ABF58AD0308CCB1030818490020A5
:1069B800844900209A5200201C4900209049002058
:1069C80008B5FFF7D5FF13F0F3F8FEF7C1F8BDE8F7
:1069D800084013F0D5B800BFF0B50C292BD8DFE874
:1069E80001F06F2A2A2A4C2A2A2A2B2A2A2A070047
:1069F800046AB2F80CE097881668674D24F480544E
:106A08000462036A4468C16923F4005343EA0E33FD
:106A180021F4E641A84243EA073341EA062100F09F
:106A2800B58005F50065A84200F0B0809268446022
:106A3800C16102640362F0BD046A96899588D2F840
:106A480000E0554F24F480740462036A4468C16905
:106A580023F4007343EA062321F07301B84243EAA2
:106A6800052341EA0E017ED04C4DA8427BD09268A6
:106A78004460C161C2630362F0BD046A9689958867
:106A8800D2F800E0444F24F010040462036A44681A
:106A9800816923F0200321F0807143EA061321F471
:106AA800E641B84243EA051341EA0E2148D03B4D7E
:106AB800A84245D092684460816182630362F0BD58
:106AC800046A9389B2F804E01768334E24F001048D
:106AD8000462056A4468816943EA0E0321F480313F
:106AE80025F002059BB221F07301B04243EA050389
:106AF80041EA070114D0294DA84211D005F5406597
:106B0800A8420DD005F58065A84209D005F5806535
:106B1800A84205D092684460816142630362F0BD77
:106B2800D689158A578A23F0080333433D43D6880C
:106B380024F4407423F00403ADB233432C43E9E753
:106B4800D589178AD68823F0800343EA051324F4ED
:106B58004064558A23F0400344EA870443EA061355
:106B680044EA8504A6E7D589178AD68823F4006302
:106B780043EA052324F44054558A23F4806344EA05
:106B8800071443EA062344EA051470E7158A24F437
:106B9800804444EA851449E7002C01400034014050
:106BA8002DE9F04FC822002183B07948794CDFF8ED
:106BB8000892794D794E7A4FDFF800822EF015FA57
:106BC80078487949DFF8F8E1DFF8F8C1002213596D
:106BD800834200F0C280B3F1804F00F0CA80AB421C
:106BE80000F0C980B34200F0C880BB4200F0C78003
:106BF800734500F0C680634500F0C580434500F04A
:106C0800C480DFF8C4A153457AD00AF5806A534599
:106C180008BF092375D01432782AD8D15D4C634D4A
:106C2800634E614F04F1780802E01434A04564D043
:106C3800A379002BF9D023794FEA131909F1FF3909
:106C4800B9F1050F03F00F03EFD835F8190040FA32
:106C580003F2D207E9D54FF0010A0AFA03F3013B20
:106C680018402CF0EFFD16F809305249184411EB82
:106C7800C002DAD051F83000DFF850E1217A00F193
:106C880038439B0A1EF8033003F01F0E5B09022BE2
:106C98000AFA0EFA63D0032B66D0012B58D09388DA
:106CA8000093B3FA83F3C3F11F039BB2DA0800EB36
:106CB800820203F00703D2F820E09B004FF00F0C8C
:106CC8000CFA03FC2EEA0C0EC2F820E0D2F820E001
:106CD80001FA03F343EA0E03136269460023022212
:106CE80014348DF804208DF805308DF806308DF8B1
:106CF800073023F001FCA0459AD103B0BDE8F08F1E
:106D0800082309EBC3034FF0010B93F820A00AF006
:106D18001F034FEA5A1ABAF1020F0BFA03F311D004
:106D2800BAF1030F08D0DA457FF475AFD1F814A093
:106D380043EA0A034B616EE7D1F81CA043EA0A0351
:106D4800CB6168E7D1F818A043EA0A038B6162E7D0
:106D58007B694AEA03037B61A1E70023D1E7BB69AA
:106D68004AEA0303BB619AE7FB694AEA0303FB614A
:106D780095E70123C5E70223C3E70323C1E70423FB
:106D8800BFE70523BDE70623BBE70723B9E700BF35
:106D9800CC4A002054720308000400400008004058
:106DA80000100040002C014000100240186F03083A
:106DB800246F0308DC500020E8530308004001401A
:106DC8000014004000340140004401404C720308A4
:106DD80001490248FEF79ABF6C4B00200040014071
:106DE80001490248FEF792BF444B0020003401409D
:106DF80001490248FEF78ABF444B00200034014095
:106E080001490248FEF782BF1C4B002000040040E5
:106E180002494FF08040FEF779BF00BFF44A0020D6
:106E280001490248FEF772BFCC4A0020002C0140FD
:106E380001490248FEF76ABFCC4A0020002C0140F5
:106E48002DE9F04104684A4DA30AAB4272D009D833
:106E5800B3F5801F6AD04A3DAB425AD14FF0700E4D
:106E6800022608E0434DAB4268D00335AB4252D10D
:106E78004FF0C00E042647794FEA970C002961D0DD
:106E8800B000634685190227D4F80C809F400CEBAC
:106E98004503BFB2384D03F1040C47EA080745F82B
:106EA800231045F82C20E760EFF31181502282F37C
:106EB8001288821905EBC202136973B31362043393
:106EC800821905EBC202576917B11F605369043371
:106ED800821905EBC202976917B11F6093690433E1
:106EE800821905EBC202D76917B11F60D369043351
:106EF8000027CAB21F6082F31188304405EBC00036
:106F0800036A6BB9E3684FF6FE721340E360BDE8AD
:106F1800F081BDE8F081BDE8F08105EB0E03CFE715
:106F2800E36843F00103E360BDE8F0814FF0480EE9
:106F38000126A0E74FF0200E00269CE74FF0980EA0
:106F4800032698E7BF08022306FA03F0BB40DB4399
:106F5800E768094D9BB23B4087190CEB470CE3608F
:106F68000CF1040345F82C1045F823209CE700BFDA
:106F78004B0010004D001000CC4A002030B50368CB
:106F88005C4D18885C4CB4FBF2F20139013AAB4213
:106F980094B283B089B282B266D05848834263D033
:106FA800B3F1804F60D0A0F5983083425CD000F5F3
:106FB8008060834258D0524883425BD000F580609D
:106FC80083427DD022F4407200F58C3092B2834225
:106FD8001A80D9621C850ED0484A93420BD002F51C
:106FE8004062934207D002F58062934203D002F5D3
:106FF8008062934201D100221A8601225A611A88BE
:107008003C4992B242F001028B421A8062D0B3F13D
:10701800804F61D03B4A934260D002F58062934230
:107028005ED002F5006293425CD002F58062934222
:107038005AD002F59032934258D002F540629342FA
:1070480056D002F5806293421ED002F580629342C8
:1070580008BF092219D002A84FF0012340F8043DC7
:1070680023F014FA03B030BD254822F070028342A1
:1070780092B2A3D101201A80D9621C8558611A885E
:1070880092B202431A80C5E708221F4B03EBC203E2
:1070980001A893F821408DF80440012300228DF8BF
:1070A80005308DF807308DF8062023F0EFF91B2CFA
:1070B800D8D1164B019301A823F0E8F903B030BDED
:1070C80001201A80D9621C8558611A8892B202433D
:1070D8001A809CE70022D8E70122D6E70222D4E7EB
:1070E8000322D2E70422D0E70522CEE70622CCE726
:1070F8000722CAE7002C014000A24A0400340140DC
:107108000010004000040040E85303081901000182
:10711800204B98422DD0B0F1804F2CD0A3F594335A
:1071280098422AD003F58063984228D003F500637B
:10713800984226D003F58063984224D003F5903313
:10714800984222D003F54063984220D003F580632B
:10715800984207D003F58063984208BF092202D0FD
:107168000020704708220C4B03EBC20393F8200061
:1071780070470022F7E70122F5E70222F3E703222E
:10718800F1E70422EFE70522EDE70622EBE7072205
:10719800E9E700BF002C0140E85303082DE9F04F50
:1071A800013085B0C3B203930B4602918B4C8C4ED1
:1071B800002B00F09A8032208A4D8B4FDFF82C92FA
:1071C80022F03CFC4FF4FA7A4FF0100C4FF47A702E
:1071D800D9F80430C3F30803002B40F0DE80EFF346
:1071E8001183002B40F0D9802968A26800BF2B6862
:1071F8009942F9D1D7F800E000FB0EF39B1AB3FBD4
:10720800FEF300FB01314FF0010E0191D9F8043073
:10721800C3F30803002B40F08780EFF31183002BA2
:1072280040F082802B68A16800BF2A689342F9D198
:10723800D7F800B000FB0BF2521AB2FBFBF200FBCE
:107248000323019A9B1AB3F57A7FDFD3BAF1010AB7
:10725800BED1039B002B40F0BD804FF47A7ADFF853
:107268008C9150464FF0100CD9F80430C3F3080342
:10727800002B75D1EFF31183002B71D12968A26817
:1072880000BF2B689942F9D1D7F800E000FB0EF354
:107298009B1AB3FBFEF300FB01314FF0010E019185
:1072A800D9F80430C3F3080313BBEFF31183FBB918
:1072B8002B68A16800BF2A689342F9D1D7F800B0BB
:1072C80000FB0BF2521AB2FBFBF200FB0323019AFC
:1072D8009B1AB3F57A7FE3D3BAF1010AC4D1029BB2
:1072E800013B0293002B7FF466AF05B0BDE8F08F39
:1072F800EFF311888CF31288A1682368DB0344BF7D
:10730800C6F800E0A1682B6832685FFA88F888F34D
:107318001188D7F800801A4400FB08F35B1AB3FB06
:10732800F8F300FB0233D2E7EFF311888CF31288ED
:10733800A1682368DB0344BFC6F800E0A1682B6896
:1073480032685FFA88F888F31188D7F800801A4401
:1073580000FB08F35B1AB3FBF8F300FB023370E79A
:10736800EFF311828CF31288D4F808E02368D9036C
:1073780003D501233360D4F808E02B683168D2B212
:1073880082F311883A68194400FB02F3A3EB0E0359
:10739800B3FBF2F300FB01317FE7EFF311828CF3CB
:1073A8001288D4F808E02368D90303D50123336091
:1073B800D4F808E02B683168D2B282F311883A68B1
:1073C800194400FB02F3A3EB0E03B3FBF2F300FB3B
:1073D800013118E7184622F0A1F93EE710E000E075
:1073E800985500209C550020A055002000ED00E095
:1073F800204B5B68C3F3080330B4BBB9EFF31183C8
:10740800A3B91D4B1D4C1868A16800BF1A689042AB
:10741800F9D11B4B1C684FF47A7202FB04F3591A1A
:10742800B1FBF4F130BC02FB00107047EFF311829E
:10743800102383F3128811498C680B6813F4803F7A
:10744800104B02D0012018608C680B49D2B20D682D
:10745800186882F311880A4B19684FF47A72284425
:1074680002FB01F31B1B30BCB3FBF1F302FB003042
:10747800704700BF00ED00E09C55002010E000E0E0
:10748800A0550020985500202DE9F84F8046FFF7B9
:10749800AFFF254E2549DFF8A0E0254A254D844653
:1074A80010274FF47A740120DEF80430C3F3080380
:1074B800D3B9EFF31183BBB90B68D2F808A000BFAA
:1074C800D1F800904B45F7D1D6F800B004FB0BF982
:1074D800A9EB0A09B9FBFBF904FB0393A3EB0C0323
:1074E8004345E1D3BDE8F88FEFF3118A87F312889B
:1074F800D2F808B01368DB0344BF2860D2F808B09C
:107508000B68D5F800905FFA8AFA8AF31188D6F8E2
:1075180000A0994404FB0AF3A3EB0B03B3FBFAF3B3
:1075280004FB0933DAE700BFA05500209C55002072
:1075380010E000E09855002000ED00E02DE9F04F44
:10754800DFF830C1474A4849484E494D8046102720
:1075580018F1FF38C0F08480DCF80430C3F3080366
:10756800002B5CD1EFF31183002B58D10B68946882
:1075780000BF08688342F9D1D6F800904FF47A70BA
:1075880000FB09FEAEEB040EBEFBF9FE00FB03EEAA
:10759800DCF80430C3F308034FF47A740120FBB914
:1075A800EFF31183E3B90B68D2F808A000BFD1F854
:1075B80000904B45F7D1D6F800B004FB0BF9A9EBC6
:1075C8000A09B9FBFBF904FB0393A3EB0E03B3F51C
:1075D8007A7FBDD2DCF80430C3F30803002BDFD078
:1075E800EFF3118A87F31288D2F808B01368DB0327
:1075F80044BF2860D2F808B00B68D5F800905FFA4D
:107608008AFA8AF31188D6F800A0994404FB0AF391
:10761800A3EB0B03B3FBFAF304FB0933D5E7EFF352
:10762800118487F31288D2F808901368D80303D519
:1076380001232B60D2F808900B682868E4B284F321
:107648001188D6F800A04FF47A7400EB030E04FBFF
:107658000AF3A3EB0903B3FBFAF304FB0E3E97E727
:10766800BDE8F08F10E000E09C550020A0550020F8
:107678009855002000ED00E030B4EFF3118310229C
:1076880082F312880649074C0A6807480132002528
:107698000A602560DBB2026883F3118830BC70474A
:1076A8009C5500209855002010E000E00F4B1B88E7
:1076B800014643B90E4B0F4A1B7810680BB981F08D
:1076C8000101FCF7F4BB0C4B5A691AB118B91A68D6
:1076D800106058747047094A18681188084A92FB64
:1076E800F1F2012102605974704700BF74550020FF
:1076F80076550020785500207C55002094550020B0
:1077080020A107001D4B70B55C68236D626BDD69B5
:10771800C2B1A36B2BB12B0702D5236D08221A62C5
:1077280070BD2A06F7D5A26A616A8A4220D0511C28
:10773800A069A162825C2069266D81423285EAD304
:10774800A362E8E7A906E4D5E26A22B1988C216B26
:1077580080B29047DDE7E1699B8C6069DBB24E1C23
:10776800E6614354E169E368994228BFE261D0E7E2
:10777800226D136823F080031360CCE7142C0020DB
:107788001D4B70B51C68236D626BDD69C2B1A36BBC
:107798002BB12B0702D5236D08221A6270BD2A0669
:1077A800F7D5A26A616A8A4220D0511CA069A162F9
:1077B800825C2069266D81423285EAD3A362E8E7BC
:1077C800A906E4D5E26A22B1988C216B80B2904771
:1077D800DDE7E1699B8C6069DBB24E1CE6614354CE
:1077E800E169E368994228BFE261D0E7226D136836
:1077F80023F080031360CCE7142C002070B4EFF35F
:107808001186502383F31288836B1A68D20720D419
:107818005D686DB9446A826A944217D081691144DF
:10782800D9600ED9A21A5A608462002280F85420C6
:107838001A6842F00102F1B21A6081F3118870BC33
:10784800704701698A1A5A608562EEE7012380F859
:107858005430F1B281F3118870BC70472DE9F04FB4
:10786800C04B1E788BB0002E40F0BB80BE4BBF4C87
:107878001D78DFF818A3DFF81893DFF8188305F0F0
:107888000105A4F10A0B54F80A3CBBB1CC2707FB4D
:1078980006B71846FBF714FB80B154F80A0CFBF73F
:1078A80009FB14F8023C8BB9242830D0F5B154F800
:1078B8000A3C1846FBF704FB0028EED10136032EDC
:1078C80004F1CC04DFD10BB0BDE8F08F012B22D03E
:1078D800022B2AD0032B36D0042B66D0052B3FD0A1
:1078E800062B4ED054F80A2C1346D2E754F80A3C1B
:1078F80023281A4600F089819D49897E8142C8D192
:107908009C4BCAF80090C3F80C801346C1E70123CA
:1079180004F8023CCBE74D2854F80A2C0CBF02238C
:10792800002304F8023C1346B3E700233C2804F87C
:10793800023C45D03E28D5D10122032304F8012C6E
:1079480004F8023CB3E7C02814D80022042304F842
:10795800050C04F8040C04F8062C04F8023CA6E70D
:1079680014F8063C14F8052C9A422FD814F8043C55
:10797800834203D0002304F8023C98E7062304F866
:10798800023C14F801ECBEF1000F00F08281BEF158
:10799800010F00F0C68101360023032E04F8023CD3
:1079A80004F1CC047FF46FAF8DE714F8043C04F8BD
:1079B800030C5840052304F8040C04F8023C76E74D
:1079C800032204F8013C04F8022C70E714F8042C94
:1079D800F9184240013304F8042C04F8063C887274
:1079E80065E7654B186800283FF46DAFFCF7E7FFC3
:1079F800DFF8A4A1614DDFF8A491DAF80000FBF7E5
:107A08005FFA00283FF45FAFDAF80000FBF752FA9C
:107A180009281BD03F2819D02B68002B67D10428D0
:107A280000F0A9810C2800F0E9807F28E5D0A0F1BA
:107A38002002D2B25E2AE0D80BB92028DDD05A1C29
:107A480009F803002A6024F059FCD6E72C68002CBA
:107A58005BD14B4FA34607F59878BBF1000F08BFE1
:107A6800BB4608374745F8D1BBF1000F00F07881D5
:107A7800083FDBF800003A68065D135D9E4220442B
:107A880002EB040140F06A81661E4E4422460BB99F
:107A9800FD2A5DD906F8013F01322A6010F8013F3E
:107AA80011F801EF9E45F2D00AB15F4512D0354872
:107AB80024F02CFC5F4508D35BF8080B24F026FC67
:107AC800092024F01BFCBB45F6D92F4824F01EFCE6
:107AD8002A680024944290D2661E4E4416F8010F7C
:107AE80024F00CFC2B6801349C42F7D385E70C2862
:107AF80000F084800A2853D00D2851D07F2800F048
:107B0800FD80FF2B3FF679AF91E71D4E002706F564
:107B18009878BB4602E0083646450DD022463168C3
:107B28004846FDF713FB0028F5D1B346002FF2D1E4
:107B3800374608364645F1D13B465F469B46002B03
:107B480097D1002F3FF459AF0E4824F0DFFBB3E77D
:107B5800511C202009F80200296009F801300A4662
:107B6800A3E700BF7F490020BF5500205A7B0020B3
:107B78004C4D002000ED00E0302D0020382E002074
:107B8800C4560308547C03085C7C0308FC9F00204F
:107B9800EFBEADDE0400FA05342D0020382D00209C
:107BA80024F035FC23217C482DF036FA002800F01B
:107BB800E080A0EB0900286088B1431E19F8031083
:107BC800202940F0E68009EB030204E012F8011DC9
:107BD800202947D10346581E002BF7D12B604FF4BC
:107BE8008072002148462DF000FA6C4B1B78002B60
:107BF8003FF469AE6A4824F089FBFEE6694824F040
:107C080085FB674824F082FBF7E667496748C9782F
:107C1800674ADFF8CCE19362003118BF0121017097
:107C28006449D1624021136382F8341082F83550D8
:107C3800614962480B602C32CEF80020574A012374
:107C4800137024F0E9FC564824F060FB4FF4006000
:107C58000AF0E2F85A4B9B7E232B00F0928014F82E
:107C6800023C3DE62B60574C002204F5987809F851
:107C7800032002E00834444577D0216848460EF0D6
:107C880089FF0028F6D044456FD2636898470023DF
:107C9800A4E74D4BADF822E00FCB0DF1280C02AF55
:107CA80087E80F004CF824ED14F8051C14F8033C81
:107CB800069404EB010E624639464FF0010C06A803
:107CC800CDF81CE0ADF820308DF824C007F02EFB6D
:107CD800E8B9019F002304F8023C002F3FF4EEAD01
:107CE80054F80A0C0CF0C8FD013654F80A0CB847D1
:107CF800032E04F1CC047FF4C6ADE4E5013B002279
:107D080032482B6009F8032024F000FB75E6029A3C
:107D18002F4B03923946A4F10A0002930CF026FD7A
:107D2800D7E714F8053C14F8032C0694234407936A
:107D38006E2A4FF0000308930993ADF820207FF4D2
:107D48002AAE06A8FDF781FA06A8FDF773FA06A879
:107D5800FDF770FA06A8FDF76DFA1CE62246A3E6C1
:107D68001C48083F24F0D2FAA6E61B4824F0CEFAB5
:107D78008DE7286820E708480EF055FB0BB0BDE8F2
:107D8800F08F164A14F8023CC2F80C80CAF800902A
:107D9800A6E5034667E700BF382D00207F4900208D
:107DA8005C7C0308647C030884490020F4260020D6
:107DB800BC1F002021270008342D0020907C0308D8
:107DC8004C4D0020C4560308545403088C7C030807
:107DD8007C7F0020547C0308707C030800ED00E0E1
:107DE800302D00202DE9F04F2DED068BA04BA14A38
:107DF8001C7897B000F59C41203181460B911160A9
:107E0800002C00F0EA869C4A1268904240F2838077
:107E18009A4A069216689A499A4A0591013C1C703A
:107E2800994B049206F480560893002E40F0818006
:107E3800964B1B78022B01F09481042B01F083816F
:107E4800012B01F03781924B9945089B9B7800F2F2
:107E58009685002B40F097858E4B0793069B1E68EE
:107E680016F4805740F08786DFF860A2049BB3F9C8
:107E78000610059B5D8BA942B4BF00250125864BE2
:107E88001B6813F080535ED0079A127812F0010233
:107E98005FD00598408C884241F3B882002D5ED1AE
:107EA8007E4C94F88C10002959D17D487D49006892
:107EB80090F82D0000240C604C608C607A490028F2
:107EC8004ED10870002A4FD0F0064DD5774A127867
:107ED800D10649D4002F47D1002B45D1720243D493
:107EE800734B1B78002B02F01982724B9B78002D84
:107EF80042F081823BB1704A704B12681B689B1A32
:107F0800002BC2F26D821020644C2AF035FD01234B
:107F180084F88D3028E0594B06931E68594B584A0F
:107F2800049306F48056584B05920893002E3FF4AC
:107F38007FAF00215848FDF796FC00287FF478AF02
:107F48001AF0C4FE74E774029ED4079A127802F0FD
:107F58000102524C002184F88C10002DA5D0524902
:107F680001200870002AAFD1554B1A78002A40F03A
:107F7800BD800599049C488BB4F90070898BB4F9CD
:107F88000240B842B4BF8026002646F04003B942FA
:107F9800D8BF33469B0843F08006A042B8BF33469B
:107FA800049F43F04006A142C8BF33469B08B7F977
:107FB8000440B7F9066043F08007A042B8BF3B46CB
:107FC80043F04007A142C8BF3B469B0843F08007E7
:107FD800324C8642C8BF3B4643F0400794F88EE0D7
:107FE8008E42B8BF3B469E4501F04A84A4F89020D3
:107FF80084F892202E4984F88E300E78002E01F0F5
:108008004B835F2B01F0BE836F2B01F0FD83079B31
:108018001B78DE076AD494F89210002966D1B4F967
:108028009030322B62DD94F88E200120572A84F894
:1080380092004DD0069B1B685D0741F199825A2A30
:1080480041F0968294F89430002B42F05E8194F8C7
:10805800963083F0010384F89630002B42F0D681E5
:108068000C202AF089FC174B174D099341E000BFFB
:10807800C033002098320020BC3300200450002078
:10808800204D0020967E00203C3F00201239002021
:10809800404B4C00BF5500203C37002034200020C6
:1080A800184900208C3900208C220020F839002043
:1080B80074060020943700209C550020944B002023
:1080C800FF4900201C490020144900207834002072
:1080D800884B894A19684FF47A73B3FBF1F3C3EB01
:1080E800431103EB8103DB00A2F8A830834B844DD6
:1080F8000993069B1B685F0700F1B4860DF15009D0
:10810800804E0A950022C9F804203446149240F69D
:10811800330B4FF0190840F28337049D02E0043412
:10812800544522D0A178E378994218FB0170F6D221
:1081380094F801E00EF1040E18FB037135F91E30B6
:108148005B45A8BF5B46B3F5617FB8BF4FF4617369
:108158009842E4DA9942E2DB21782729DFD84846B9
:108168000434FDF771FB5445DCD1674A0A9D137846
:10817800664A99E8030082E80300002B40F0F08586
:10818800634B1A78002A00F06A8501215F48FDF7E1
:108198006AFB002840F0E782089BDB78002B40F060
:1081A800E2825C4B0A932B881FB227F001071FFA63
:1081B80087F84345A5F8008001F00280564F4FF03C
:1081C80002090E204FF0140A4FF0FF0B87F80090B9
:1081D80087F801A087F802B02AF0CEFB49464B4841
:1081E800B5F80080FDF73FFB002841F09A8228F09F
:1081F80002039BB243452B800BD0474B022014212E
:10820800FF2218700E2059709A702AF0B5FBB5F845
:108218000080424B424A197850680C9318F0030FBB
:1082280008BF81F00201C1F340010B92FBF73FFE4A
:1082380024213648FDF717FB30B9079A13785F07F2
:1082480044BF23F0040313700A9B1B6813F00A0F42
:1082580011D006212D48FDF706FB002801F0AD805E
:108268002B88580641F1258207212848FDF7FBFA9B
:10827800002840F0C8870C212448FDF7F4FA2A8822
:10828800002800F0508342F480739A422B8009D072
:10829800214B022214211A700E20FF2259709A7065
:1082A8002AF06AFB1F4B1B78082B00F048830E2B23
:1082B80000F04583069BD3F8008018F4806F6BD0DC
:1082C800194B1B79002B00F0308214210F48FDF761
:1082D800CAFA002840F02E8216F09CFF01200CF00C
:1082E80015FD002855D0DFF844A000274FF0CC0B2F
:1082F800A14620E0F44F00207C4D00201C490020BE
:108308001449002028340020445800203C3700201D
:108318007F490020C048002010310020645500200B
:1083280068550020EC390020E4460020507B0020EE
:10833800DFB2022F2CD80BFB07F87B1C5AF8084039
:10834800002CF5D1032290F9023002940192C278F0
:10835800E24951F82220009218462246234601217C
:108368000CF05EFB034607EB470000EB00100A9396
:1083780053B121460AEB8000CC222CF036FE0A9B32
:108388004AF808300137FFB21FF036F90028D0D17B
:108398004C46069BD3F80080079B93F800A0D04B6F
:1083A8001AF0010A00F0418201221A70099B04990F
:1083B8001B68B1F906105A89CA480127914207700B
:1083C80080F21982C84B4FF07E521A60059BC74F46
:1083D800B3F81890049B97F90420B3F90030387863
:1083E80097F801C0002AA3EB090714BF01224FF038
:1083F800FF32002FB8BF7F42B7F5FA7FA8BF4FF40E
:10840800FA77B84280F2F4813F1A07EE907AF8EED4
:10841800E77AB74F4B45C7ED007A03DAF1EE677A92
:10842800C7ED007A049BB3F902E0AEEB0903002B19
:10843800B8BF5B42B3F5FA7FA8BF4FF4FA7398420E
:1084480080F2D3811B1A07EE903AF8EEE77AF145ED
:10845800C7ED017A03DDF1EE677AC7ED017A049B77
:10846800B3F90400A0EB0903002BB8BF5B42B3F5D6
:10847800FA7FA8BF4FF4FA736345CCBFA3EB0C0394
:10848800002302FB03F207EE902AF8EEE77A48454C
:10849800C7ED027ABCBFF1EE677AC7ED027A18F42D
:1084A800805800F07F81B1F5FA6F924BA8BF4FF466
:1084B800FA61B1F57A7F1A78B8BF4FF47A71A1F5ED
:1084C8007A71002A41F01D818B4ADFF844E282FB71
:1084D8000130CB17C3EB6013581C6FF0630C3EF9E7
:1084E80010003EF913E00CFB0313A0EB0E0003FB96
:1084F80000F382FB0312DB17C3EB62139E440FFAEF
:108508008EFE07EE90EAB8EEE78A87ED038AB8F1A7
:10851800000F40F066842B885A0640F1FB807749AB
:10852800774A91ED018AD2ED019A92ED026A91EDB6
:10853800034A92ED030A91ED029A92ED007AD1ED89
:10854800005AD7ED011A97ED002A6E4A6E4938EEA7
:10855800445A79EEC63A77EE007A65EE233A75EE1C
:10856800C96A75EE890A37EE401A66EEA76AB0EE58
:10857800633AA0EE813A13F00303B0EE665A78EE40
:10858800044A79EE867AA0EE815AF0EE638AA4EE68
:10859800A73AD4EEA78AA4EEE75A33EE263AF0EECD
:1085A800687AF0EE674AF6EE008A35EE88AAE0EEC1
:1085B800C14A28EEC33A35EE635A77EE293A77EE88
:1085C800E67AAAEE233A25EE285A76EE403A34EEB9
:1085D80049AAE0EE817A74EEA64AAAEE235A34EE4E
:1085E800094A37EE697A64EEA84A63EE036AE4EE54
:1085F800074A75EEC85A36EE006A67EEA87AB0EEFA
:10860800667A95EE057AE5EE056AE5EE867AB1EECC
:10861800648AF0EE665AF0EE476AB1EE674AE8EE11
:10862800246A63EE270A67EEA43AE4EE275AB1EE0D
:10863800450AB0EE609AB0EE631AA4EE277A23EEEC
:10864800244AE7EEA76AA5EE249AA0EE031AE8EEFC
:10865800245AB0EE448A31EEA16AE0EE240AA5EE6F
:10866800278A66EEA16A72EE028AE5EE033A61EEA7
:10867800211A26EE096AA4EEA47AA0EE274A0CBFB6
:10868800D7ED022ADFED212A82ED005AA2EE256AF3
:10869800E8EEA06AE2EE081A73EEA33A27EE227A11
:1086A80034EE044AF0EE005AE3EEA26AA4EE226A1F
:1086B800A1EEA57AC7ED016AC1ED366A81ED356A8A
:1086C80087ED006A81ED377A82ED013AC2ED027AD0
:1086D800C2ED034AF3B987ED027A1BE05C6D03082B
:1086E800C0550020C4220020402200206C37002002
:1086F800F4460020982600201F85EB511C06002018
:108708002C06002064060020342000200000000011
:10871800DC4C0020BAF1000F40F024811DF0D2F9A2
:1087280017B0BDEC068BBDE8F08F079B1B78D90707
:108738007FF5D2AD4FF40F7023F09AFC00283FF478
:1087480028AE0CF055F94FF40F7023F027FC0028E1
:108758003FF41FAE0CF04CF94FF40F7023F01EFCE1
:108768000028EED115E69A4B0A931B689B077FF504
:108778001AADB5F8008018F0010F7FF438AD48F055
:10878800010398452B803FF432AD924B022214210D
:108798001A700E20FF2259709A702AF0EDF8B5F879
:1087A800008024E5059B5A8B9142C0F20685B1F5FD
:1087B800FA6FD4BFC2EB0101C2F5FA614FF47A73C4
:1087C80003FB01F184480378C2F5FA62B1FBF2F1C8
:1087D800002B3FF479AE4378804A01FB03F182FB1A
:1087E8000123C917C1EB63116EE6DFED7D7A2EE632
:1087F800DFED7B7A0DE6B1F5FA6F80F2D784187A4F
:108808008B1A03FB00F3C2F5FA6293FBF2F3C3F190
:10881800640307EE903AF8EEE77A9FED727A724BAE
:1088280067EE877AC3ED007AD0E51B780693002BB4
:108838007FF4BCAD6D4A1268002A3FF4B7AD6C4AAC
:10884800079212F8030CDFF8E0B11146D71E1CF0AE
:10885800BBFE9BF80090079A002800F03086069B24
:10886800B9F1000F53D107F1080178791CF0ACFE7B
:10887800002841F02D855F49B87A1CF0A5FE002834
:1088880000F03086B9F1020F41F01E855A49F87B95
:108898001CF09AFE002841F013855849387D1CF0D9
:1088A80093FE002800F03086B9F1040F41F00485EA
:1088B8005349787E1CF088FE002841F0F98451491C
:1088C800B87F1CF081FE002800F03086B9F1060F51
:1088D80041F0EA844C4997F823001CF075FE002803
:1088E80041F0DE84494997F828001CF06DFE002805
:1088F80000F03086B9F1080F41F0CE84444997F86A
:108908002D001CF061FE00283FF450AD09231A46E3
:1089180002EB820217443F4A7878B9788BF8003026
:108928001070517042E522F480739BB29A422B80FA
:108938007FF4AEAC384B1B78082B7FF4B8AC2A8890
:1089480022F040039BB29A422B803FF4B3AC214BF8
:10895800022214211A700E20FF2259709A702AF0F0
:108968000BF8A7E40C9B19780B9B01F00101186820
:10897800FBF79DFA17B0BDEC068BBDE8F08F13B975
:10898800089A01239370254B089A1D7892F8214084
:1089980007931B201CF042FE012C05F001088146BC
:1089A80000F0088705F00205089A1D4E92F820305D
:1089B800DFF878A01B4F09959346052B00F29E8798
:1089C800DFE813F0BE00B4003600FC00FE00F10042
:1089D800C048002010310020982600201F85EB5148
:1089E800000000000AD7233C40220020C455002084
:1089F800DE300020E8300020ED300020F23000208A
:108A0800F7300020FC300020013100200631002022
:108A18000B310020C8550020EC390020BF5500203C
:108A2800D44C0020104900200200002074060020C9
:108A3800012C04BF05238BF82030B8F1000F12D0A9
:108A4800059B3088B3F918100022134661F30F0212
:108A580060F31F4261F30F03049861F31F4303603F
:108A6800032342600993BF4DDBF814102A68914232
:108A780080F0028647F230510322CBF81C108BF8A5
:108A88002020022009F0C8F91AF020F92968DBF83B
:108A98001C200A440421CBF818208BF82010012C44
:108AA80040F07D872A68DBF81810914280F026870D
:108AB8009AF8000020B91CF0B1FD002840F01E878C
:108AC8003A6822F002023A602A687388642101FB3E
:108AD80003234FF480600022CBF810308BF820205D
:108AE8008BF8032009F068F99BF8203065E71CF043
:108AF8009BFD012807D19B4D72882B68642101FBDF
:108B08000233CBF81030B9F1000F02D0B379002B43
:108B18004BD1012C00F0F286924DDBF810102A6838
:108B28009142C0F0318701238BF82030012C3AD0D4
:108B3800F379012B46D01CF005FD9BF820303CE76B
:108B4800B8F1000FD3D1099D4FF48060B9F1000F3F
:108B580000F0568309F048F9089A00231361002DA4
:108B68003FF47CA9284629F007FF069B1E6816F4E7
:108B780080573FF479A91D217B48FCF774FE002833
:108B88007FF472A9794B03F1500A03E004339A4544
:108B980000F0BA861A78262AF8D19978DA789142BC
:108BA800F4D2FFF763B96F4D8EE71CF0CBFC0322BC
:108BB8004FF47A738BF82020CBF81C30694D60E7AE
:108BC800684D6CE71CF0BEFC032240F6B8338BF806
:108BD8002020CBF81C30634D53E7654F3B78002BC2
:108BE80001F05782634BDFF89881DFF898B1DFF81E
:108BF80098A1059345465E46049099460EE019F8FB
:108C080004109847032C28DC88B93B782AF8020F0F
:108C180001349C4205F1040580F24981072CE1B238
:108C28003046DBF80430EADD984700B2EDE738F863
:108C380024206B88801A4FF47A719B1A01FB00F08C
:108C480040F6CA0290FBF3F00844904240F2EE234B
:108C5800A8BF10469842B8BF184600B2D5E7DFF85B
:108C68002C91DFF82CA1444F0A9209F15A084FF0D1
:108C7800010B494619F8010C1CF0A6FC00B399F841
:108C8800040099F8023099F803E000EB400107EB83
:108C98008101013BD1F8A02003EB430353449342E5
:108CA8000ED097F8CC20C1F8A0300BFA00F022EAD9
:108CB80000000A9B81F89CE0C1F8A43087F8CC003A
:108CC80009F10609C145D4D12C4B264A1B780A93D1
:108CD800099BDFF8C0A012681B680B93AAF19C09D6
:108CE8004FF0000B9046DAF8043083B31F7877B35F
:108CF800DAF80820A8EB0202002A0CDB99F8CC204D
:108D0800012101FA0BF122EA010208F5FA7189F84A
:108D1800CC20CAF808100A9ACAB19AF800205978E3
:108D28000432D2B2002940F0B58305990498098B22
:108D380030F9122001F1C800824240F3F78599F812
:108D4800CC109A7841FA0BF3D80740F181860BF1E1
:108D5800010BBBF1040F0AF10C0AC4D1FFF715BAD5
:108D6800024B1DE09C5500203C3700202834002091
:108D7800F4340020204D0020342000202D3F002016
:108D880008350020204A002032200020F52F00203E
:108D980064540308D020002004339C423FF4F0A917
:108DA80019782329F8D19878DA789042F4D2AD4826
:108DB800FCF759FD00283FF4E3A9AB4B1B6813F4FB
:108DC800003341F013820022A84B1046995C142905
:108DD80002F10C0201F0BC8001301828F6D1FFF72F
:108DE800CFB91D219F48FCF73EFD28B100F060BDBA
:108DF8000436B4423FF48FAB31782629F8D1B278E3
:108E0800F3789A42F4D2089BDB78002B7FF483AB8B
:108E18009448FCF728FDDFED967A002801F0508190
:108E280038EE678A934A9449FDEEC87ACDED047A04
:108E3800BDF910301B0382FB0302DB17C3EBA21240
:108E4800C9F57A731BB203FB02F343F30F334B44A8
:108E580007EE903AF8EEE77A0123C7ED037A0B7034
:108E6800FFF759BB854C94F896305BB1079B1B788C
:108E7800DE0707D5049BB3F90620059B5B8B9A4256
:108E880000F3D88511217748FCF7EDFC002800F0A5
:108E9800AB8294F89A302BB994F8943013B93223F2
:108EA800A4F89830012384F89A30FFF727B9DDF841
:108EB8001090734A06926F49126842F2010AA1FBA8
:108EC800091B12EA0A0A4FEA9B1B00F08A826D4DC1
:108ED8006D486E4C6E492E780078267008701EB169
:108EE8006B490E7886F00106644C0F2184F8241033
:108EF800002B00F0E683059D664BB5F826C0B5F853
:108F080024E0059D109318462D8B0078624B12952E
:108F180094F825500995614D0495A3FB00535B080F
:108F280003EB4303C31ADBB20F90CDF834C002F44D
:108F380080520C9304F128000BF59673CDF84490F9
:108F480097F80080DDF82490DFF860C10994534C4D
:108F58000E91139200210A930896CDF81CE0089B05
:108F6800002B00F02B83099B079D33F911201FFA72
:108F780082FEAE454FEA410303D30D9DAE4540F254
:108F880062835CF82120934580F02283E25EBAF187
:108F9800000F40F0378301314145E25200F10600ED
:108FA800DDDB0E9A099C3E4B84F824200F2A4946A3
:108FB8000CBF01220022DDF8449084F825101A70B5
:108FC80000F08683374B3049314ADFF8E4B0089324
:108FD8001C46042001230B70137008F01DFFDBF8FA
:108FE8000030A1686268E3605B1A934284BF002383
:108FF80084F82130069B3C781E68002C01F04D80D7
:10900800059A294DB2F824E0178B244916F48056A6
:10901800284640F0998332460EE0437803EB8303F9
:1090280003EB830303F2EE239BB20132A24221F841
:10903800023B00F102000ED015F81230002B00F0B0
:109048000683022BE9D001320B8821F8023BA242A9
:1090580000F10200F0D1109A137801331370FEF773
:10906800E4BE00BF3C370020E82F00202C65030831
:1090780000007A44D34D6210B8220020342000202A
:109088000450002074320020300200202D3F0020C0
:1090980031020020DD330020ABAAAAAA967E002068
:1090A8001E4A00203C3F00203C350020E0330020D1
:1090B8009C550020D84CD4F88830A9EB0303002B2A
:1090C800FEF6C1AED54AD64B527C059933F812301C
:1090D8008A7DDFEDD46A9FEDD46AC97D9BB207EE25
:1090E800102A07EE903AB8EEC77AF8EEE77A27EE3C
:1090F800267A67EE867A0B9AC4F88820C7EE876AC4
:1091080040F2FF32FCEEE67ACDED077ABDF81C306E
:10911800934228BF134609B1D31A9BB2C348C44D22
:109128000178C44C35F81160226825F81130921B7B
:1091380013440131C04D236001F00F021B09027076
:109148002B80FEF780BEFEF753F9BC4BBC4A1B6868
:10915800C31A93427EF777AEB74B00221A80FEF708
:1091680072BE059A0499537DD27D013B31F91330C3
:109178001AB1C3F53B6308331BB2A3F57A7307EE44
:10918800903A9FEDB07AAC4AF8EEE77A40F2FF31B8
:1091980067EE877AFCEEE77ACDED077ABDF81C30EA
:1091A8008B4228BF0B461380FEF74DBE1B7AC3F1D6
:1091B800640307EE903AFFF72EBB4146FFF702BB68
:1091C8000221A148FCF74FFB00283FF410A82F808C
:1091D80018F0020F7FF41DA848F0020343452B80C6
:1091E8003FF417A8994B022214211A700E20FF226F
:1091F80059709A7029F0C0FBB5F80080FFF709B8DC
:1092080008F0DAFDA8E4924AB2F90030002BB8BFA2
:109218005B42B3F5E17FBFF62EA8B2F90230002B0E
:10922800B8BF5B42B3F5E17FBFF625A8894B93ED44
:10923800096AD3ED076A93ED057AD3ED037A76EEE2
:10924800866A77EE877A76EEA66AB7EE007A37EE08
:10925800666A77EEA77AB0EEC66AF0EEE75AB4EE21
:10926800E56AF1EE10FAB4BFB0EE655AB0EE465AB0
:10927800B5EE405AF1EE10FA40F0AD839FED767AE4
:10928800B4EEE56AF1EE10FA44BF9FED746A36EE6B
:10929800477AB7EE006AF4EEC66AF1EE10FAC8BF74
:1092A800DFED6F6AF5EEC07AC8BF36EEC77AF1EE29
:1092B80010FA48BFB1EE477AF6EE007A27EE677AE1
:1092C800DFED667A77EE276ABDEEE66A16EE103AAB
:1092D8002033402B40F25786DFED626A624ADFEDA9
:1092E800617AC2ED006AFDEEC76AC2ED017A16EE38
:1092F800903A2033402BC2ED027A49D8DFED587AF4
:10930800B4EEE77AF1EE10FA40F3E8879FED576A7A
:10931800DFED576A01E0B0EE677AB4EEE67AF1EE77
:1093280010FA77EE467AF6DC9FED527AF4EEC77AB9
:10933800F1EE10FA40F1E0879FED4C6ADFED4E6ADE
:1093480001E0F0EE477AF4EEE67AF1EE10FA37EE45
:10935800867AF6D4DFED417AB4EEE77AF1EE10FAC8
:1093680040F38186DFED3E7A37EEC77A27EE076A4B
:10937800DFED425ADFED426ADFED427AE6EE256A1A
:1093880067EE065AE6EE267AA5EEA77AF0EE477A59
:109398003D4BC2ED037A1A6812F4003240F054864D
:1093A8003A4B1046995C0A2902F10C0200F05185EB
:1093B80001301828F6D1FEF75EBF2A8822F0400354
:1093C8009BB29A422B803EF44FAF204B02221421CD
:1093D8001A700E20FF2259709A7029F0CDFAFEF704
:1093E80043BF2B490E787AE594F89430002B3EF46D
:1093F80085AE079B1B7813F001037EF47FAE012234
:1094080084F8943084F89520FEF778BE024C012148
:1094180084F88C10FEF7A3BD3420002014550020DA
:10942800345500200000C842000080441339002051
:109438001839002014390020343F00204823002028
:1094480060E316006F12833F3C3700201031002084
:10945800C44800203C060020A7DFA834DB0FC93F22
:10946800DB0F4940000000001C060020DB0FC9404C
:10947800E4CB1641DB0F49C0E4CB16C192E741B9F2
:109488009730083C15A82ABEE82F00202C65030851
:109498002D3F0020012900F0038599F8CC200123F5
:1094A80003FA0BF30BF1010B1343BBF1040F89F81B
:1094B800CC300AF10C0A7FF416ACFEF766BE511DDB
:1094C80078791CF081F800283FF4D5A9B9F1010F8B
:1094D80040F0FE8607F10D01B87A1CF075F80028F7
:1094E80040F0F286B549F87B1CF06EF800283FF48E
:1094F800D4A9B9F1030F40F0E386B149387D1CF0D7
:1095080063F8002840F0D886AE49787E1CF05CF8F5
:1095180000283FF4D4A9B9F1050F40F0C986AA493B
:10952800B87F1CF051F8002840F0BE86A74997F88C
:1095380023001CF049F800283FF4D4A9B9F1070F1B
:1095480040F0AE86A24997F828001CF03DF80028A4
:1095580040F0A2869F4997F82D001CF035F80028A6
:109568003EF424AFB9F1090F3EF420AFFFF7CEB9AE
:109578005D2A00F065855B2A00F06F825E2A00F0A4
:10958800F885562A00F00586972A00F07586A72ADE
:1095980000F0E585904D2B889B0740F0B285A2F13D
:1095A800B703072B00F28B82DFE813F07D028902F4
:1095B800890289027102890265026502079B002BF4
:1095C8003FD05CF8212093454FEA4103FFF4DEAC1D
:1095D800824A824DD25C05EB030E002A00F094808B
:1095E800022A47D19EF8012002EB820202EB820296
:1095F80002F2EE2292B2032933DD12B2BAF1000F61
:109608003FF4C9AC0C9D20F81520B9F1000F03D127
:109618000F9D022D7FF6BFACB0F802900288B0F81B
:1096280004E04A4496446E4A0FFA8EFE82FB0E52BC
:109638006C4DA2EBEE7225F803E012B24FF001096F
:10964800A9E41A464B000A9D4CF821509FE4D3B276
:10965800022B04D9032B7FF4F6AC7346E5E43B46B2
:10966800E3E4012505FA01FE0E9D25EA0E0512B276
:109678000E958CE4E25ABEE75B4A1278002A7FF422
:10968800F9A9B8F1000F3FF4F5A9012C40F0368193
:109698009BF82030FFF791B931465448FCF7E3F8BE
:1096A800002800F0C98084F8936019F0FDFDFEF7EA
:1096B800AEBC43F0400293422A807FF486AEFEF7A8
:1096C800D3BD4B4B4B4A109201221A704A4B04935C
:1096D8001B214648FCF7C7F800287FF473AC474BBA
:1096E800DFF820B108931946DBF80030CA688B60B0
:1096F8009B1AC82B00F2D584069B1E6806F4805678
:10970800A9E45B78FFF768B8CAB2022A40F2BC83C2
:10971800032AAFD1129A139D079E002D08BF324627
:1097280069E728F0010292B242452A803FF450AD21
:109738000E2087F8009087F801A087F802B029F07A
:109748001BF9B5F8008043E500220FE0437803EBEE
:10975800830303EB830303F2EE239BB20132A2429D
:1097680021F8023B00F102003FF475AC15F8123005
:109778001BB1022BEAD00B88F0E7D3B2032BFAD83F
:109788003B46EBE7B2F5FA7FFEF6B0AC94F89230C0
:10979800002B7EF4ABAC079B1B7801210B4084F8AF
:1097A800921000F0BA8319F091FA154B0A4D0993FB
:1097B800FEF79FBC0025FFF7F7B800BFED3000208B
:1097C800F2300020F7300020FC300020013100206A
:1097D800063100200B310020144900203C350020C0
:1097E80056555555A42000207C2200203C370020E7
:1097F8001E4A0020DD330020967E00203C3F0020DA
:109808001C4900209C550020B2F5FA7FFEF66EAC8C
:1098180094F89230002B7EF469AC079A12780121F3
:10982800D70784F8921000F1178419F03DFDC24B58
:10983800C24D0993FEF75DBC079BC14A1B781060B7
:10984800DB077EF5E8ABBF4B1B78002B3EF44EAC34
:10985800089BDB78002B7EF449AC94F893300133F5
:10986800DBB2032B84F893307EF640ACB64B5B78C2
:1098780013B9002D7EF43AAC19F028FAFEF7C7BBED
:10988800B24AB3491068B4F99020C66981FB060151
:109898008911F617701A00F5FF407F3082423EF7B3
:1098A800A9AB891B0A4412B2A4F89020FEF7A2BB08
:1098B800089BDB78002B7FF49FAADFEDA67AA449EA
:1098C80038EE678AC9F5FA63FDEEC87A1BB2CDEDAA
:1098D800047ABDF91020120381FB0201D217C2EBF2
:1098E800A11203FB02F343F30F334B4407EE903A04
:1098F800B8EEE78A87ED038AFFF77EBA099D002D47
:109908003EF4ACAAFFF72EB9934A059BD588049A72
:109918001B8BB2F906105A1B914240F388802B44E6
:109928009942B4BF00250125FEF7A9BAC8398A4271
:1099380042DA99F8CC109A7841FA0BF3D9073FF537
:1099480006AA524201200C9229F0FCF87B1E0C9AC0
:10995800162B00F28281DFE813F004021802EC01F2
:109968003D022C025102D701C201AD0198018301C9
:1099780080013D0272015102D701C2015D01490116
:10998800350166021F01DA001BF0DCFD032140F6F9
:10999800B8328BF82010CBF81C20FFF772B8AB4612
:1099A8000899DBF80020CB69099D13448B61002DD1
:1099B8003EF454AAFFF7D6B899F8CC30012202FA3F
:1099C8000BF223EA020308F5FA7289F8CC30CAF8D8
:1099D8000820FFF7BCB9B4EEE56AF1EE10FA8CBFC7
:1099E800B0EE654AB0EE464AC4EE054A9FED5B2AE2
:1099F8009FED5B5ADFED5B1ADFED5B2A9FED5B3A6B
:109A0800DFED5B3A9FED5B4AA4EE825AE4EEE12A71
:109A1800A4EE857AA4EEA23AB0EE475AB0EE637A85
:109A2800A4EE837AA4EE874A84EE057A28E4012519
:109A3800FEF725BA00215048FBF715FF00287FF4F0
:109A480021AA322384F89600A4F89830FFF71ABAAE
:109A5800002A0CBF0120022075E7484B0122022092
:109A68004749484C0B60344B2270344D099329F018
:109A780069F8FEF73EBB304A424B09921146424A0A
:109A88000A6002225A701BF02DFEFEF732BB2A4AEA
:109A98003C4B099211463D4A0A6000225A701BF05D
:109AA80021FEFEF726BB244A364B09921146384A56
:109AB8000A6001225A701BF015FEFEF71ABB792ABC
:109AC80000F082847A2A00F076849E2A00F06B8463
:109AD8009D2A00F06084AE2A00F05584AD2A00F07B
:109AE8004A84EF2A00F04484FD2A00F03E84FB2AD1
:109AF80000F02B84FE2A00F07084F72A00F07884A6
:109B08007B2A00F01B840C4B0993FEF7F2BAD9F8B4
:109B1800D000204B90F836109B7811446429A8BFD8
:109B2800642121EAE17180F83610002B40F0998415
:109B380023F090FDB1E400BF1C4900201449002027
:109B4800984B00202D3F00209437002034450020FA
:109B5800D34D621000007A44BC4C002099FB243F8E
:109B680069A2163E39094E3DE3B59E3E88FA163E77
:109B780045FE7F3FA7DFA8343C370020E85200208D
:109B88001849002084490020A84900209049002055
:109B98009C490020BA530020D9F8D000BC4B90F85B
:109BA80037109B781144FE29A8BFFE2121EAE171F4
:109BB80080F83710002BBBD016201BF079FDD9F8A0
:109BC800D000B5E7D9F8D000B14B81781144C82945
:109BD800A8BFC82121EAE17181709B78002BA7D02A
:109BE80014201BF065FDD9F8D000A1E7D9F8D00002
:109BF800A74B41781144C829A8BFC82121EAE171BF
:109C080041709B78002B93D013201BF051FDD9F89D
:109C1800D0008DE7D9F8D0009D4B01781144C829B0
:109C2800A8BFC82121EAE17101709B78002B3FF49D
:109C38007FAF12201BF03CFDD9F8D00078E7944B99
:109C48000B989B78417911446429A8BF642121EAC3
:109C5800E1714171002B40F0F383D9F8D00067E738
:109C6800D9F8D0008A4B017A9B781144C829A8BF3B
:109C7800C82121EAE1710172002B3FF459AF0B2092
:109C88001BF016FDD9F8D00052E7D9F8D000804B68
:109C9800C1799B781144C829A8BFC82121EAE1717C
:109CA800C171002B3FF444AF0A201BF001FDD9F825
:109CB800D0003DE7D9F8D000754B81799B781144E5
:109CC800C829A8BFC82121EAE1718171002B3FF49E
:109CD8002FAF09201BF0ECFCD9F8D00028E7D9F801
:109CE800D0006B4B417993F802E01144C829A8BF12
:109CF800C82121EAE1714171BEF1000F40F08E8365
:109D0800112F7FF462AF13E7D9F8D000604B0179C7
:109D180093F802E01144C829A8BFC82121EAE171DB
:109D28000171BEF1000F40F09283102F7FF461AFF4
:109D3800FEE60B99564B0F790C931744642FA8BF76
:109D4800642727EAE7770F711BF0CCFC0C9B9B7804
:109D5800002B82D0032039461BF0AAFCD9F8D0008A
:109D6800E6E60B984A4B01781144FA29A8BFFA2174
:109D780021EAE17101709B78002B3FF46EAF01205E
:109D88001BF096FCD9F8D000D2E60B98404B8178AE
:109D980011446429A8BF642121EAE17181709B788C
:109DA800002B3FF45AAF02201BF082FCD9F8D000F8
:109DB800BEE60B98364BC1799B78114481F30801B4
:109DC800C171002B3FF449AF05201BF071FCD9F895
:109DD800D000ADE60B982E4B817993F802E0114440
:109DE8006429A8BF642121EAE1718171BEF1000FE5
:109DF80040F01E830D2F7FF423AF2EE7D9F8D00053
:109E0800234BC17893F802E01144C829A8BFC821A0
:109E180021EAE171C170BEF1000F40F027830F2FD6
:109E28007FF4FBAE84E60B98194B41781144B1F5E9
:109E3800967FA8BF4FF4967121EAE17141709B7833
:109E4800002B3FF40AAF15201BF032FCD9F8D000E4
:109E58006EE61049D1F800E04200BEF1000F08D0CC
:109E6800171803EB87079EF801E07F787745BEF463
:109E780002AA1044084F094A03EB800300200B6034
:109E880038801060FEF7F7B9129AFFF7B4BB00BF2D
:109E9800BA53002038220020202300202423002049
:109EA80004999B7831F91220B2F5617F4FF49661DD
:109EB80091FBF3F3C0F2E48040F633019142A8BF6E
:109EC80011460C2FA1F5617191FBF3F100F0778138
:109ED800182F7FF4E2AAC9B2C8290B46A8BFC82325
:109EE800D9F8D020D77DD8B2B8423FF4D6AADF1B24
:109EF800C44BD07548BF0737FF109B780137FFB2B6
:109F08003BB9002F3FF4C9AA384628F01BFEFFF7DB
:109F1800C4BA18201BF0CCFBF3E7BB49096811F45D
:109F2800003140F04581B94B08465D5C0F2D01F1C9
:109F38000C0170D001301828F7D10023FA3A84F8C0
:109F48009230B34BA4F89020B24D0993FEF7D1B8E4
:109F5800B149D1F800E04200BEF1000F08D017184F
:109F680003EB87079EF801E07F787745BEF408A9E0
:109F78000244AA4FAA4803EB820300220B603A80EE
:109F88000260FEF7FDB8B4EEE77AF1EE10FA40F39E
:109F9800AC81DFEDA45A9FEDA46A01E0F0EE676A98
:109FA800F4EEC66AF1EE10FA76EEE57AF6DCDFED4D
:109FB8009F6AF4EEE67AF1EE10FA40F19381DFED54
:109FC800995A9FED9B6A01E0F0EE667AF4EEC67A44
:109FD800F1EE10FA77EEA56AF6D4DFED967AF4EE94
:109FE800E76AF1EE10FA40F3C880DFED937A77EE76
:109FF800E66A66EEA65A9FED915A9FED916ADFEDEB
:10A00800917AA5EE856A26EEA55AE5EE867AE5EE02
:10A01800276AFFF763B980490F68450037B12E18E2
:10A0280003EB86067F787678BE4286D205447B4E5F
:10A038007B4803EB850300250B60358005607CE7D2
:10A04800814B002201200BE5804B1B78032B00F08D
:10A058001F810022FFF7A4B97D4A6E4D13606C4B37
:10A068000993FEF746B8DFED7B7AB4EEE77AF1EEB6
:10A0780010FA44BFDFED6D7A37EEC77AFFF776B98D
:10A088000C2F00F0BC80182F7FF407AA00210B4684
:10A0980026E7714A0592FEF70CBF06F48056FEF7D4
:10A0A800DABF6E4A069B1E68136823F00403136028
:10A0B800089A012306F4805682F82130FEF7CBBFB8
:10A0C80038EE678A664B67491870FDEEC87AC9F59D
:10A0D800FA63CDED047ABDF91020120381FB020169
:10A0E800D217C2EBA1121BB203FB02F343F30F33E7
:10A0F8004B4407EE903AF8EEE77AC7ED037AFEF79D
:10A108000ABA0023BB2A149300F0BF80B72A00F0D4
:10A11800EF80BE2A00F0E080BD2A7FF4D0AC4FF675
:10A12800FE71514A3A48D6890990908933440144CE
:10A13800D38191810FF03CFDFAF70AFD0FF020FD65
:10A14800FCF74CF8012028F0FDFCB4F89030002210
:10A15800FA3BA4F8903084F89220FDF7CABF434A2E
:10A168002C4D137843F004031370294B0993FDF722
:10A17800C0BF3F4B0222032072E4DFED367AF4EED3
:10A18800E76AF1EE10FA44BFDFED287A77EEE66A67
:10A198002FE70FF00DFDFAF7DBFC0FF0F1FCFCF7F1
:10A1A8001DF8012028F0CEFC94F88E20FFF7ECB9BA
:10A1B80026490978032900F0A3801946B3E6CFB2EF
:10A1C8002C4B0D915B78BB423FF467A90D4B0C9368
:10A1D800384619F009FF0C9B0D999B781BB1C9B241
:10A1E8000C201BF065FA0137FFB28AE6174B1B7883
:10A1F800032B7EF4E8AD28F0A3FBFDF7C1BF0027D1
:10A208003946DDE7BA530020E82F00202C65030803
:10A218001C49002014490020382200202023002057
:10A2280024230020DB0FC940E4CB1641DB0F49C0D3
:10A23800E4CB16C1DB0FC93FDB0F494092E741B9B8
:10A248009730083C15A82ABE9A520020373F0020B4
:10A25800984B0020DB0FC9BF204D0020104900207B
:10A26800B8220020D34D621074370020F83900203E
:10A278003653002084490020814B824D4FF4C87228
:10A288001A80814B0993FDF734BF1946022348E72A
:10A2980028F056FBFDF7EFBF08231A46FEF738BB38
:10A2A80007231A46FEF734BB06231A46FEF730BBCF
:10A2B80005231A46FEF72CBB04231A46FEF728BBD3
:10A2C80003231A46FEF724BB02231A46FEF720BBD7
:10A2D80001231A46FEF71CBB022122E7F0EE477A5B
:10A2E800FFF722B8F0EE676A77E6F0EE667A5EE688
:10A2F80019464FF6FE7314E7B0EE677AFFF72AB8EF
:10A3080028F01EFBB4F9902017E65F4B84F89410F0
:10A3180084F895005B4D0993FEF7A5BD002D3DF42B
:10A32800F2AD5A4C94F88D30002B3DF41DAE28F058
:10A3380007FB002384F88D30FDF716BE4FF4FA6151
:10A34800022019F079FDFFF7DEBB0021022019F089
:10A3580073FDB4F890304C4A0992963B0022A4F859
:10A36800903084F89220FDF7C4BE00210120EEE76A
:10A3780000210846EBE7FF21002020F063FB94F85A
:10A388008E20FFF7AEBB0121002020F05BFB94F884
:10A398008E20FFF7A3BB0021FF2020F053FB94F889
:10A3A8008E20FFF798BB0021012020F04BFB94F88A
:10A3B8008E20FFF78DBB364A334B0993137A43F04F
:10A3C80001031372FDF795BE314A2F4B0993137A97
:10A3D80023F001031372FDF78CBE00210320B6E7BA
:10A3E8002A4C18F073FC002384F88D30FDF7BCBDAF
:10A3F80000210420ABE7002B93D02649264A0968A0
:10A408004FF47A7000FB031313608AE70B2028F0DF
:10A41800B3FA1D4B1B4D0993FDF76BBE11200D932D
:10A428000C921BF045F9D9F8D0000D9B0C9A67E403
:10A438000D200D930C921BF03BF90D9B0C9AD9E45F
:10A448000E201BF035F9D9F8D000FFF771BB1020AA
:10A458000D930C921BF02CF9D9F8D0000D9B0C9A97
:10A4680063E417201BF024F9FFF7F7BB0F200D93C7
:10A478000C921BF01DF9D9F8D0000D9B0C9ACEE474
:10A48800F64C0020144900201C49002034200020EC
:10A49800044A00209C550020944B00202DE9F04FE1
:10A4A8002DED0E8BDFF8F4B093B0DBF804200490A8
:10A4B80058469047002800F08E82BBF8A87000210B
:10A4C8008BF85110002F6DD1BBF93A00DBF82450FE
:10A4D800DBF82810BBF93860DBF82040BBF93C20DA
:10A4E800DFF8BCA0401B521ACBF830009BF8521082
:10A4F800CBF83420341B0BF12C00CBF82C4013F094
:10A508005DFDDAF80020910041F1B587DBED0C5ACA
:10A518001F4CDBED0B7A1F4994ED406AD4ED416A7C
:10A5280094ED427AD4F80C2109681B4B0293B8EEDB
:10A53800E58ADBED0D5AF8EEE77AF8EEE58A0132A6
:10A5480077EE867A38EE268A78EE878A8A42C4EDD4
:10A55800407A84ED418AC4ED428AC4F80C2101F0A6
:10A568004E8393F800E0BEF1140F02F090870023A9
:10A57800D4F814510393062D01F29B84DFE815F0FB
:10A58800F815BA161B15CD16060C37177D1500BF22
:10A5980014210020FC390020D44600207C4D0020E6
:10A5A80004500020DE4BDF481A6805934FF47A7593
:10A5B800B5FBF2F2C2EB421502EB8502D500DA4B8D
:10A5C800DFF8C88344780293ADB2AF421E78B8F979
:10A5D800060003F07680DBF87C30BBF93810DBF836
:10A5E800602003F1010E07EE901A0A44BEF1010F34
:10A5F800CBF87CE0CBF86020F8EEE77A03F06E80C9
:10A60800DBED1B5ADBED1D6A07EE10EA37EEE56A53
:10A61800B8EEC75A012F86EE057A37EE257A77EE1F
:10A62800C77A8BED1C7AE7EE866A8BED1B7AF0EE23
:10A63800667ACBED1E6ACBED1D6A03F00B84DBF85E
:10A648009030BBF93A10DBF8642003F1010E07EEF5
:10A65800901A0A44BEF1010FCBF890E0CBF86420C1
:10A66800F8EEE77A03F05580DBED205ADBED226A3D
:10A6780007EE10EA37EEE56AB8EEC75A012F86EE04
:10A68800057A37EE257A77EEC77A8BED217AE7EEF1
:10A69800866A8BED207AF0EE667ACBED236ACBEDF5
:10A6A800226A03F0AF83DBF8A430BBF93C10DBF877
:10A6B800682003F1010E07EE901A0A44BEF1010F5B
:10A6C800CBF8A4E0CBF86820F8EEE77A03F03C80FA
:10A6D800DBED255ADBED276A07EE10EA37EEE56A6F
:10A6E800B8EEC75A012F86EE057A37EE257A77EE4F
:10A6F800C77A8BED267AE6EE276A8BED257AF0EE9F
:10A70800667ACBED286ACBED276A03F06E83874C17
:10A71800A8F80600BBF8A820029B013A1E78ABF8FF
:10A72800A82005990022072E4A608A60CA6040F076
:10A738005981FCF75DFE029BDFF850821E78049B6E
:10A74800C01A94F82831A8F800000693002B40F0AE
:10A758004F81744A5279002A01F07E81744A127836
:10A76800013AD2B2072E84F8282102F0EC810023A6
:10A778000793704BD4F83421D3F800A0684B0593A5
:10A78800049B9FED6D6AD4ED4C9A6C49C4F8343142
:10A798009A1A07EE902AF8EE677AB7EE007AC6EEB4
:10A7A800278A0025664BDFF8E891DFF8E881654FD6
:10A7B80003932E46D1ED006A94ED4BDA9FED629A31
:10A7C800DFED62AA9FED62CA9FED62AADFED62BA71
:10A7D8009FED62BA77EE69CA6CEEA6CAF4EEC7CAF4
:10A7E800F1EE10FA88BFF0EE47CA5D4B99ED008A8A
:10A7F8002B44D3ED007AF5EE407AF1EE10FA17D03B
:10A80800584B2B4493ED007A78EE476AB0EEE66A2F
:10A81800F4EEC67AF1EE10FA08D5F5EEC06AF1EE5C
:10A8280010FACCBF37EE878A37EE678A83ED008A45
:10A838004D4B1A88930739D0022E37D09AF82E102C
:10A848004A4B07EE901A2B4493ED007A4B42F8EEF0
:10A85800E76A07EE903A26EE877AF8EEE77AB4EEE2
:10A86800E77AF1EE10FA0AD407EE901AF8EE677A52
:10A87800F4EEC77AF1EE10FA88BFF0EE477A3C4B57
:10A888003C4903EB460331F91600B3F90C30C31AFF
:10A8980007EE103AB8EEC77AD007E7EE497A41F1E9
:10A8A8007780354B93ED008A27EE888A059B94F8CC
:10A8B80068212B4493ED01EA78EE4EDA002A00F085
:10A8C800F7802E4BD4F86C2104991B688A1A9A4297
:10A8D80040F3EE809AF84830022B02F08381022E72
:10A8E80004F04F84264B1B68990700F19780254B8D
:10A8F80087ED00CA1B689342C0F2CA80F7EE007A5F
:10A90800F4EEE79AF1EE10FA40F1D28005991E4B69
:10A91800D1ED017A93ED007AF0EEE77A3CE000BFE2
:10A92800F44F0020684D0020D44600201421002058
:10A938006837002018490020002474492471002039
:10A94800803900208C390020CDCCCC3DAE47813FEA
:10A95800000000000000C84200003443610BB63B11
:10A968001871002058220020144900206422002079
:10A9780074370020C4480020007100202C7100208A
:10A98800C04800202871002034710020D8460020DB
:10A998004C22002098390020F4EEC77AF1EE10FA24
:10A9A80040F18680D1ED027AF0EEE77AB4EEE77AEC
:10A9B800F1EE10FA7CDDD1ED037AF0EEE77AB4EE31
:10A9C800E77AF1EE10FA73DD0F4B1B689B075FD532
:10A9D8000E490F4B43E00F4B0F4C1E780293072E86
:10A9E8003FF4A7AE94F828310693002B3FF4B1AE9C
:10A9F800013B84F82831012E01F0AD8213B0BDEC83
:10AA08000E8BBDE8F08F00BFC0480020C44800206E
:10AA180074370020D446002014210020D34BD44999
:10AA2800DFF8C8E331F916C09EED008ADFF8C0E30D
:10AA380087ED00CA03EB460028EE098AB0F90C003E
:10AA4800A0EB0C0007EE900AF8EEE77ADEF80000BB
:10AA580027EE888A904278EE4EDABFF64FAFB3F908
:10AA68000C20B1F900E0C348AEEB020E00688EEA94
:10AA7800EE72A2EBEE7282421ADAB3F90E30B1F935
:10AA88000220D21A82EAE273A3EBE27398420FDD46
:10AA9800B94B1A88002384F86831002A43F072857C
:10AAA800B64AB74B1178186881F00101F9F7FFF938
:10AAB800B44B2B4493ED000A039B2DEE000A022EA3
:10AAC80020EE2D0AA3EC010A039304F0D383AE4BC6
:10AAD800D7ED006A93ED007AAC4BD3ED007AAC4B1E
:10AAE80093ED006AAB4B67EE277A2B4427EEAC7ADE
:10AAF800D3ED007A67EE277AF0EE665AEDEEA75AA4
:10AB0800B1EE467AB4EEE57AF1EE10FA08DCB4EE6E
:10AB1800E56AF1EE10FA8CBFB0EE657AB0EE467ACF
:10AB280094ED4C6AF7EE007AB4EEE76AF1EE10FAAB
:10AB3800ACBF0123002343B1F0EEE66AF0EEC77A1A
:10AB4800F4EEE67AF1EE10FA01D587ED007A022EDE
:10AB580004F0C782904A914B52F826001B68B0EE69
:10AB68004E0A98478E4A8F4B52F826001B68984722
:10AB78009AF8373023B18C4B1B88002B00F06F8775
:10AB8800B0EE4C8A894B38EE400A2B4493ED008A8C
:10AB980083ED000A9AF8483030EE480A20EE288AF9
:10ABA800002B33D0824B1B7813F0010300F0BB86D7
:10ABB800F7EE007AF4EEE79AF1EE10FA94F86831BD
:10ABC800C1F20885002B00F0EF87D4F86C31049AA5
:10ABD800D31A784A12689A4218DD774BD3ED007A77
:10ABE800F0EEEDDAF4EEE7DAF1EE10FA42F10B806E
:10ABF800614B1A88002384F86831002A00F09F8688
:10AC08006E494A6912B10A6813604B746C4B94F828
:10AC180078212B4493ED000A2DEE000A20EE088AD5
:10AC280088ED008A32B9039B87ED00CA03ED01CA9B
:10AC380088ED00CA0136032E09F1040908F1040859
:10AC480007F1040705F104057FF4CFAD029B1A78DC
:10AC5800072A01F0C484012A01F0628700230393C4
:10AC680094F88021002A41F0A981DFF888A1554B8A
:10AC7800DAF800201968D60491F82C0000F10A8748
:10AC8800DFF87491504AB9F81A3092ED006A4F4AC9
:10AC98004F4ED2ED005AD6ED036A4E4A84ED646AEF
:10ACA80007EE103A4C4B92ED005AD3ED007AD3EDF3
:10ACB800013AD3ED024A84ED626AB8EEC77A35EEFE
:10ACC800C64A012236EEC77A84ED614AC4ED655A58
:10ACD80084F89821C7EE055A0A8D534206EE103AB9
:10ACE8003E4BDFED3F6A93ED005A3E4B93ED004A31
:10ACF800B7EE007AF4EEC75A35EE045AF1EE10FAC0
:10AD080088BFF0EE475A35EE275AB8EEC66AF4EE19
:10AD1800E65AF1EE10FA07EE902AB4EEC65AB8BF1A
:10AD2800F0EE665AF1EE10FAC4ED685AB8EE677A9A
:10AD380001F13083B4EEC75AF1EE10FA88BFB0EED5
:10AD4800475A264BDFED286AD3ED017A254B93ED60
:10AD5800014A77EE847A25EE265A77EEA37AB4EE86
:10AD6800E76AF1EE10FA52DC48E000BF74370020C1
:10AD7800C44800203071002074550020765500200A
:10AD880078550020D47000201070002004000020A6
:10AD980048710020E0700020187000201470002016
:10ADA8006C70002068700020144900208422002064
:10ADB800BF5500202C710020387100207C550020E0
:10ADC800EC70002018490020E435002048370020A6
:10ADD800F4460020C44C00208C3900208039002023
:10ADE80000000000983900206F12833A007100209B
:10ADF8002871002004500020204D0020B4EEE77A8E
:10AE0800F1EE10FA8CBFB0EE676AB0EE476AED4B10
:10AE18004A8DD3ED027A9FEDEC7A534204EE103A54
:10AE280074EEA77AB8EEC44A26EE076AF4EEC47A3E
:10AE3800F1EE10FA0AD407EE102AB8EE474AB4EE3B
:10AE4800E74AF1EE10FA88BFB0EE674ADF4ADFED55
:10AE5800DE7A527824EE274A0AB9B1EE444A00282D
:10AE680041F00286B7EE003AD94E3278002A02F055
:10AE78003886D849DFEDD87AD1ED024AD1ED016A9A
:10AE880091ED037A66EE244AE5EE264AE4EE074A97
:10AE980063EE244AF4EEE74AF1EE10FAB4BFF0EE9E
:10AEA800673AF0EE643A98BFF0EE647A012ACDED85
:10AEB8000A4A02F0638691ED067AD1ED052AD1EDB2
:10AEC800076A26EE077AA5EE227AA4EE267A23EE02
:10AED800077AB4EEE77AF1EE10FAB4EEE37A8CBFB3
:10AEE800F0EE676AF0EE476AF1EE10FA88BFF0EE0E
:10AEF800676AB4BFF0EE637AF0EE477A022A8DED06
:10AF08000B7A00F0DE8091ED0A7AD1ED092AD1EDB5
:10AF18000B3A26EE077AA5EE227AA4EE237A23EEE0
:10AF2800077AB4EEE67AF1EE10FAB4EEE77A8CBF5F
:10AF3800F0EE663AF0EE473AF1EE10FA98BFF0EE0E
:10AF4800636AA8BFF0EE477A032A8DED0C7A00F009
:10AF5800B88091ED0E7AD1ED0D2AD1ED0F3A26EE9B
:10AF6800077AA5EE227AA4EE237A23EE077AB4EEC6
:10AF7800E67AF1EE10FAB4EEE77A8CBFF0EE663AB4
:10AF8800F0EE473AF1EE10FA98BFF0EE636AA8BF08
:10AF9800F0EE477A042A8DED0D7A00F09280D1ED1B
:10AFA800123AD1ED112A91ED137A66EE233AE5EEC5
:10AFB800223AE4EE073A63EE233AF4EEE63AF1EE8B
:10AFC80010FAF4EEE73A8CBFB0EE667AB0EE637A28
:10AFD800F1EE10FA98BFF0EE476AA8BFF0EE637A78
:10AFE800052ACDED0E3A6CD0D1ED163AD1ED152AE1
:10AFF80091ED177A66EE233AE5EE223AE4EE073A47
:10B0080063EE233AF4EEE63AF1EE10FAF4EEE73A9C
:10B018008CBFB0EE667AB0EE637AF1EE10FA98BFA4
:10B02800F0EE476AA8BFF0EE637A062ACDED0F3A34
:10B0380047D0D1ED1A3AD1ED192A91ED1B7A66EE77
:10B04800233AE5EE223AE4EE073A63EE233AF4EEC9
:10B05800E63AF1EE10FAF4EEE73A8CBFB0EE667A13
:10B06800B0EE637AF1EE10FA98BFF0EE476AA8BF27
:10B07800F0EE637A072ACDED103A22D091ED1E7AD0
:10B08800D1ED1D2AD1ED1F3A26EE077AA5EE227AD8
:10B09800A3EE847A27EE037AB4EEE67AF1EE10FA9C
:10B0A800B4EEE77A8CBFB0EE666AB0EE476AF1EEAE
:10B0B80010FA8DED117A98BFF0EE466AA8BFF0EE4F
:10B0C800477A77EEE67AF7EE006AF4EEE67AF1EE82
:10B0D80010FAC4ED4C7A43F3848586EEA77A022AE7
:10B0E800DDED0B7A67EE244A67EE877ACDED0A4AE2
:10B0F800CDED0B7A2DD0DDED0C7A67EE877A032A39
:10B10800CDED0C7A25D0DDED0D7A67EE877A042A2D
:10B11800CDED0D7A1DD0DDED0E7A67EE877A052A22
:10B12800CDED0E7A15D0DDED0F7A67EE877A062A17
:10B13800CDED0F7A0DD0DDED107A67EE877A072A0C
:10B14800CDED107A05D0DDED117A27EE877A8DEDF9
:10B15800117A2249096811F0805801F0EE81F6EE63
:10B16800005AC4ED685A002A02F0B5841C4B94EDCD
:10B17800656A1C491C4F1D78DFF874E094F9983112
:10B1880094ED645AB7F90670C878DAF80010DEED65
:10B19800004A0597BDEEC66A07EE103AB9F81A706C
:10B1A800124B079716EE10EABDEEC56A05F0010CC2
:10B1B80001F4805701F0100501F4800108911B7813
:10B1C80018E000BF803900206F12833AEC39002064
:10B1D80082460020344C0020000000003C3700204C
:10B1E800BF5500203C3F0020967E00204458002098
:10B1F800304C0020D4ED616AD4ED627AB8EEC77A9B
:10B2080016EE101A002840F02D87002D41F0FB8221
:10B21800D24D9DED0A5A95ED006AD14825EE866A11
:10B22800A5EE076AB0EE675AA6EE265ABDEEC56AC5
:10B2380016EE108A16EE107AF045A8BF77464145FB
:10B24800C8BF0F4606EE107AB8EEC66A012A80ED2E
:10B25800006A00F0DC8095ED046A9DED0B5A25EE3E
:10B26800866AA5EE076AB0EE675AA6EE265ABDEEC4
:10B27800C56A16EE108A16EE107AF045A8BF774612
:10B288004145C8BF0F4606EE107AB8EEC66A022AD4
:10B2980080ED016A00F0BB8095ED086A9DED0C5ABF
:10B2A80025EE866AA5EE076AB0EE675AA6EE265A1C
:10B2B800BDEEC56A16EE108A16EE107AF045A8BFE4
:10B2C80077464145C8BF0F4606EE107AB8EEC66A03
:10B2D800032A80ED026A00F09A8095ED0C6A9DEDD4
:10B2E8000D5A25EE866AA5EE076AB0EE675AA6EEF5
:10B2F800265ABDEEC56A16EE108A16EE107AF0458B
:10B30800A8BF77464145C8BF0F4606EE107AB8EE8B
:10B31800C66A042A80ED036A79D095ED106A9DED1E
:10B328000E5A25EE866AA5EE076AB0EE675AA6EEB3
:10B33800265ABDEEC56A16EE108A16EE107AF0454A
:10B34800A8BF77464145C8BF0F4606EE107AB8EE4B
:10B35800C66A052A80ED046A59D095ED146A9DEDF8
:10B368000F5A25EE866AA5EE076AB0EE675AA6EE72
:10B37800265ABDEEC56A16EE108A16EE107AF0450A
:10B38800A8BF77464145C8BF0F4606EE107AB8EE0B
:10B39800C66A062A80ED056A39D095ED186A9DEDD2
:10B3A800105A25EE866AA5EE076AB0EE675AA6EE31
:10B3B800265ABDEEC56A16EE108A16EE107AF045CA
:10B3C800A8BF77464145C8BF0F4606EE107AB8EECB
:10B3D800C66A072A80ED066A19D095ED1C6A9DEDAC
:10B3E800115A65EE865AE7EE055AE6EEA57AFDEEA5
:10B3F800E77A17EE905AAE45A8BFAE46A942D8BF25
:10B40800714607EE901AF8EEE77AC0ED077ABCF1BC
:10B41800000F00F03487534A1268002A40F03C8736
:10B42800514A127892B1307868B14D4FDFF858819F
:10B438000025E8B2D8F80030B7EC010A9847307810
:10B4480001358542F5DB494A12689047029B1A7814
:10B45800072A01F0DA800025DAF80020530501F107
:10B468000E80434B1B78BBB1424AB9F81A30B2F987
:10B4780006209A4210DC404B1B78012B01F07883A0
:10B48800192B01F075830E2B06D0082B04D03B4EE8
:10B498000023B360C4F8403194F8AA6126B1384B50
:10B4A8001B889F0741F0268394F8B021002A40F0BA
:10B4B800858799F81E70002F00F02E84022F01F066
:10B4C8000883032F41F0018399F82030C3EB43111F
:10B4D80003EB8101C90089B299F81F300233DBB24E
:10B4E800002A00F08185002900F07E85254807683C
:10B4F800B1FBF7F10FB2A4F8E071002B03F0528012
:10B5080007EE907AF8EEE77AF7EE006A86EEA77A09
:10B518001A4E012BD4ED7D6AD6ED007A77EEE67AE5
:10B5280067EE877AC4ED797A3AD0D6ED017AD4ED10
:10B538007E6A77EEE67A022B67EE877AC4ED7A7A2E
:10B548002ED0D6ED027AD4ED7F6A77EEE67A032B19
:10B5580067EE877AC4ED7B7A22D017E0344C00205E
:10B56800B43900200C7000206C5B0020405800208B
:10B5780074060020967E0020EC390020F446002056
:10B5880014490020D439002038580020D6ED037A19
:10B59800D4ED806A77EEE67A67EE877AC4ED7C7A36
:10B5A80002990978092903F03981002F40F3BA83F9
:10B5B8009BB394ED7D7AD4ED797A77EE877A012B77
:10B5C800C4ED7D7AC6ED007A21D094ED7E7AD4ED73
:10B5D8007A7A77EE877A022BC4ED7E7AC6ED017A05
:10B5E80015D094ED7F7AD4ED7B7A77EE877A032BAA
:10B5F800C4ED7F7AC6ED027A09D0D4ED807A94ED55
:10B608007C7A77EE877AC4ED807AC6ED037A013BBF
:10B61800022BB8BF0223DBB20693069B002A18BF91
:10B6280002239E46CB4BDFEDCC6A1A68029B9178C9
:10B638001878137807EE903AF8EEE77AB0EE007AC9
:10B6480067EEA67AF4EEC77AF1EE10FA40F38D862B
:10B65800DFEDC26A37EEC77AB0EE676AA7EE266AF0
:10B66800F0EE466A96ED007A9FEDBD6A27EE066A0F
:10B67800F0EEC65A84ED546AC4ED575A99B107EEF4
:10B68800101AB8EEC75A9FEDB47A66EE064A25EE50
:10B69800075AB7EE007A37EE457A64EEA54AA4EE6B
:10B6A800857A26EE076A9FEDAF7A537926EE877A78
:10B6B80027EE067ACBB1DFEDA86A9FEDAB6A65EE9F
:10B6C800A65A06EE903AF8EEE66A66EEA56AF4EE39
:10B6D800C66AF1EE10FA01F39E81F7EE005A75EE94
:10B6E800E66A85EEA66A27EE067A0C289FED9F8A01
:10B6F800DFED9F6A00F04887B4EEC87AF1EE10FAE1
:10B7080098BFB0EE478AB4EEE68AF1EE10FAB8BFF9
:10B71800B0EE668A84ED4E8ABEF1000F00F0DD803F
:10B72800B0EE007AF4EEC77AF1EE10FA05DD37EEE6
:10B73800C77ADFED8A6AE7EE267A96ED017ADFEDC1
:10B74800886A27EE267AF0EEC75A84ED557AC4ED5A
:10B75800585A99B106EE901A9FED7F6AF8EEE66A9C
:10B7680027EE075A66EE866AB7EE006A36EE666A14
:10B7780025EE255AA5EE266A27EE067ADFED796AC8
:10B78800937967EEA67A67EE877AABB107EE103A3F
:10B79800B8EEC77A9FED706ADFED736A27EE257AF7
:10B7A80027EE067AB4EEE67AF1EE10FA41F3378125
:10B7B800DFED706A67EEA67A0C2800F0C586DFED2B
:10B7C8006B6A9FED6B7AF4EEE67AF1EE10FA88BFB9
:10B7D800F0EE667AF4EEC77AF1EE10FAB8BFF0EE42
:10B7E800477ABEF1010FC4ED4F7A76DD5378DFED6D
:10B7F8005A6A07EE903AF8EEE77AB0EE007A67EE0A
:10B80800A67A537AF4EEC77AF1EE10FA05DD37EE30
:10B81800C77ADFED526AE7EE267A96ED027ADFED17
:10B82800506A27EE267AF0EEC75A84ED567AC4EDB0
:10B83800595A9BB106EE903A9FED476AF8EEE66AD0
:10B8480027EE075A66EE866AB7EE006A36EE666A33
:10B8580025EE255AA5EE266A27EE067ADFED416A1F
:10B86800D37967EEA67A67EE877AFBB107EE103ACE
:10B87800B8EEC77A9FED386ADFED3B6A27EE257A86
:10B8880027EE067AB4EEE67AF1EE10FA01F3D580E7
:10B89800B5EEC07AF1EE10FA02F10483B7EE006A51
:10B8A80036EE477AC6EE076A67EEA67A0C2800F0ED
:10B8B8008986DFED2E6A9FED2E7AF4EEE67AF1EEB8
:10B8C80010FA88BFF0EE667AF4EEC77AF1EE10FA55
:10B8D800B8BFF0EE477AC4ED507A092800F0208608
:10B8E80099F82160002E40F0D585002384F8B03106
:10B8F80023F0A0FB002840F03B831F4B1B7823B9A3
:10B908001E4B9B78002B41F0F080029B1E78072E7F
:10B918007FF471A8FBF76CFD194B029A401B16784F
:10B92800D880FFF768B894F86821002A3FF46EA918
:10B93800144A84F868311288002A7FF461A9124AEF
:10B94800124B1178186881F00101F8F7B0FAFFF787
:10B958005DB900BF1C4900200AD7233CD7A3684122
:10B968006F12033B00004843A4707D3F00C0F944B8
:10B9780000C0F9C40000C8427F490020BA53002023
:10B98800D8460020745500207655002078550020B0
:10B9980094ED577AB1F90000D4ED586AB1F902E094
:10B9A800E24AF4EEC76A80EAE0738EEAEE71A3EB2E
:10B9B800E073F1EE10FAA1EBEE71B8BFF0EE476A52
:10B9C8008B42B8BF0B4607EE103A1378B8EEC77A29
:10B9D80027EE097A002B40F0B880D54B93ED006A2A
:10B9E800B4EEEA6AF1EE10FA41F17A80F7EE005A05
:10B9F80075EEC65A3BEEC77A65EE8B5ACD4BA7EE6D
:10BA0800256A93ED007A26EE076AB5EEC06AF1EE74
:10BA180010FA40F28E85CAEE065AB7EE007AB0EEFA
:10BA2800476AA6EEE56AF0EE466AF4EEC76AF1EEFA
:10BA380010FA88BFF0EE476AF5EEC06AF1EE10FA28
:10BA4800B8BFF0EE4C6ABC4B93ED007A67EE877A8C
:10BA5800A7EEA68AFEF72ABF0122FEF783BEB74BE0
:10BA6800B74A2B4493ED007AD2ED007AB54B67EED6
:10BA7800277AF7EE006AF4EEE67AF1EE10FA93ED23
:10BA8800007A88BFF0EE667A67EE877A27EE888AB2
:10BA9800FFF778B8AC4BDFF8EC921A78AB4ED507C5
:10BAA8005CBFB9F81820A4F88C21A94AD6ED037A0E
:10BAB800128807EE102AB8EEC77AF4EEC77AF1EECC
:10BAC80010FA41F2C587A34D2B8807EE103AB8EE5D
:10BAD800C77AF4EEC77AF1EE10FAC1F255809E4AA1
:10BAE8009E4D92ED006AD5ED006A94F99821C4ED57
:10BAF800646A76EE665A012AC4ED626AC4ED615A38
:10BB080084ED656A01F0D785049BC4F89C31002553
:10BB180037EEC77AFCEEE77A914E84ED687A17EE35
:10BB2800902AA4F88C21012296ED005A84F89821D5
:10BB38008C4A954241F2BC878B4BD3ED007AD3ED0A
:10BB4800013AD3ED024AFFF7C5B87A4B93ED005A94
:10BB5800B5EEC05AF1EE10FA40F3EB84834BD3ED07
:10BB6800004AF5EEC04AF1EE10FA40F3E28434EEF2
:10BB7800C77A66EECA5A87EE246AC5EE856AB7EEBA
:10BB8800007AB4EEC76AF1EE10FA88BFB0EE476AE1
:10BB9800B5EEC06AF1EE10FA76EE876AB8BFB0EE7D
:10BBA8004C6A66EE266A40E7714AD2ED007AB0EE3A
:10BBB800C87AB4EEE77AF1EE10FA7FF727A86D4A53
:10BBC800D2ED007AB0EEED7AB4EEE77AF1EE10FA43
:10BBD8007FF71CA8684AD9ED007A92ED007AF0EE5A
:10BBE800E77AF4EEC77AF1EE10FA7FF50FA8012292
:10BBF8000499C4F86C1184F86821FEF7EABF07EECF
:10BC0800102A1978DFF88081C4F80C71B8EEC77A69
:10BC1800F7EE006A132986EE879AB8F90400B4F89B
:10BC280010619BED070A01F0D284544A544992ED01
:10BC3800001AD2ED053A92ED122A92ED173AD2ED9A
:10BC4800091AD2ED0E4A92ED016A92ED064A92ED7A
:10BC58000A7AD2ED0F5AD2ED132AD2ED186A92ED74
:10BC6800045AD2ED030A67EE897A69EE288A29EE2A
:10BC7800088AE1EE273A01EB86070025A2EE283A6A
:10BC8800C4F80051C4F80451E1EE884AA6EE274AE8
:10BC9800E7EE085A92ED167A92ED0D6A92ED021AC5
:10BCA800D2ED0C1AC7ED003AE2EEA86A25EE635A07
:10BCB80027EE437A92ED0B2AD2ED152AC7ED204ADA
:10BCC800A0EEE34A26EE646AD2ED143A82ED054A04
:10BCD800A1EE275AF0EE477AE1EEE45AA2EE086A9E
:10BCE800E2EEC36AE3EEA87A82ED065AC2ED0E5A76
:10BCF80082ED0F6A87ED403AC2ED176AC2ED187AF5
:10BD0800C4F80851721C02F01F02A4F81021A8F808
:10BD18000400029BFEF725BCA4F8E071002A3FF45A
:10BD2800E7AD0A4E4FF0020E7CE400BF0C71002014
:10BD38001471002008710020047100207022002076
:10BD4800FC700020F8700020BF550020F446002049
:10BD5800C84C0020CA4C002048370020B44C0020B2
:10BD6800D04C00208FD003008C39002010710020A7
:10BD78003C71002038710020407100208C3C00206C
:10BD8800203A0020204D0020D84600209C4A1178F7
:10BD9800D4F818719B4B9FED9C7AFE009A1982ED9E
:10BDA800007A002979D09948B0EE476AF0EE476AE0
:10BDB8000022F0EC017A013267EEA77A05EE902AAC
:10BDC800B4EEE77AF1EE10FAF8EEE55AB8BFB0EE45
:10BDD800677A8A4276EEA76AA7EEA56AE9D1F5EEF8
:10BDE800C06A9A19F1EE10FA82ED007A55DDC6EEB6
:10BDF800265A874A87490988F7EE007A75EEE75A86
:10BE0800D2ED007A65EEA77AFDEEE77A17EE902A72
:10BE1800812A42F357808A42A8BF0A4607EE902A31
:10BE2800F8EEE77A7C4AF01902EB800292ED057A87
:10BE3800D2ED003A92ED066A92ED014AD2ED046A1B
:10BE4800D2ED034A92ED025AA3EEA77AA4EE276A2E
:10BE580066EEC76AA7EE646ABDEEC77AE5EE276AA2
:10BE680017EE100A812882ED056AC2ED066A42F3D0
:10BE780026808142A8BF014607EE901AF8EEE77ABD
:10BE8800FCEEE77ACDED057ABDF8142099198A8081
:10BE98001FB9BEF1130F02F0AC86BEF1150F41F0C9
:10BEA800DC801E44DFF89081B28828F81720D4F887
:10BEB80014515A4A013582FB05325119EA17C2EB6F
:10BEC800A102C2EBC202AD1AC4F814515448D4F806
:10BED8001C11049B534D02682D78C4F81C31591A63
:10BEE8000A440260002D40F0DB8107EE901A4E4EA6
:10BEF800DFF864914D4FB8EEE78A06F5F07506F560
:10BF08001378F6EC017A9BED070ADBF80832F8EEB5
:10BF1800E77A284627EE800A9847A5F1E000DBF883
:10BF280028319847A5F17000DBF898319847D6F882
:10BF3800EC00DBF8AC309847D7ED007AA9EC010AA1
:10BF4800E0EE087A2435A845E7EC017AD9D1029BBE
:10BF58001E78FEF744BD364B364A19681288364BB0
:10BF6800C96919805A8013B0BDEC0E8BBDE8F08FFB
:10BF7800324C22F01BFF6378022B00F0E985032B7B
:10BF88007FF4BBAC41F2B813E35C002B41F015839E
:10BF980041F2A403E35C002B41F00A8341F2E80379
:10BFA800E35C002B41F00E8341F22C13E35C002B81
:10BFB8003FF4A3AC224823F03BFD9EE4214B224EE4
:10BFC8001A7812F0010F327840F04C83002A00F002
:10BFD800458592001D491E48DFF880A0DFF8809053
:10BFE80027F008FFFFF717BAB4F8E071013F3FB236
:10BFF800002FA4F8E0717FF791AE164EFFF7D8BA7C
:10C00800023A0020F83C0020000000001421002023
:10C01800043A0020003A0020203C00209324499252
:10C02800F44B0020F9390020A84D0020F84B0020DF
:10C03800344500200C2D0020D8460020B85B002095
:10C04800E46C0020BF55002082460020102D0020FF
:10C05800B4390020F4460020F84F00200450002096
:10C06800204D0020002D00F0BD86BCF1000F42F0ED
:10C07800A382CA4D002B42F0378195ED006A9DEDF1
:10C088000A5AC74825EE866AFDEEE44AA5EE076A15
:10C09800B0EE675AA6EE265A14EE901ABDEEC56A9F
:10C0A80016EE10CA16EE107AF445A8BF7746614519
:10C0B800C8BF0F4606EE107AB8EEC66A012A80EDB0
:10C0C800006A00F0DF8095ED046A9DED0B5A25EEBD
:10C0D800866AA5EE076AB0EE675AA6EE265ABDEE46
:10C0E800C56A16EE10CA16EE107AF445A8BF774650
:10C0F8008C45B8BF0F4606EE107AB8EEC66A022A1B
:10C1080080ED016A00F0BE8095ED086A9DED0C5A3D
:10C1180025EE866AA5EE076AB0EE675AA6EE265A9D
:10C12800BDEEC56A16EE10CA16EE107AF445A8BF21
:10C1380077468C45B8BF0F4606EE107AB8EEC66A49
:10C14800032A80ED026A00F09D8095ED0C6A9DED52
:10C158000D5A25EE866AA5EE076AB0EE675AA6EE76
:10C16800265ABDEEC56A16EE10CA16EE107AF445C8
:10C17800A8BF77468C45B8BF0F4606EE107AB8EED2
:10C18800C66A042A80ED036A7CD095ED106A9DED9D
:10C198000E5A25EE866AA5EE076AB0EE675AA6EE35
:10C1A800265ABDEEC56A16EE10CA16EE107AF44588
:10C1B800A8BF77468C45B8BF0F4606EE107AB8EE92
:10C1C800C66A052A80ED046A5CD095ED146A9DED77
:10C1D8000F5A25EE866AA5EE076AB0EE675AA6EEF4
:10C1E800265ABDEEC56A16EE10CA16EE107AF44548
:10C1F800A8BF77468C45B8BF0F4606EE107AB8EE52
:10C20800C66A062A80ED056A3CD095ED186A9DED50
:10C21800105A25EE866AA5EE076AB0EE675AA6EEB2
:10C22800265ABDEEC56A16EE10CA16EE107AF44507
:10C23800A8BF77468C45B8BF0F4606EE107AB8EE11
:10C24800C66A072A80ED066A1CD095ED1C6A9DED2A
:10C25800115A65EE865AE7EE055AE6EEA57AFDEE26
:10C26800E77A17EE905AAE45A8BFAE46A942D8BFA6
:10C27800714607EE901AF8EEE77AC0ED077A002AC1
:10C288003FF4C9A892004749454827F0B3FD464AFC
:10C298001268002A3FF4C4A820F0E4F9FFF7C0B8F8
:10C2A80007EE901A414D424BDFF80881DFF80891FC
:10C2B8000394F8EEE78A05F5B8760027CDF81880DC
:10C2C8001C46029BDBED077A1B78172B51D095EDA6
:10C2D800007AB8EEC78A082B28EE278A07D1B0EE75
:10C2E800480A059327F0C6FE059BA8F80000DAF86F
:10C2F800002092000BD5002F02F00787B0EE480A05
:10C30800DBF8083206F170009847B0EE408AB0EECC
:10C31800480ADBF82831A6F170009847DBF8983115
:10C3280030469847029B1B78032BB0EE408A2CD0EE
:10C33800D5F8F000DBF8AC30B0EE480A9847D9EDF4
:10C34800007AA4EC010AE0EE287A0137032F06F1FF
:10C35800240608F1020805F10405E9EC017AB0D1D8
:10C36800029B039C1E78FEF73ABBF0EE676AFFF764
:10C3780079B995ED007A0BEB4702B8EEC78A128FB0
:10C38800A8F8002028EE278AB1E727F073FEA8F85E
:10C398000000CDE7B0EE465AFEF7D3BC344C00207F
:10C3A800B4390020102D00200C700020A84D00206A
:10C3B800F84F0020D8460020F84B00209B499C4BA2
:10C3C800D1F8EC101B6844F620608142A8BF0146F2
:10C3D800B1F57A7FB8BF4FF47A7189B213F0100FB4
:10C3E800A4F8B211DAF8003000F0C983DB0441F197
:10C3F8006D85904BD3F800E0BEF832707F088E4E02
:10C408008E48D4F8B431D6ED037AA0FB010188092F
:10C41800642191FBF0F11429BDEEE77A04EB4306A1
:10C42800A8BF142101339942C4F8B43117EE10CAD9
:10C43800DCBF0023C4F8B43104EB4303A6F8B8C149
:10C44800B3F9B83107EE103AB8EEC77A77EEC77A83
:10C45800FDEEE77ACDED037ABDF90C1081EAE173C0
:10C46800A3EBE173BB4201F3A48675494FF07E53F9
:10C478000B60FFF71EB8734B0293734C26E5DBF88D
:10C488000830002B3EF4EDAF7049A1F14C009847FD
:10C49800FEF7E7BF1E216648F9F7E5F900283FF4E3
:10C4A80024AA6B4B1B885A063FF51FAA94F804323E
:10C4B800B34242F0D581624BD4ED827AD3ED016A62
:10C4C80094ED505ADFED635A9FED636A27EEC57A03
:10C4D80068EE277AA8EE267AE5EE267AB4EEE57AB3
:10C4E800F1EE10FA88BFB0EE657AB4EEC67AF1EED6
:10C4F80010FAF4EEE57AB8BFB0EE467AF1EE10FA2B
:10C5080088BFF0EE657AF4EEC67AF1EE10FAB8BF9D
:10C51800F0EE467A84ED4E7AC4ED507AFFF7E5B92D
:10C52800FDEEC87A4D4A17EE903A9780D380FFF710
:10C53800D7B9DFED4B6AFFF786BADAF8001049027F
:10C548003EF50DAEFEF70FBE9FED427ADFED426A73
:10C558004249F4EEC77AF1EE10FA98BFB0EE677A66
:10C56800FDEEE77AB4EEE67AF1EE10FA17EE903ABD
:10C57800B8BFB0EE667ABEF1010F84ED4F7A4B80FA
:10C588003FF734A9FFF7ACB9B4EEC87AF1EE10FA68
:10C5980098BFB0EE478ABDEEC77AB4EEE68ADFF8F8
:10C5A800BCC0F1EE10FA17EE103AB8BFB0EE668ACA
:10C5B80084ED4E8AACF80030BEF1000F7FF4B0A8CD
:10C5C800FFF78EB9BDEEE77A244B17EE102A9A8052
:10C5D800FFF76FB9002B3EF419ABFEF7F6BAFAF77E
:10C5E80007FF029BDFF874801A78079B012AA0EBEB
:10C5F8000300A8F8020000F09582072A7EF42EAB0B
:10C60800FAF7F6FE0390FEF72BBBFAF7F1FE029B52
:10C6180012491A78039B072AA0EB030088807EF44E
:10C628001AAFFAF7E5FE0546FEF716BF50020020DE
:10C638003C37002018490020F4460020D34D6210F2
:10C6480004000020D446002014210020C84D0020FA
:10C658001449002000C0F94400C0F9C4D84600209D
:10C6680000000000002A00F0F981D4ED583A94ED5A
:10C67800574AD4ED627AF34994ED617A91ED005A04
:10C68800D4ED555A94ED546AEF4DF048F4EEC43A9F
:10C69800F3EE046AF1EE10FA77EEA64A00F1C282D0
:10C6A80095ED026A26EE656AB0EE674AA6EE074A7D
:10C6B800B4EEE44A34EE666AF1EE10FA48BFB0EE22
:10C6C800456A012A80ED006A00F0C88195ED066A86
:10C6D80026EE656AB0EE674AA6EE074AB4EEE44A6B
:10C6E80034EE666AF1EE10FA48BFB0EE456A022AE7
:10C6F80080ED016A00F0B28195ED0A6A26EE656A5E
:10C70800B0EE674AA6EE074AB4EEE44A34EE666A2B
:10C71800F1EE10FA48BFB0EE456A032A80ED026ACE
:10C7280000F09C8195ED0E6A26EE656AB0EE674AC8
:10C73800A6EE074AB4EEE44A34EE666AF1EE10FA61
:10C7480048BFB0EE456A042A80ED036A00F086818E
:10C7580095ED126A26EE656AB0EE674AA6EE074ABC
:10C76800B4EEE44A34EE666AF1EE10FA48BFB0EE71
:10C77800456A052A80ED046A00F0708195ED166A15
:10C7880026EE656AB0EE674AA6EE074AB4EEE44ABA
:10C7980074EE666AF1EE10FA48BFF0EE456A062AB2
:10C7A800C0ED056A00F05A81D5ED1A6A66EEE56AB1
:10C7B800B0EE674AA6EE874AB3EE046AB4EEE44ADE
:10C7C80074EE466AF1EE10FA48BFF0EE456A072AA1
:10C7D800C0ED066A00F04281D5ED1E6ADFF874A24A
:10C7E800DFF8749266EEE55AE5EE877AF4EEE74AEA
:10C7F80077EEC67AF1EE10FAC8BFF0EE457AC0EDD2
:10C80800077AFEF708BE904D9DED0A5A95ED006A2D
:10C81800BCF1000F41F0E68125EE866A8B48A5EE53
:10C82800076AB0EE675AA6EE265ABDEEC56A16EE3E
:10C8380010CA16EE107AF445A8BF77466145C8BFFE
:10C848000F4606EE107AB8EEC66A012A80ED006A35
:10C858003FF418AD95ED046A9DED0B5A25EE866AF6
:10C86800A5EE076AB0EE675AA6EE265ABDEEC56A6F
:10C8780016EE10CA16EE107AF445A8BF7746614541
:10C88800C8BF0F4606EE107AB8EEC66A022A80EDD7
:10C89800016A3FF4F7AC95ED086A9DED0C5A25EE58
:10C8A800866AA5EE076AB0EE675AA6EE265ABDEE6E
:10C8B800C56A16EE10CA16EE107AF445A8BF774678
:10C8C8006145C8BF0F4606EE107AB8EEC66A032A5D
:10C8D80080ED026A3FF4D6AC95ED0C6A9DED0D5AD9
:10C8E80025EE866AA5EE076AB0EE675AA6EE265AC6
:10C8F800BDEEC56A16EE10CA16EE107AF445A8BF4A
:10C9080077466145C8BF0F4606EE107AB8EEC66A8C
:10C91800042A80ED036A3FF4B5AC95ED106A9DEDED
:10C928000E5A25EE866AA5EE076AB0EE675AA6EE9D
:10C93800265ABDEEC56A16EE10CA16EE107AF445F0
:10C94800A8BF77466145C8BF0F4606EE107AB8EE15
:10C95800C66A052A80ED046A3FF494AC95ED146A22
:10C968009DED0F5A25EE866AA5EE076AB0EE675A66
:10C97800A6EE265ABDEEC56A16EE10CA16EE107A55
:10C98800F445A8BF77466145C8BF0F4606EE107A42
:10C99800B8EEC66A062A80ED056A3FF473AC95EDD9
:10C9A800186A9DED105A25EE866AA5EE076AB0EE64
:10C9B800675AA6EE265ABDEEC56A16EE10CA16EEDE
:10C9C800107AF445A8BF77466145C8BF0F4606EE02
:10C9D800107AB8EEC66A072A80ED066A3FF452ACB0
:10C9E80095ED1C6A9DED115A65EE865AE7EE055ADB
:10C9F800E6EEA57AFDEEE77A17EE905AAE45A8BFA7
:10CA0800AE46A942C8BF8E4607EE90EAF8EEE77A2E
:10CA1800C0ED077A33E49FED0E6AFEF764BEB5EE0B
:10CA2800C07AF1EE10FA01F14182B7EE006A36EEF3
:10CA3800477AC6EE076AFEF7BDBEDFED056AFEF768
:10CA480033BF00BF304C0020344C0020B4390020E4
:10CA58000000C84204500020204D0020DFF878A3D1
:10CA6800DFF87893FEF7D7BCC8494A79002A3EF424
:10CA7800F9A9C74A1278002A3EF4F4A90B78C549E7
:10CA8800DFEDC54A07EE903A0B88B8EE677A07EEF5
:10CA9800902A06EE903AF8EEE77AF8EE666A67EEC4
:10CAA800277AB7EE007A87EEA63AB4EEE43AF1EECA
:10CAB80010FA88BFB0EE643AB4EEC73AF1EE10FA55
:10CAC800B8BFB0EE473AFEF7CFB9B44B5988FEF776
:10CAD80003BDB4F8B21101F57A7189B2FEF7FCBC56
:10CAE800AF4B93ED006AFEF790BF04980EF0D2FDAD
:10CAF800FEF70BBFAB4B9FEDAC7AD3ED087AF4EEA3
:10CB0800C77AF1EE10FA00F2F7849FEDA87AA84EE2
:10CB1800D6ED037A77EE877AC6ED037AFEF7C4BCC2
:10CB2800DFF8BC82FAF764FCA249D4F87C210968D2
:10CB38000390821A511AC4F87C01A8F80420A8F8B6
:10CB48000610FEF78DB8FAF753FC0790FDF711BEF3
:10CB5800A3784FF0010A072B3EF6CFAEDFE813F0BB
:10CB68003D0755072D072207BE0682068C063907A2
:10CB7800914B9B7B002B3EF48AACFEF78DBCD80012
:10CB88003FF534ACFEF795BCB4F88C51954240F2B1
:10CB9800FE8494F8A451002D40F0C687874A884E39
:10CBA80092ED007AD6ED007A94F99821C4ED647A72
:10CBB80077EE676A012AC4ED627AC4ED616A84ED92
:10CBC800657A02F00880049BC4F89C317D4A9FED89
:10CBD800777A92ED005A84ED687A012284F89821D8
:10CBE800FEF7A6BF784B1B88002B40F0F385774AE9
:10CBF800774B11781868F7F75AF9D4F86C21049B29
:10CC08009A1AFDF76CBE734BD9ED007A93ED007A52
:10CC1800F0EEE77AF4EEC77AF1EE10FA7DF7F6AFA8
:10CC2800FDF7E6BFD5ED015A65EEC65AB0EE674A84
:10CC3800A5EE874AB4EEE44A74EE665AF1EE10FAAD
:10CC480048BFF0EE455A012AC0ED005A3FF406AF3E
:10CC5800D5ED055A65EEC65AB0EE674AA5EE874A85
:10CC6800B4EEE44A74EE665AF1EE10FA48BFF0EEFC
:10CC7800455A022AC0ED015A3FF4F0AED5ED095AE3
:10CC880065EEC65AB0EE674AA5EE874AB4EEE44AA6
:10CC980074EE665AF1EE10FA48BFF0EE455A032AD0
:10CCA800C0ED025A3FF4DAAED5ED0D5A65EEC65A1C
:10CCB800B0EE674AA5EE874AB4EEE44A74EE665AC7
:10CCC800F1EE10FA48BFF0EE455A042AC0ED035AB7
:10CCD8003FF4C4AED5ED115A65EEC65AB0EE674AB8
:10CCE800A5EE874AB4EEE44A74EE665AF1EE10FAFD
:10CCF80048BFF0EE455A052AC0ED045A3FF4AEAEDF
:10CD0800D5ED155A65EEC65AB0EE674AA5EE874AC4
:10CD1800B4EEE44A74EE666AF1EE10FA48BFF0EE3B
:10CD2800456A062AC0ED056A3FF498AED5ED196A42
:10CD380066EEC66AB0EE674AA6EE874AF3EE045A74
:10CD4800B4EEE44A74EE656AF1EE10FA48BFF0EE0C
:10CD5800456A072AC0ED066A3FF480AED5ED1D6A24
:10CD6800DFF874A0DFF8749026EEC66AE6EE077A5C
:10CD7800F4EEE47A77EEE57AF1EE10FAB8BFF0EE69
:10CD8800457AC0ED077AFEF746BB00BFB0480020E1
:10CD9800F246002038460020713DAA3F204A002074
:10CDA80008710020CC4B00208FC2753C00000000A9
:10CDB800F4460020D43900200C50002048370020C9
:10CDC800B44C0020D04C002074550020765500202B
:10CDD800785500204071002004500020204D00208C
:10CDE800D8460020D94D002B41F0A08095ED006A6F
:10CDF8009DED0A5AD64825EE866AFDEEE44AA5EE70
:10CE0800076AB0EE675AA6EE265A14EE901ABDEEDF
:10CE1800C56A16EE108A16EE107AF045A8BF774656
:10CE28004145C8BF0F4606EE107AB8EEC66A012A19
:10CE380080ED006A3EF4EBAA95ED046A9DED0B5A6D
:10CE480025EE866AA5EE076AB0EE675AA6EE265A60
:10CE5800BDEEC56A16EE108A16EE107AF045A8BF28
:10CE680077468845B8BF0F4606EE107AB8EEC66A10
:10CE7800022A80ED016A3EF4CAAA95ED086A9DED82
:10CE88000C5A25EE866AA5EE076AB0EE675AA6EE3A
:10CE9800265ABDEEC56A16EE108A16EE107AF045CF
:10CEA800A8BF77468845B8BF0F4606EE107AB8EE99
:10CEB800C66A032A80ED026A3EF4A9AA95ED0C6AB7
:10CEC8009DED0D5A25EE866AA5EE076AB0EE675A03
:10CED800A6EE265ABDEEC56A16EE108A16EE107A30
:10CEE800F045A8BF77468845B8BF0F4606EE107ACA
:10CEF800B8EEC66A042A80ED036A3EF488AA95ED66
:10CF0800106A9DED0E5A25EE866AA5EE076AB0EE08
:10CF1800675AA6EE265ABDEEC56A16EE108A16EEB8
:10CF2800107AF045A8BF77468845B8BF0F4606EE89
:10CF3800107AB8EEC66A052A80ED046A3EF467AA3C
:10CF480095ED146A9DED0F5A25EE866AA5EE076ADF
:10CF5800B0EE675AA6EE265ABDEEC56A16EE108ADE
:10CF680016EE107AF045A8BF77468845B8BF0F4639
:10CF780006EE107AB8EEC66A062A80ED056A3EF417
:10CF880046AA95ED186A9DED105A25EE866AA5EE1B
:10CF9800076AB0EE675AA6EE265ABDEEC56A16EEC7
:10CFA800108A16EE107AF045A8BF77468845B8BFB4
:10CFB8000F46FEF70ABA674ED4ED017A94ED006A7F
:10CFC8003188726977EEA77AF0EE006AB0EE677A78
:10CFD800A6EE267A4E1E04EBC601D6EE267A08394E
:10CFE8001032F6EE003A27EE237A67EEA37A84ED44
:10CFF800207AC4ED217A584C274604F1800091ED3F
:10D00800027A91ED036AD7ED036AD7ED027A52ED01
:10D01800014A12ED025A37EE674A76EEC65A77EEA3
:10D02800277AE4EE845A013EA1F10801E5EE047A7C
:10D0380007F1080702F1080236EE267A00F1080027
:10D04800E4EE877AE5EE475A67EEA37A25EEA37AEF
:10D05800C0ED007A80ED017AD1D1BEF1140F7EF4D3
:10D0680028AFFAF7C5F9039BDFF80081C01AA8F8C2
:10D078000200D4F81451FEF71CBFD4F81831B4F8E4
:10D0880010C1364ACCF120095FFA89F90CEB431735
:10D0980002EB87075FEA990201F0BC8501321601AD
:10D0A8002F48304907EB060807F1100212ED024A33
:10D0B80012ED035A12ED016A12ED047A50ED024A9C
:10D0C80050ED035A50ED016A50ED047A64EE244A9B
:10D0D80065EE255A66EE266A67EE277A1032904585
:10D0E80041ED024A41ED035A41ED016A41ED047AEE
:10D0F80000F1100001F11001D8D11B48A6F1100170
:10D108000F4400EB0108214419F0030209D0B7ECE1
:10D11800017AF8EC017A67EE277A013AE1EC017AB4
:10D12800F5D1BCF1000F41F05380BEF1140F7EF42D
:10D13800C0AEFAF75DF9039BDFF83080D4F81451DC
:10D14800C01AA8F80200FEF7B4BE00BF344C002095
:10D15800B4390020083A002014210020203A002089
:10D16800B03B002024210020A03B0020D84600200E
:10D17800D04E318873684FEA51094FEA89005FEA57
:10D18800D10C04EB000204EB810500F0A18000F152
:10D1980010010CF1010CC84F02EB0C1C2944103291
:10D1A80003F1100E05F1100050ED032A50ED043A7A
:10D1B80017ED043A17ED032A50ED026A10ED016AE3
:10D1C80017ED021A57ED010A11ED044A11ED035A41
:10D1D80052ED044A52ED035A12ED027A52ED017AE9
:10D1E80051ED021A11ED010A73EE238A32EE228AFA
:10D1F80047ED048A07ED038A71EE268A30EE868AA7
:10D2080047ED028A07ED018A74EE848A35EE858A35
:10D2180042ED048A02ED038A77EE218A37EE808A8E
:10D2280042ED028A02ED018A73EE633A75EE655AA1
:10D238001EED035A32EE623A74EE644A25EE638AB2
:10D248001EED044A23EE052A64EE652AA3EE048A3D
:10D258001032944524EE843AA3EE842A07F110078D
:10D268000EF1100EA5EE853A00F1100001F1100143
:10D27800E4EE852A00ED078A00ED082A01ED073A59
:10D2880041ED082A5EED055A1EED065A71EE666AF2
:10D2980030EEC66A31EEC77A70EE677A26EE253A26
:10D2A80065EEE63A25EE674A67EE054AE6EE053A88
:10D2B800A6EE853AA7EE254AE7EEA54A00ED063A1E
:10D2C80040ED053A01ED064A41ED054A7FF46CAFA1
:10D2D8001FFA89F91A464946784819F0ADFE72686E
:10D2E8004946284619F0A8FE029B1A78142A7FF4AA
:10D2F800C0AEB6E66F4E7148B268B18925F03EFD02
:10D30800029B93F800E0BEF1140F01F0EB84D4F80F
:10D3180014510135C4F814514EE6DFF8B89199F864
:10D3280000108F0801F00386654E07F101084FEAE7
:10D33800481806EB080C06F12002A6F1700012ED61
:10D34800076A52ED056A12ED037A52ED017A52ED41
:10D35800025A12ED084A52ED064A12ED045A26EE18
:10D36800066A66EEA66A27EE077A67EEA77AA4EE43
:10D37800046A20329445E4EEA46A00F11000A5EE98
:10D38800057AE5EEA57AF1EEC65AB1EEE66AF1EE57
:10D39800C76AB1EEE77A40ED085A00ED076A40ED3A
:10D3A800066A00ED057ACAD1A8F12002324404EBDE
:10D3B800071711F0030018BF08320FD052ED017A99
:10D3C80012ED027A67EEA77A0138E7EE077A02F1E2
:10D3D8000802B1EEE77AA7EC017AEFD1BEF1140F9B
:10D3E80001F06D840135C4F81451FEF7D1BCD4F8AE
:10D3F800185134493448354BEA00114415448A8899
:10D40800196800EE102A643AC82AA8BFC822782AE8
:10D41800B8BF782207EE902AB8EEC07AF8EEE77A1D
:10D4280000EB850577EE670A77EE876A67EE877AFD
:10D4380020EEA67AB8EE400AC7EE870A2846D5F845
:10D448001490D5F81880EF692E6A18F049FE029BEF
:10D45800C5F8149093F800E0C5F81880BEF1140FD1
:10D46800EF612E6201F01E84D4F81821184BD4F80D
:10D478001451013283FB0213A3EBE27303EB430362
:10D48800D31A0135C4F81831C4F81451F7E5F9F77F
:10D49800AFFF029B039093F800E0BEF1140F05BFA5
:10D4A800DFF83480D4F81451D4F81451A8F8005097
:10D4B800FDF761B8083A002024210020142100203B
:10D4C80094210020F83C0020884F0020F44F0020D1
:10D4D80056555555023A0020D8460020306E99BC62
:10D4E8002716983DA40DC93F843459BEDB0F494027
:10D4F800D06D393A00000000F0EEE76AB7EE005A46
:10D5080035EE665A1FED0B4A5FED0B5A1FED0A6A9E
:10D518001FED0C7A94ED6B0AF1EEC54AE6EE845ADB
:10D52800F5EEC07AA6EEA56AF1EE10FAA6EE867AB6
:10D5380048BF5FED127A27EE247A48BF37EEC77AE4
:10D5480027EE000A26F096FDB0F5617F00F3A2866B
:10D5580007EE900AF8EEE76A5FED1B7A66EEA76AB7
:10D5680007EE906ABDEEE67AF8EEE77A17EE103A23
:10D578002033402B41F295841FED220A26F07AFDD4
:10D5880000B207EE900AB8EEE77AFFF7C0BAC14AD0
:10D5980002F1500503E00432954200F0C582137889
:10D5A800262BF8D19678D3789E42F4D2FFF7F1BAB9
:10D5B800B94822F03DFAFEF7F1BCB84822F038FA33
:10D5C800FEF7E6BCB64822F033FAFEF7EDBCB54DDF
:10D5D800B54F95ED004A95ED057AD5ED014A95EDE3
:10D5E800066AD5ED046A95ED035AD5ED025A67EE41
:10D5F800897A07EB8602A4EE277AA4EEA76A66EE7C
:10D60800C76AA5EE476AE5EEA76A20EE070A85ED28
:10D61800056AC5ED066A82ED007A29EE088A26F0C9
:10D6280029FD69EE288AD5ED0E5AD5ED176A95EDD4
:10D63800091AD5ED121A95ED0F5A95ED187A95ED50
:10D648000A2AD5ED132A95ED0D6AD5ED167A95EDD2
:10D658000C3AD5ED0B3A95ED154AD5ED144AE1EEA5
:10D66800085A002207EB8601E8EEA16A00B2C4F866
:10D678000021A2EE085AC4F80421C4F80821A8EE33
:10D68800A27A26EE656A67EEE67AA3EE655AA3EEFD
:10D69800886AA6EEC47AE8EEA47A85ED0E5AC1ED42
:10D6A800205A85ED0F6AC1ED406A85ED177AC5ED00
:10D6B800187AFEF727BBD4F89C51049B5D1BFEF734
:10D6C80027BABBF93820CBF8201007EE902A0121A1
:10D6D800F8EEE77ACBF86020CBF87C100022012F17
:10D6E800CBED1C7ACBED1B7ACBF8742001F06B8262
:10D6F800AF427CF4A4AFBBF93A20CBF8642007EE24
:10D70800902A00210122F8EEE77ACBF82410CBF812
:10D7180090200022012FCBED217ACBED207ACBF897
:10D72800882001F05482AF427CF4BDAFBBF93C20A5
:10D73800CBF8682007EE902A00210122F8EEE77A5C
:10D74800CBF82810CBF8A4200022012FCBED267AA5
:10D75800CBED257ACBF89C207CF4D9AF9FED538A8A
:10D76800032E49D04CB107EE904AF8EEE77AF4EE72
:10D77800C87AF1EE10FA01F1DF834D4A4D4C116879
:10D78800DBF86820A8F8060094F8200102EB55029F
:10D7980092FBF5F50022CBF828508A620A63CA6228
:10D7A80028B1454A126832F480637CF4B3AF434A27
:10D7B800126812F4003241F0FE8141481146835C40
:10D7C800012B02F10C0200F0928301311829F6D1E5
:10D7D800FCF7A0BF3B494B69002B3DF480A83A48B1
:10D7E8003A4B008893FBF0F00B684FF0010E18607D
:10D7F80081F811E0FDF773B8B0EE480A26F03AFC5C
:10D8080000B2AFE723690622652BA27034D92278CB
:10D81800032A14BF6FF0FF026FF07F02A3F16503C4
:10D8280003EA020303F1010314BF4FF4807280225C
:10D838009A42236120D23A68E768023203EB07086C
:10D84800904581F04984224A6760D16FC4F8088006
:10D85800490203FB01F30521176042F81C3C42F81A
:10D86800183CA170A2681B49012024F01DF9012869
:10D8780041F028840623A3700021174823F034FDC3
:10D88800012841F01F84A3780133DBB2A370FFF7AE
:10D8980062B900BF283400205C6C0020706D002045
:10D8A800A06C00208C3C0020203A002000000000E2
:10D8B800344500201421002010490020E82F0020C2
:10D8C8002C6503087C5500209455002020A10700F2
:10D8D8004C6D0020BC5B0020286D00202278237D41
:10D8E800AF4FDFF8FC92032A14BF4FF480784FF053
:10D8F8008008002B42D0012BFBD1AA4B6268196823
:10D90800386800234FEA412E4FF0FF31B1FBFEF19A
:10D9180012EB010B43F1000C0021614500F10200FC
:10D9280008BF584538BF83465A469F49022021F010
:10D9380059F9032801F26B8101A353F820F000BFC5
:10D9480003B9000859D9000803B9000859D90008D3
:10D958006268A3682669991AB14284BFE2602161AE
:10D9680003283FF44FAF0133B3FBF8F208FB123240
:10D978000AB143449B1A0022636022753A684946FB
:10D988000232002021F02EF9032801F2408101A380
:10D9980053F820F003B900084DDA000803B900086D
:10D9A8000DD8000841F27013E35C002B3DF4A5AFDD
:10D9B8007E4822F03DF8FDF7A0BF7D4B0093032081
:10D9C800A070302305227B49784824F041FAFDF7FE
:10D9D80094BF03236370FDF790BF00230AAE31465E
:10D9E8001846092220F0BEFF01287DF486AF0A9B65
:10D9F80093F8FE21552A01F0128141F2B412022156
:10DA08000123A1546370FDF778BF0AAE41F2FC17F9
:10DA18003146E0590023092220F0A4FF01287DF4B3
:10DA28006CAF00230A9A2370B2F80B30B3F5007F6D
:10DA380001F0E38241F2B41203210123A15463707F
:10DA4800FDF75BBF636884F814A00133A36054E753
:10DA5800594A5A4DD2ED006A594A95ED006A127832
:10DA6800C4ED646A84ED656A002A00F0238276EECC
:10DA7800665A94F99821C4ED615A0132C4ED626A7C
:10DA880000F08A85049BC4F89C31002537EE677A3C
:10DA9800FCEEE77A4B4E84ED687A17EE902AA4F8EC
:10DAA8008C21FF2296ED005A84F89821FEF740B8A1
:10DAB800DFED457A454B94ED687AC3ED007AC3ED06
:10DAC800017AC3ED027A424BF0EE674AF0EE673A0C
:10DAD8001968FDF7FFB83F4B1D7805F0010CFDF7FD
:10DAE80096BC3D49DFED3D7A0968C4ED4C7A11F0EA
:10DAF800805840F0C383DAF8001011F4800800F071
:10DB0800EC814FF00008B6EE007A67EE877AF4EE03
:10DB1800E57AF1EE10FAC8BFF0EE675A40F3AE832B
:10DB2800C4ED685AFDF71FBB234A244DD2ED007A95
:10DB3800234A95ED007A1278C4ED647A84ED657A0B
:10DB4800002A00F0318377EE676A94F99821C4EDD2
:10DB5800616A0132C4ED627A00F05A86049BC4F807
:10DB68009C3100259FED187A164E84ED687AFF22C5
:10DB780096ED005A84F89821FDF7DABF73EEE77A3C
:10DB8800B7EE007AF4EEC77AF1EE10FAC4ED4C7AEB
:10DB980041F3278084EEA77A8DED0A7AFDF7D9BA8A
:10DBA800C06D0020C86D0020C05B0020286D0020DB
:10DBB80049100308987C0308E4350020B84C00207D
:10DBC80044580020CC4C0020000000008C39002074
:10DBD80018490020BF5500203C3700200000008075
:10DBE800BC5B0020002F00F0CD8625EE866ACC486D
:10DBF800A5EE076AB0EE675AA6EE265ABDEEC56ACC
:10DC080016EE10CA16EE107AF445A8BF774661459D
:10DC1800C8BF0F4606EE107AB8EEC66A012A80ED34
:10DC2800006A3DF4F8AB95ED046A9DED0B5A25EEBC
:10DC3800866AA5EE076AB0EE675AA6EE265ABDEECA
:10DC4800C56A16EE10CA16EE107AF445A8BF7746D4
:10DC58006145C8BF0F4606EE107AB8EEC66A022ABA
:10DC680080ED016A3DF4D7AB95ED086A9DED0C5A3D
:10DC780025EE866AA5EE076AB0EE675AA6EE265A22
:10DC8800BDEEC56A16EE10CA16EE107AF445A8BFA6
:10DC980077466145C8BF0F4606EE107AB8EEC66AE9
:10DCA800032A80ED026A3DF4B6AB95ED0C6A9DED52
:10DCB8000D5A25EE866AA5EE076AB0EE675AA6EEFB
:10DCC800265ABDEEC56A16EE10CA16EE107AF4454D
:10DCD800A8BF77466145C8BF0F4606EE107AB8EE72
:10DCE800C66A042A80ED036A3DF495AB95ED106A87
:10DCF8009DED0E5A25EE866AA5EE076AB0EE675AC4
:10DD0800A6EE265ABDEEC56A16EE10CA16EE107AB1
:10DD1800F445A8BF77466145C8BF0F4606EE107A9E
:10DD2800B8EEC66A052A80ED046A3DF474AB95ED39
:10DD3800146A9DED0F5A25EE866AA5EE076AB0EEC5
:10DD4800675AA6EE265ABDEEC56A16EE10CA16EE3A
:10DD5800107AF445A8BF77466145C8BF0F4606EE5E
:10DD6800107AB8EEC66A062A80ED056A3DF453AB10
:10DD780095ED186A9DED105A25EE866AA5EE076A9C
:10DD8800B0EE675AA6EE265ABDEEC56A16EE10CA60
:10DD980016EE107AF445A8BF77466145C8BF0F460E
:10DDA80006EE107AB8EEC66A072A80ED066A3DF4D8
:10DDB80032AB95ED1C6A9DED115A65EE865AE5EE7B
:10DDC800075AE6EEA57AFDEEE77A17EE902A964511
:10DDD800A8BF96468A42A8BF714607EE901AF8EE89
:10DDE800E77AC0ED077AFDF716BBBEF1010F7FF7A2
:10DDF800B5AC07EE103AB8EEC77AC7EE876AB1EE4F
:10DE0800E68AADE4BEF1010F40F3E18607EE103A71
:10DE1800B8EEC77AC7EE876AB1EEE68A032E13D04A
:10DE28004CB107EE904AF8EEE77AF4EEC87AF1EED4
:10DE380010FA01F18180DBF8642002EB550292FBB5
:10DE4800F5F2CBF824206EE4B0EE480A26F012F979
:10DE580000B2E5E7BEF1010F40F3B58607EE103AD0
:10DE6800B8EEC77AC7EE876AB1EEE68A032E13D0FA
:10DE78004CB107EE904AF8EEE77AF4EEC87AF1EE84
:10DE880010FA01F15980DBF8602002EB550292FB91
:10DE9800F5F2CBF820202BE4B0EE480A26F0EAF899
:10DEA80000B2E5E7F7EE006AFDF7FEBCF7EE006AA0
:10DEB800FDF780BC76EEC65AF0EE466AD9E58222B6
:10DEC800FDF7E4BFDFED177AFDF7ACBF164BD3F8CB
:10DED80000E0BEF93270FEF792BAB6EE007AF4EEC0
:10DEE800C75AF1EE10FA3FF70EAEFDF73CB9D4F879
:10DEF80024614A003EB1551800EB850576786D78A7
:10DF0800B542BCF407AC0A4400EB82000022C4F816
:10DF18002401A4F80C22C4F81022FCF7FBBB00BFB4
:10DF2800B4390020000002431849002095ED006A2A
:10DF38009DED0A4AE44825EE866AFDEEE43AA4EE31
:10DF4800076AB0EE674AA6EE264A13EE901AB4EEB8
:10DF5800C45AF1EE10FAB0EE446A88BFB0EE646AB3
:10DF6800BDEEC66A16EE108A16EE107AF045A8BF06
:10DF780077464145C8BF0F4606EE107AB8EEC66A26
:10DF8800012A80ED006A3DF442AA95ED046A9DEDF0
:10DF98000B4A25EE866AA4EE076AB0EE674AA6EE3B
:10DFA800264AB4EEC45AF1EE10FAB0EE446A88BFBD
:10DFB800B0EE646ABDEEC66A16EE108A16EE107AE6
:10DFC800F045A8BF77468845B8BF0F4606EE107AD9
:10DFD800B8EEC66A022A80ED016A3DF418AA95EDEA
:10DFE800086A9DED0C4A25EE866AA4EE076AB0EE33
:10DFF800674AA6EE264AB4EEC45AF1EE10FAB0EE1D
:10E00800446A88BFB0EE646ABDEEC66A16EE108A2E
:10E0180016EE107AF045A8BF77468845B8BF0F4678
:10E0280006EE107AB8EEC66A032A80ED026A3DF45D
:10E03800EEA995ED0C6A9DED0D4A25EE866AA4EED3
:10E04800076AB0EE674AA6EE264AB4EEC45AF1EE65
:10E0580010FAB0EE446A88BFB0EE646ABDEEC66AD4
:10E0680016EE108A16EE107AF045A8BF7746884556
:10E07800B8BF0F4606EE107AB8EEC66A042A80EDDD
:10E08800036A3DF4C4A995ED106A9DED0E4A25EE8C
:10E09800866AA4EE076AB0EE674AA6EE264AB4EE90
:10E0A800C45AF1EE10FAB0EE446A88BFB0EE646A62
:10E0B800BDEEC66A16EE108A16EE107AF045A8BFB5
:10E0C80077468845B8BF0F4606EE107AB8EEC66A9E
:10E0D800052A80ED046A3DF49AA995ED146A9DED30
:10E0E8000F4A25EE866AA4EE076AB0EE674AA6EEE6
:10E0F800264AB4EEC45AF1EE10FAB0EE446A88BF6C
:10E10800B0EE646ABDEEC66A16EE108A16EE107A94
:10E11800F045A8BF77468845B8BF0F4606EE107A87
:10E12800B8EEC66A062A80ED056A3DF470A995ED39
:10E13800186A9DED104A25EE866AA4EE076AB0EECD
:10E14800674AA6EE264AB4EEC45AF1EE10FAB0EECB
:10E15800446A88BFB0EE646ABDEEC66A16EE108ADD
:10E1680016EE107AF045A8BF77468845B8BF0F4627
:10E1780006EE107AB8EEC66A072A80ED066A3DF404
:10E1880046A995ED1C6A9DED114A65EE865AE7EEA3
:10E19800045AE6EEA57AB4EEE75AF1EE10FAC8BFD3
:10E1A800F0EE647AFDF723B977EEC76AF0EE477AA6
:10E1B800CBE4BEF834309FED457A07EE903AF8EE9E
:10E1C800E77A434B67EE877AC3ED007AFDF771B9BA
:10E1D800404A4FEA89065FEA9C0900EB060802EB11
:10E1E800C313264400F0FE8609F101094FEA091914
:10E1F80003EB090703F1100208F1100006F1100102
:10E2080012ED024A12ED035A12ED016A12ED047A78
:10E2180050ED024A50ED035A50ED016A50ED047A70
:10E2280064EE244A65EE255A66EE266A67EE277A7A
:10E238001032974241ED024A41ED035A41ED016A1D
:10E2480041ED047A00F1100001F11001D8D1A9F1D3
:10E2580010094B4408EB09004E441CF0030C3EF433
:10E2680064AFB3EC017AF0EC017A67EE277ABCF17F
:10E27800010CE6EC017AF4D1FEF757BFB7EE007A4D
:10E2880077EE677AF4EEE75AF1EE10FA88BFF0EE0F
:10E29800675A45E407EE906ADFED0F6AF8EEE77A11
:10E2A80066EEA65A9FED0D5A9FED0D6A9FED0D7A09
:10E2B800A5EE856A26EEA55AA5EE867AE5EE076AEA
:10E2C80026EEA70AFFF75AB9B43900206F12833A2D
:10E2D80004000020203A002084F9223F92E741B947
:10E2E8009730083C15A82ABE95ED006A9DED0A4AAC
:10E2F800AE4825EE866AFDEEE43AA4EE076AB0EE73
:10E30800674AA6EE264A13EE907AB4EEC45AF1EEA6
:10E3180010FAB0EE446A88BFB0EE646ABDEEC66A11
:10E3280016EE10CA16EE101AF445A8BF71466745D6
:10E33800C8BF394606EE101AB8EEC66A012A80ED43
:10E34800006A3DF49FAF95ED046A9DED0B4A25EEFA
:10E35800866AA4EE076AB0EE674AA6EE264AB4EECD
:10E36800C45AF1EE10FAB0EE446A88BFB0EE646A9F
:10E37800BDEEC66A16EE10CA16EE101AF445A8BF0E
:10E388007146BC45B8BF394606EE101AB8EEC66AE3
:10E39800022A80ED016A3DF475AF95ED086A9DED9E
:10E3A8000C4A25EE866AA4EE076AB0EE674AA6EE26
:10E3B800264AB4EEC45AF1EE10FAB0EE446A88BFA9
:10E3C800B0EE646ABDEEC66A16EE10CA16EE101AF2
:10E3D800F445A8BF7146BC45B8BF394606EE101AC9
:10E3E800B8EEC66A032A80ED026A3DF44BAF95ED9C
:10E3F8000C6A9DED0D4A25EE866AA4EE076AB0EE1A
:10E40800674AA6EE264AB4EEC45AF1EE10FAB0EE08
:10E41800446A88BFB0EE646ABDEEC66A16EE10CADA
:10E4280016EE101AF445A8BF7146BC45B8BF394668
:10E4380006EE101AB8EEC66A042A80ED036A3DF4A7
:10E4480021AF95ED106A9DED0E4A25EE866AA4EE81
:10E45800076AB0EE674AA6EE264AB4EEC45AF1EE51
:10E4680010FAB0EE446A88BFB0EE646ABDEEC66AC0
:10E4780016EE10CA16EE101AF445A8BF7146BC4530
:10E48800B8BF394606EE101AB8EEC66A052A80EDFE
:10E49800046A3DF4F7AE95ED146A9DED0F4A25EE3A
:10E4A800866AA4EE076AB0EE674AA6EE264AB4EE7C
:10E4B800C45AF1EE10FAB0EE446A88BFB0EE646A4E
:10E4C800BDEEC66A16EE10CA16EE101AF445A8BFBD
:10E4D8007146BC45B8BF394606EE101AB8EEC66A92
:10E4E800062A80ED056A3DF4CDAE95ED186A9DEDDE
:10E4F800104A25EE866AA4EE076AB0EE674AA6EED1
:10E50800264AB4EEC45AF1EE10FAB0EE446A88BF57
:10E51800B0EE646ABDEEC66A16EE10CA16EE101AA0
:10E52800F445A8BF7146BC45B8BF394606EE101A77
:10E53800B8EEC66A072A80ED066A3DF4A3AE95EDEB
:10E548001C6A9DED114A65EE865AE7EE045AE6EE1E
:10E55800A57AB4EEE75AF1EE10FAC8BFF0EE647A85
:10E56800FDEEE77A17EE901A8E45A8BF8E468F42C9
:10E57800D8BF774607EE907AF8EEE77AC0ED077ACB
:10E58800FDF77DBE0A494A69002A3CF491AA0A6847
:10E5980013604B74FCF78CBAD4F89C51049B5D1B38
:10E5A800FFF774BA034EFCF7FBBF00BFB439002075
:10E5B8007C550020F4460020002F00F0AC83E04D8D
:10E5C8009DED0A4A95ED006A25EE866AA4EE076A73
:10E5D800B0EE674AA6EE264AB0EE446A33B1B4EE0E
:10E5E800445AF1EE10FAC8BFB0EE646AFDEEE44A90
:10E5F800BDEEC66A14EE907A16EE101A8F4214EE2B
:10E6080090CA00F3F2847145A8BF714606EE101A4D
:10E61800CC48B8EEC66A012A80ED006A3CF4FBAE2D
:10E6280095ED046ADDED0B4A25EE866AA4EE876A4D
:10E63800F0EE674AE6EE264AB0EE646A002B00F078
:10E64800BB84B4EEE45AF1EE10FA40F3B5843946CF
:10E658007145A8BF714606EE101AB8EEC66A022ABE
:10E6680080ED016A3CF4D7AE95ED086ADDED0C4A01
:10E6780025EE866AA4EE876AF0EE674AE6EE264A39
:10E68800B0EE646A002B00F08D84B4EEE45AF1EE2B
:10E6980010FA40F3878439467145A8BF714606EEE3
:10E6A800101AB8EEC66A032A80ED026A3CF4B3AECB
:10E6B80095ED0C6ADDED0D4A25EE866AA4EE876AB3
:10E6C800F0EE674AE6EE264AB0EE646A002B00F0E8
:10E6D8005F84B4EEE45AF1EE10FA40F359843946F7
:10E6E8007145A8BF714606EE101AB8EEC66A042A2C
:10E6F80080ED036A3CF48FAE95ED106ADDED0E4AAD
:10E7080025EE866AA4EE876AF0EE674AE6EE264AA8
:10E71800B0EE646A002B00F03184B4EEE45AF1EEF6
:10E7280010FA40F32B8439467145A8BF714606EEAE
:10E73800101AB8EEC66A052A80ED046A3CF46BAE7E
:10E7480095ED146ADDED0F4A25EE866AA4EE876A18
:10E75800F0EE674AE6EE264AB0EE646A002B00F057
:10E768000384B4EEE45AF1EE10FA40F3FD8339461F
:10E778007145A8BF714606EE101AB8EEC66A062A99
:10E7880080ED056A3CF447AE95ED186ADDED104A58
:10E7980025EE866AA4EE876AF0EE674AE6EE264A18
:10E7A800B0EE646A002B00F0D683B4EEE45AF1EEC2
:10E7B80010FA40F3D08339467145A8BF714606EE7A
:10E7C800101AB8EEC66A072A80ED066A3CF423AE32
:10E7D80095ED1C6ADDED114A65EE865AE4EE875A1E
:10E7E800E5EEA67A002B00F0AE83F4EEC57AF1EEE2
:10E7F80010FA40F1A8833A467245A8BF724694467B
:10E8080007EE90CAF8EEE77AC0ED077AFCF703BE88
:10E81800D4F89C51049B5D1BFFF7A4B996ED000A40
:10E828000593039225F026FC4749DFF850E1D1F81B
:10E83800EC10DFF84CC1039AACF800008EFB013EE7
:10E84800C917C1EBAE1107EE901AF8EEE77A059BEF
:10E85800FDEEE77A17EE901AACF80210FCF7A5BEA9
:10E8680007EE906ADFED396A9FED397A84F8046221
:10E87800F8EEE77A67EEA67A77EE876ABDEEE66A83
:10E8880016EE103A2033402B40F2B582DFED316AA4
:10E89800314BBDEEE77AC3ED016A17EE103A20332B
:10E8A800402B00F2EF829FED2D7AF4EEC77AF1EE5D
:10E8B80010FA40F32384DFED2A5A9FED2A6A01E01B
:10E8C800F0EE477AF4EEC67AF1EE10FA37EEE57A12
:10E8D800F6DCDFED257AB4EEE77AF1EE10FA40F1D6
:10E8E8000A84DFED1F5A9FED216A01E0B0EE677AD6
:10E8F800B4EEC67AF1EE10FA77EE257AF6D49FEDEB
:10E90800147AF4EEC77AF1EE10FA40F3BE829FED66
:10E91800137A77EE677A67EEA75A9FED155A9FED3F
:10E92800156A9FED157AA5EE856A27EEA55AA5EE1C
:10E93800867AE5EE077AC4ED827AFDF7C1BD00BF9D
:10E94800344C0020B43900205002002035FA8E3CA7
:10E95800DB0FC93F0000000004000020DB0F494026
:10E96800DB0FC940E4CB1641DB0F49C0E4CB16C12D
:10E9780092E741B99730083C15A82ABED34D6210DA
:10E98800D846002025EE866AA5EE076AB0EE675ADB
:10E99800A6EE265ABDEEC56A16EE100A814200F3AD
:10E9A800B0817045A8BF704606EE100AB8EEC66A78
:10E9B800B8F1000F00F0CF83DE48012A80ED006A2D
:10E9C8003CF429AD95ED046A9DED0B5A25EE866A57
:10E9D800A5EE076AB0EE675AA6EE265ABDEEC56ADE
:10E9E80016EE107AB94200F38A817745A8BF7746B8
:10E9F80006EE107AB8EEC66AB8F1000F00F0F2839E
:10EA0800022A80ED016A3CF406AD95ED086A9DED99
:10EA18000C5A25EE866AA5EE076AB0EE675AA6EE8E
:10EA2800265ABDEEC56A16EE107AB94200F3718116
:10EA38007745A8BF774606EE107AB8EEC66AB8F1F1
:10EA4800000F00F0F083032A80ED026A3CF4E3AC87
:10EA580095ED0C6A9DED0D5A25EE866AA5EE076ABE
:10EA6800B0EE675AA6EE265ABDEEC56A16EE107AC3
:10EA7800B94200F34C817745A8BF774606EE107A75
:10EA8800B8EEC66AB8F1000F00F0C283042A80ED20
:10EA9800036A3CF4C0AC95ED106A9DED0E5A25EE64
:10EAA800866AA5EE076AB0EE675AA6EE265ABDEE4C
:10EAB800C56A16EE107AB94200F327817745A8BFD8
:10EAC800774606EE107AB8EEC66AB8F1000F00F085
:10EAD8009483052A80ED046A3CF49DAC95ED146A94
:10EAE8009DED0F5A25EE866AA5EE076AB0EE675AC5
:10EAF800A6EE265ABDEEC56A16EE107AB94200F3A4
:10EB080002817745A8BF774606EE107AB8EEC66A46
:10EB1800B8F1000F00F01483062A80ED056A3CF472
:10EB28007AAC95ED186A9DED105A25EE866AA5EE29
:10EB3800076AB0EE675AA6EE265ABDEEC56A16EE0B
:10EB4800107AB94200F3CC807745A8BF774606EE25
:10EB5800107AB8EEC66AB8F1000F00F00783072AEA
:10EB680080ED066A3CF457AC95ED1C6A9DED115A90
:10EB780065EE865AE7EE055AE5EEA67AFDEEE77AE7
:10EB880017EE902A914203DC7245A8BF72461146DF
:10EB980007EE901AF8EEE77AB8F1000F7FF434AE7A
:10EBA800089B002B7FF430AE059B079A9342B8BFB1
:10EBB800F0EE647A28E6604A1278032A00F0198297
:10EBC8000022FEF7FABD9FED668AFFF74FB99FED69
:10EBD800648AFFF723B9D4F89C51049B5D1BFDF7A9
:10EBE800F5BF5649096811F080587EF48CAFFEF7DE
:10EBF80082BF9FED530ADFF8588125EE800A25F081
:10EC080039FAD4F81451A8F80600FDF752B9237D53
:10EC1800FEF76FBE4B484C498046FEF775BA93F82D
:10EC2800FF21AA2A7EF4E9AED3F8C61149B193F8B8
:10EC3800C221A2F10B0001282DD902F0F702062A01
:10EC480029D0D3F8D61149B193F8D221A2F10B00FB
:10EC5800012820D902F0F702062A1CD0D3F8E611C1
:10EC680049B193F8E221A2F10B00012813D902F06F
:10EC7800F702062A0FD0D3F8F61100293EF4BDAEEC
:10EC880093F8F231A3F10B02012A04D903F0F70338
:10EC9800062B7EF4B2AE41F2FC120123A150A37000
:10ECA800FEF7B4BEF8F7A4FB029BDFF8A48093F844
:10ECB80000E0039BC01AA8F80200FEF7D5BBF8F7DE
:10ECC80097FB029BDFF8888093F800E0039B99F894
:10ECD8000010D4F81451C01AA8F80400FEF782BB3B
:10ECE8000F4634E7F8F784FB029BDFF8648093F85B
:10ECF80000E0039BC01AA8F80200FEF708BB0F4605
:10ED080076E6084650E60F46FEE60F46D9E60F4679
:10ED1800B4E60F468FE60AA9BDEEE46A01EB82026B
:10ED280094460A48034D09941A4616EE107A43464B
:10ED38002CE000BFB4390020373F00203C370020CA
:10ED48000000C842A03B002014210020344C0020C1
:10ED5800D846002092E741B99730083C15A82ABE4A
:10ED680000000000E4CB1641DB0FC940E4CB16C11C
:10ED7800DB0FC93FDB0F4940DB0FC9BFDB0F49C0C1
:10ED88006145A5EC016A00F1100031D090ED006AF0
:10ED9800B1EC014A25EE866AA7EE046AB0EE674A2E
:10EDA800A6EE864AB0EE446A32B1B4EE445AF1EEA9
:10EDB80010FAC8BFB0EE646ABDEEC66A16EE108AD5
:10EDC800474506EE107A04DCF045A8BFF04606EE8B
:10EDD800108AB8EEC66A002BD2D1089C002CCFD17D
:10EDE800059CA046079CA045B8BFB0EE646AC7E77B
:10EDF800099CFCF710BBF4EEC77AF1EE10FA40F369
:10EE080081815FED275A1FED296A01E0F0EE476A1C
:10EE1800F4EEC66AF1EE10FA36EEE57AF6DC5FED4E
:10EE2800296AB4EEE67AF1EE10FA40F161815FEDFD
:10EE3800325A1FED326A01E0B0EE667AB4EEC67A55
:10EE4800F1EE10FA77EE256AF6D41FED377AF4EE74
:10EE5800C76AF1EE10FA40F3B9801FED3A7A77EEFF
:10EE6800666A66EEA65A1FED455A1FED456A1FED04
:10EE7800457AA5EE856A26EEA55AA5EE867AE5EED0
:10EE8800076A05E55FED4A7A55E51FED457AF4EE28
:10EE9800C77AF1EE10FA44BF1FED487A77EE677A29
:10EEA80039E51FED4C7AF4EEC76AF1EE10FA40F33B
:10EEB80028825FED535A1FED556A01E0F0EE476A6C
:10EEC800F4EEC66AF1EE10FA36EEE57AF6DC5FED9E
:10EED800556AB4EEE67AF1EE10FA40F17A815FED08
:10EEE8005E5A1FED5E6A01E0B0EE667AB4EEC67A4D
:10EEF800F1EE10FA77EE256AF6D41FED637AF4EE98
:10EF0800C76AF1EE10FA05DD1FED667A77EE666ADC
:10EF1800FFF7C6B91FED687AF4EEC76AF1EE10FA8A
:10EF280044BF1FED6A7A77EE666AFFF7B9B9C54F35
:10EF380007F18002FEF73DBAA8F80600ABF8A85022
:10EF4800C04CFBF7EEBBFDEEE77A17EE902ABA420B
:10EF5800FFF656AC50E4BDEEC66A16EE101AB9427A
:10EF6800BFF62AAC39462AE4BDEEC66A16EE101A78
:10EF7800B942BFF6FDAB3946FFF7FDBBBDEEC66A29
:10EF880016EE101AB942BFF6CFAB3946FFF7CFBB22
:10EF9800BDEEC66A16EE101AB942BFF6A1AB3946E5
:10EFA800FFF7A1BBBDEEC66A16EE101AB942BFF64E
:10EFB80073AB3946FFF773BBBDEEC66A16EE101A7F
:10EFC800B942BFF645AB3946FFF745BB9FED9E7A80
:10EFD800F4EEC76AF1EE10FA44BF9FED9C7A77EE23
:10EFE800666A3EE74046FFF738B914EE901AFFF715
:10EFF8000DBB23F0A5FCFBF78DBB137C022B7EF425
:10F0080019AD92F8FE31552B7EF414AD92F8FF310C
:10F01800AA2B7EF40FADD689E7598D4B37441F6074
:10F0280092F80DE041F210210EF1FF337F2B44F8E6
:10F0380001E03EF6FFACCEF100033EEA03037EF4A6
:10F04800F9AC4FEA4E2341F21821013B6350D08AB4
:10F0580000B9506A7F4941F20423E050B2F81130F8
:10F068005B0103F2FF135B120B60B2F8131001B9D6
:10F07800116A40001E440644891B41F2082C40F6E0
:10F08800F476B1FBFEF1B14244F80C1040F2358140
:10F098004FF6F476B14240F2D18003212170D26A52
:10F0A8006D493B44184441F20C2641F21C2309786F
:10F0B800A051E25009B924F06BFEA3780133A37084
:10F0C800FCF71BBC02287CF418AC41F2B4120123F3
:10F0D800A3546370FCF711BC21F0D0FF2369FEF73D
:10F0E800B2BB94F87831002B7BF4B0ADFBF79BBD35
:10F0F800F0EE476AA9E6F0EE477A00E4B0EE677AE8
:10F10800FFF7E7BBB0EE667A89E6132B05D1B0EEC0
:10F11800480A24F0AFFF069B1880B0EE480ADBF8D7
:10F1280008324E489847029B1B78132BB0EE408A52
:10F138007DF4EDA824F09EFF069B5880FDF7E7B804
:10F14800089B002B7FF4E8AC059B079FBB42B8BF28
:10F15800B0EE646AE0E4089B002B7FF42DAC059BBD
:10F1680007988342B8BFB0EE646A25E4089B002B79
:10F178007FF4F5AC059B079FBB42B8BFB0EE646A4D
:10F18800EDE4DFED377AB4EEE7EAF1EE10FA26DCCB
:10F19800DFED347AB4EEE7EAF1EE10FA1FD4324B21
:10F1A800D3ED007AB1EE677AF4EEC7DAF1EE10FA31
:10F1B80012D4F4EEE7DAF1EE10FA88BFF0EE67DA6F
:10F1C8002A4B87ED00CA1B689342BBF697ABFBF747
:10F1D800FBBBF0EE476A90E6F0EE47DAF0E7DFEDCA
:10F1E80024DAEDE7089B002B7FF40AAC059B079F08
:10F1F800BB42B8BFB0EE646A02E4089B002B7FF400
:10F2080068AC059B079FBB42B8BFB0EE646A60E478
:10F21800089B002B7FF43AAC059B079FBB42B8BF05
:10F22800B0EE646A32E4089B002B7FF40CAC059BBB
:10F23800079FBB42B8BFB0EE646A04E402222270A2
:10F2480000222DE714210020DB0FC9BFDB0F49C0C6
:10F25800B86D0020D86D0020986D0020884F0020E0
:10F2680000C0F84400C0F8C4447100202871002090
:10F2780000000000244A254B10681B689847244B5F
:10F28800D7ED006A93ED007A224BD3ED007A224B3A
:10F2980083ED020A214B67EE277A2B4427EEAC7ADE
:10F2A800D3ED007A1E4B67EE277AF0EE665AEDEE44
:10F2B800A75A93ED006AB1EE467AB4EEE57AF1EE1C
:10F2C80010FA08DCF4EEC65AF1EE10FA8CBFB0EE74
:10F2D800467AB0EE657A134B1B78012B02D0192BB6
:10F2E8007BF41EACDFED107AF4EEE7DAF1EE10FAFB
:10F2F800CCBF01230023FBF71EBC01232370FEF7BC
:10F3080099BBB0EE667AE2E5BC700020D0700020B0
:10F31800107000200400002080390020E0700020D8
:10F3280048710020746F0020000096422DE9F047D4
:10F33800B0F908400C81E4B2442C8CB00D46174655
:10F3480000F0018406462FD9812C00F04C8300F28E
:10F358008180542C00F0AE8040F2B8806E2C00F012
:10F36800C083802C40F0B480654B1C780B3C14F0B3
:10F37800FF0412D0634F00220A2629683B88481CE4
:10F3880028600E702968FF2B02F10102A8BFFF2335
:10F39800481CA24228600B70EFDB0124234620465C
:10F3A8006B810CB0BDE8F087052C00F0BA831ED83D
:10F3B800022C77D040F2FA82032C00F08983042CC7
:10F3C80040F08680504928462246F5F743FF002141
:10F3D8002846F5F76DFF2A680021531C01242B608D
:10F3E8002046234611706B810CB0BDE8F087242CB1
:10F3F80056D040F29182282C00F02F83382C67D108
:10F408000A68424B0124511C296014702A6805219E
:10F418001019286011702A680A21101928601170C3
:10F428002A6800211019286011702A6819781019A3
:10F43800286011702A6859781019286011702A6894
:10F44800997813192B602346117020466B810CB0F4
:10F45800BDE8F087A02C11D040F27D82B82C00F0D6
:10F468003583FE2C34D12A4C04F1080634F8021BEB
:10F478002846F5F71DFFA642F8D18EE7254B08462A
:10F488001968F5F7FEFE244B28461968F5F7F9FECA
:10F49800224B196828460124F5F7F3FE23467EE738
:10F4A8001F4BF6E704221F4928460124F5F7D2FE30
:10F4B8002346CAE70B6800215A1C2A6019702A687B
:10F4C800012413192B6023461170BEE7522C82D0F9
:10F4D8002946204601F076FC014600287FF45DAFFE
:10F4E800742C00F07682772C20D1336872689A42A7
:10F4F80040F035830C4A284623F0D2FB4DE700BF85
:10F5080082460020682600208A4900208552002073
:10F51800D8460020ACF7FF1FB0F7FF1FB4F7FF1F56
:10F52800EC530020A47C030815290308F52C00F0EF
:10F538003F83292C376801F0E981392C01F0D68105
:10F54800212C01F0918172680B3CD31BEF2C00F247
:10F55800228401A050F824F0110301089FFD00083F
:10F568009FFD00089FFD00089FFD00089FFD000803
:10F578009FFD00089FFD00089FFD00089FFD0008F3
:10F588009FFD00089FFD00089FFD00089FFD0008E3
:10F598009FFD00089FFD00089FFD00089FFD0008D3
:10F5A8009FFD00089FFD00089FFD00089FFD0008C3
:10F5B8009FFD00089FFD0008A10201089FFD0008AB
:10F5C800310201089FFD00080F0201089FFD000895
:10F5D8009FFD00089FFD0008150401089FFD000815
:10F5E8009F0301089FFD00086D0301089FFD0008A7
:10F5F800470301089FFD0008FD0101089FFD000861
:10F60800A90101089FFD00080D0101089FFD0008E0
:10F618009FFD00089FFD00089FFD0008A3F3000858
:10F628009FFD0008E10001089FFD00089FFD0008FC
:10F63800DF0601089FFD0008850601089FFD0008F8
:10F648009FFD00089FFD00089FFD00089FFD000822
:10F658009FFD00089FFD00089FFD0008F9060108AE
:10F668009FFD0008370601089FFD00089FFD000860
:10F67800F90501089FFD00089FFD00089FFD00088F
:10F688009FFD00089FFD00089FFD00089FFD0008E2
:10F69800950501089FFD0008E70401089FFD000883
:10F6A8003D0401089FFD0008C50701089FFD0008EB
:10F6B8009D07010855070108390701089FFD000843
:10F6C8009FFD00089FFD00089FFD00089FFD0008A2
:10F6D8009FFD00089FFD00089FFD00089FFD000892
:10F6E8009FFD00089FFD00089FFD00089FFD000882
:10F6F8009FFD00089FFD00089FFD00089FFD000872
:10F708009FFD00089FFD00089FFD00089FFD000861
:10F718009FFD00089FFD00089FFD00089FFD000851
:10F728009FFD00089FFD00089FFD00089FFD000841
:10F738009FFD00089FFD00089FFD00089FFD000831
:10F748009FFD00089FFD00089FFD00089FFD000821
:10F758009FFD00089FFD00089FFD00089FFD000811
:10F768009FFD00089FFD00089FFD00089FFD000801
:10F778009FFD00089FFD00089FFD00089FFD0008F1
:10F788009FFD00089FFD00089FFD00089FFD0008E1
:10F798009FFD00089FFD00089FFD00089FFD0008D1
:10F7A8009FFD00089FFD00089FFD00089FFD0008C1
:10F7B8009FFD00089FFD00089FFD00089FFD0008B1
:10F7C8009FFD00089FFD00089FFD00089FFD0008A1
:10F7D8009FFD00089FFD00089FFD00089FFD000891
:10F7E8009FFD00089FFD00089FFD00089FFD000881
:10F7F8009FFD00089FFD00089FFD00089FFD000871
:10F808009FFD00089FFD0008730701089FFD000881
:10F81800CB000108A10001089FFD00089FFD00081A
:10F828009FFD00089FFD00089FFD00089FFD000840
:10F838009FFD00089FFD00089FFD00089FFD000830
:10F848009FFD00089FFD00089FFD00084500010876
:10F858009FFD000881FF00089FFD0008E5FE0008E5
:10F868008FFE000873FE00089FFD000859FE00087F
:10F878009FFD000831FE00089FFD0008D7FD000825
:10F888009FFD0008A9FD00089FFD00089FFD0008D6
:10F8980023000108F5FF0008E1FF0008B9FF000890
:10F8A80081FD00085FFD00089FFD00089FFD00081E
:10F8B8009FFD00089FFD00089FFD00089FFD0008B0
:10F8C8009FFD00089FFD00089FFD00089FFD0008A0
:10F8D8009FFD00089FFD00089FFD00089FFD000890
:10F8E8009FFD00089FFD000845FD00089FFD0008DA
:10F8F8009FFD0008EDFC00089FFD00089FFD000823
:10F908009FFD000887FC00089FFD00089FFD000878
:10F918009FFD00086DFC0008202C7FF4D9AD0B6812
:10F92800914C591C627829601A702B682278591CEE
:10F9380029601A702B68A278591C29601A702189CD
:10F948002846F5F7B5FC2B686279591C29601A70AE
:10F958002A68A17941E5822C7FF4BAAD0B68834A05
:10F96800834C1178804A581C2860197011892846E0
:10F97800F5F79EFC7F4B2A681B88FF2B02F10101DB
:10F98800A8BFFF2329601370A16881F3100189B211
:10F998002846F5F78DFC216801F30F0189B2284646
:10F9A800F5F786FC744B2A68197816E5012C7FF464
:10F9B8008FAD0B680022591C29601A702B685A1CDD
:10F9C8002A601C702A682521531C2B60234611705D
:10F9D8003BE5336872689A4240F0BD80674A284622
:10F9E80023F05EF9D9E4664B1E780A3E16F0FF064E
:10F9F8003FF4D3AC634B644F1E4403F101080A2360
:10FA080014E0502B00F02C87002421462A68501C53
:10FA1800286028461370F5F74BFC21462846F5F771
:10FA280047FC46453FF4B9AC18F8013B0A2BE8D12E
:10FA3800564A9468116804EB84044FF6FF72640018
:10FA48009442A8BF14469142A8BF114624EAE47420
:10FA580021EAE171A4B289B2D8E70B68DFF84C81DA
:10FA68004B4E591C022229601A702B6806275A1C13
:10FA78002A601F702B680A22591C29601A702B688B
:10FA880001241A192A601C70B8F800102846F5F7E6
:10FA98000FFCB8F802102846F5F70AFC2B681A196B
:10FAA8002A601F702B685022191929601A702B6858
:10FAB8000022191929601A7031882846F5F7F8FBD1
:10FAC80071882846F5F7F4FB2346BEE4314BE0E4A1
:10FAD8000B685A1C0A601C700B685A1C0A601C7060
:10FAE80079E4244B0A681B88214CFF2BA8BFFF230D
:10FAF800511C29601370A16881F3100189B228464E
:10FB0800F5F7D6FB244B28461988F5F7D1FB216871
:10FB180001F30F0189B228460124F5F7C9FB2346F2
:10FB280093E40B221D492846F5F794FB08221C494B
:10FB38002846F5F78FFB012407221A492846F5F7CE
:10FB480089FB234681E4002A3FF427AC164B136057
:10FB58000124234679E45A1C326019783EE75A1C7E
:10FB680032601978C6E400BFB0480020F246002091
:10FB78002446002038460020373F0020212903086A
:10FB880082460020AC5403085C260020242600206E
:10FB980058260020E82F0020343F0020AC7C0308C2
:10FBA800B87C0308C47C0308050B010864370020EF
:10FBB800336872689A4240F0C386B94BFF221A70C4
:10FBC8004FF00009B74C13F045F849462022B648D3
:10FBD80084F8009025F009FA8DF80C909DF80C3007
:10FBE800072B00F2E686DFF8E882AF4E4A469DF81A
:10FBF8000C3003EB430308EBC3035B7CDBB19DF8DC
:10FC08000C3003EB430308EBC3035B699BB19DF81E
:10FC18000C3003EB430308EBC303586946F8220092
:10FC280019F098F9237856F82300F4F73BF922786D
:10FC38000132D2B222709DF80C300133DBB28DF85C
:10FC48000C309DF80C30072BD1D92B68591C296032
:10FC58001A70002F3FF4A1AB944B3B60012423465C
:10FC6800FFF7F3BB924B1B78DB0700F1948001246C
:10FC7800F6F7D8F8F6F7B2FA2346FFF7E6BB3046B0
:10FC8800F5F7D8FA3368ADF80C001A46591C3160FC
:10FC980012F8021B32608DF80E105A788DF80F207A
:10FCA800DA1C32609A788DF810201A1D3260DA78E2
:10FCB8008DF811205A1D32601B798DF8123003A877
:10FCC8000023ADF81430F5F70FFA7A4A744B12682E
:10FCD800801A4FF0010461F10001C3E904012346D1
:10FCE800FFF7B3BB7B1C33603B780F2B53D8BA1C90
:10FCF8003260C3EBC303704A7978D154F91C316080
:10FD08001344BA785A703A1D3260FA789A707A1D9C
:10FD180032603A79DA70BA1D32607A791A71FA1D4E
:10FD28003260BA795A7107F108023260FA799A7129
:10FD380001241DF063F82346FFF787BB3046F5F72B
:10FD480079FA5E4FF8813046F5F774FA0124B881E4
:10FD58002346FFF77ABB3046F5F76CFA584F3882DE
:10FD68003046F5F767FA78823046F5F763FA0124EA
:10FD7800B8822346FFF769BB3B467A1C326013F80A
:10FD8800020B3360FB1C79783360BA780FF0F2FC11
:10FD980000287FF402AB4FF0FF342346FFF755BB32
:10FDA800DFF8308198F80030002B3FF4F6AA454F71
:10FDB80000243046F5F73EFA14F042FE98F8003079
:10FDC800A7EC010A01349C42F3DBFFF7E6BA0D2BDE
:10FDD800E1D17B1C33603C78072CDCD8DFF8F88055
:10FDE80030460C27F5F726FA07FB04F708EB07045B
:10FDF800A0803046F5F71EFAE0803046F5F71AFA8B
:10FE0800336820811A46591C316012F8021BA1720E
:10FE180032605B78E3723046F5F7F5F9012448F86B
:10FE280007002346FFF711BB7B1C336038780606B2
:10FE380000F1EF851E4B1B78DC073FF5AEAA0328BF
:10FE480028BF00200124F5F7D1FF2346FFF7FDBAAC
:10FE5800174B1B78D8073FF5A0AA0124F6F7B0FD89
:10FE6800F6F7BCF92346FFF7F0BA114B1B78DA070F
:10FE78003FF593AA144A1378012443F0040313703E
:10FE88002346FFF7E2BA0A4B1B78D9073FF585AA44
:10FE98000E4B4FF4C87201241A802346FFF7D5BAD7
:10FEA800302300206F72002030720020C50903083B
:10FEB800BF5500209C550020FC2E002074370020E0
:10FEC80020580020102D0020F8390020F64C002082
:10FED80060570020824600203C2E0020092B7FF727
:10FEE8005AAFDFF8AC833B467A1CD8F80040326042
:10FEF80013F8022B227033607B78A370FB1C3360ED
:10FF0800BB78642BA8BF64233A1D63713260FB7809
:10FF1800642BA8BF64237A1DA37132603B79E37117
:10FF2800BB1D33607B79642BA8BF6423FA1D237241
:10FF38003260BB79E37007F108033360FB79237102
:10FF48003046F5F777F9726833686081D11A00296D
:10FF58000CDD591CD8F800003160521A002A1978B3
:10FF6800417203DD9A1C32605B784370012415F0FE
:10FF7800B9FB2346FFF769BAB24B1868FB1C024667
:10FF88002137991E316013F8031C1170591E316016
:10FF980013F8021C5170336013F8011C917003337D
:10FFA800BB4202F10302ECD11DF054FBFFF7F5B997
:10FFB8003B467A1C3260A44A13F8021B1170336066
:10FFC800A24A7B789370FB1C3360A14BBA789A7075
:10FFD80001242346FFF739BA9A4B9E4918684E22E6
:10FFE800012423F007FF2346FFF72FBA3A467B1C6C
:08FFF8003360994B12F8021B63
:020000040801F1
:10000000197032607A785A70FA1C3260BA789A7035
:100010003046F5F713F9934B0124D8802346FFF7B8
:1000200018BA3046F5F70AF98E4F38803046F5F7A2
:1000300005F978803046F5F701F90124B8802346A8
:10004000FFF707BAC3F34704122C3FF6A8AEBCB1C2
:100050000CAB0DF10A0803EB44094746A9F1260948
:100060003046F5F7EBF827F8020FB945F8D17E4B8B
:1000700038F8022F23F8022FB845F9D1112C09D8EE
:100080007A4A6300023B13440021223223F8021F04
:100090009342FBD1764A01231C461370FFF7D9B96E
:1000A0007B1C744933600A783B78002A40F0C08496
:1000B00004220A70704A9B001380F7F79DF96F4B7A
:1000C000012498612346FFF7C4B96D4F00233046E1
:1000D0003B60F5F79CF8012438602346FFF7B9B977
:1000E0003B46791C3160674913F8020B8870336016
:1000F0007878487093423FF454A9FB1C33605F4BFF
:10010000BA781A7201242346FFF7A3B90722B3FB7A
:10011000F2F2C2EBC2041B1B7FF441AED2B202F179
:10012000FF395FFA89F9002A3FF43BA9DFF86CA197
:1001300009F101091C462DE09AF90A209A4200F0C3
:100140003F849AF912209A427FF429AE02270AEBE3
:10015000C708304688F80230F5F770F833682AF897
:1001600037001A46591C316012F8021B88F8031038
:1001700032605A7888F80420DA1C32609A7888F85D
:1001800006201F1D37600134DB7888F80530A14553
:100190003FF407A97B1C336097F900309AF90220DD
:1001A0009A42C9D10027D2E77B1C33603B780E2BE3
:1001B0003FF6F5ADBA1C3260787803283FF6EFAD14
:1001C0003149062202FB03F28B18FC1C5871346083
:1001D000B87888543A1D3260FA785A707A1D3260C5
:1001E0003A799A70BA1D32607A79DA70FA1D326003
:1001F000BA791A7101242346FFF72BB97B1C3360AF
:10020000224B3A785A7501242346FFF722B930462B
:10021000F5F714F81E4F38603046F5F70FF87860A0
:100220003046F5F70BF80124B8602346FFF711B903
:10023000184F00233B603046F4F7E9FF3B68012488
:1002400003433B602346FFF704B900BF1849002071
:10025000684D00207437002084370020C86E0308E2
:100260006C370020BC4C00209A3200209C320020C9
:10027000C032002012390020343F002030230020FB
:10028000E82F002094370020F42F0020204D00207C
:10029000702C0020EC5300201C4900204C4D002005
:1002A0007B1C33603C780191132C3FF678ADBB1C6E
:1002B0003360787822F032FD00283FF470ADAA4B0D
:1002C000027803F82420FA1C326003EB8404BA7825
:1002D00062703A1D3260FA78A2707A1D32603A7903
:1002E000E27003F15000019902E00433834207D029
:1002F0001A78002AF9D19C78DA789442F5D2012153
:100300009A4B81F00101012419702346FFF7A1B82F
:100310009749102B4FF0000228BF10230A604A6053
:100320008A60CA600A74002B3FF43BA83268013926
:1003300013440132326012F8010C01F8010F9A42A5
:10034000F7D1FFF72EB87A1C32603C781F2C3FF6AD
:1003500026AD052B7FF423AD3046F4F758FF854BCF
:1003600043F824000FF07CFAFFF71BB8814C04F12E
:1003700040073046F4F762FF3368A4F88000591C48
:100380001A46316012F8021B84F8821032605B78E2
:1003900084F883300434A742EBD1FFF702B87B1C0A
:1003A000754C33603B7823723046F4F747FFA083E7
:1003B0003046F4F743FF20833046F4F73FFF3268BE
:1003C0006083531C33601278E2747268D31A032B73
:1003D00000F304833368D11A05290EDD5A1C3260FC
:1003E0001B78E3723046F4F712FF3368E0605A1C62
:1003F00032601B78237433687268D21A002A7EF741
:10040000D0AF5A1C32601B7884F821300124234677
:10041000FFF71FB87B1C3360584938780870D21A30
:10042000002A7EF7BEAFBB1C33607B78003318BF59
:10043000012301244B702346FFF70BB87B1C33606C
:100440004F4CDFF84C813B7888F805303046276800
:10045000F4F7F4FE388430462768F4F7EFFE72684C
:100460003368F883D11A072915DD3046F4F7E6FE24
:10047000A8F80A003046F4F7E1FEA8F80C00304670
:100480002768F4F7DBFE788430462768F4F7D6FE59
:1004900033687268B884D11A03290BDD3046F4F74B
:1004A000CDFEA8F80E003046F4F7C8FE3368726837
:1004B000A8F81000D21A002A05DD591C2268316004
:1004C0001B7882F82630F5F7EFFD16F03FF82D4B3C
:1004D0001B68002B00F07782206801241CF026FDA9
:1004E0002346FEF7B6BF3B467A1C3260DFF8A08099
:1004F00013F8022B88F802203360234A7B781370AC
:10050000FB1C3360214CBB7823713B1D3360FB78AF
:10051000092BA8BF09233046A370F4F78FFE336878
:1005200072682080D11A012905DD3046F4F786FE75
:1005300033687268E0819A4207D05A1C32601B7897
:10054000003318BF012388F80730F5F7ADFD336895
:1005500072689A423EF425AF5A1C32601B78E370F1
:1005600001242346FEF775BF2834002074060020BE
:1005700050370020B03D0020204D0020EC390020F5
:1005800018490020D4390020683700202058002066
:10059000684D0020C64B1B68002B3EF402AF11F0E3
:1005A000FDFCFF283EF4FDAE3046F4F747FE3F2841
:1005B00040F25982BF4F00243C7033687268B880A3
:1005C000D21A012A7EF7EDAE1A46591C316012F894
:1005D000021BB9700CA8326000225C7800F8242D50
:1005E00011F0AEFC9DF80C30A3423EF4DAAE20468A
:1005F00011F0CAFCFEF7D5BEAF4B1B78012B3EF6BF
:10060000D0AE7B1C39463360DFF8E08211F8023B44
:1006100088F80230FB1CD21A3160012A78783360E6
:1006200040F314823046F4F709FE0124A8F80000D4
:100630002346FEF70EBF7B1C336097F80080B8F1AD
:10064000110F3FF6ACABBB1C33609C4C7B7804F8BD
:1006500018303046F4F7F2FD40F6CA039842A8BFBE
:10066000184640F2EE23984204EB4801B8BF184602
:100670000124A0F2EE222346192092FBF0F24A70E8
:10068000FEF7E7BE7B1C33608D4B3A78DFF8608263
:100690001A700023C8F800303046F4F7B8FD32680D
:1006A000D8F800308749884C0343501CC8F8003004
:1006B000306013780B723046F4F7C0FD206030468E
:1006C000F4F7BCFD60603046F4F7B8FDA06030463A
:1006D000F4F7B4FD3046F4F7B1FDFEF762BE7B4B94
:1006E00007F108010137376017F8012C03F8012FD3
:1006F000B942F7D1FEF755BE3B467A1C744C3260C6
:1007000013F8022B227133607B7863713046F4F763
:1007100095FD336820805A1C32601B78A3713046E7
:10072000F4F78CFD336860805A1C32601B78E371EB
:1007300001242346FEF78DBE7B1C33603B78002BE3
:1007400000F07B814FF40040012401F069FB234657
:10075000FEF77FBE5F4B1B7813F001017FF41FABE8
:100760007B1C33603878012413F06AFB2346FEF7C4
:1007700070BE3B467A1C326013F8024B3360FB1CA0
:1007800078783360B978002C00F07A81012C7EF4FF
:1007900008AE13F011FC2346FEF75BBE3B467A1C05
:1007A00032604D4A13F8021BD17033604B4A7B789C
:1007B0005371FB1C33604A4BBA78DA70012423462C
:1007C000FEF747BE3046F4F739FD3046F4F736FD04
:1007D0003046F4F733FD3046F4F73BFD3368414CC7
:1007E0001946581C2268306011F8020B82F82C0060
:1007F0003160597882F83610D91C31609B7882F8C4
:1008000037303046F4F725FD3046F4F722FD304608
:10081000F4F71FFD30462768F4F710FD788730465F
:100820002768F4F70BFD336872683887D11A0129FD
:100830000ADD591C226831601B7882F82E30304660
:10084000F4F707FD33687268D31A032B09DD3046CD
:100850002768F4F7F3FC788630462668F4F7EEFC58
:10086000B0862068FFF7A4BBBC683968FFF7E7B81B
:100870003B467A1C32601C4C13F8022B62703360CA
:100880007B782370FB1C3360BB78A3703046F4F791
:10089000D5FC33682081591C1A46316012F8021BBE
:1008A000617132605B78A37101242346FEF7D1BDEC
:1008B000C4550020C8550020B85300203C35002006
:1008C000EC390020204D0020702C00201F4D00200E
:1008D000D44C0020BF550020743700202445002050
:1008E0008437002018490020B0480020BA53002067
:1008F000EC5300207B1C33603B780A2B4CD03046F5
:10090000F4F7A7FC3046F4F7A4FC3046F4F7A1FC5A
:10091000FEF747BD7B1C33603B780A2B0FD0502B72
:100920007FF4D5AE3046F4F789FC584F3880304616
:10093000F4F784FC012478802346FEF78ABD304614
:10094000F4F77CFC524FF1E75A1C194632605148CB
:1009500011F8022B027031605B784370042A04D9CD
:10096000FF2A7EF43CADFFF72FB94B490978994235
:1009700005D8022A7EF433ADFF2B7EF430AD2B6810
:1009800001241A192A601C70002F3EF40AAD434B53
:100990003B602346FEF75DBDBB1C3360404B7A785D
:1009A0001A70FA1C3260BA785A703A1D3260FA78BE
:1009B0009A7001242346FEF74CBD4A46FFF749B919
:1009C0000127FFF7C4BB37483749384A384B036023
:1009D00001240B6013602346FEF73BBD3046F4F75D
:1009E0002DFCA0843046F4F729FC33687268E0845B
:1009F000D11A03297FF7EFAC1A46591C316012F85F
:100A0000021BA17732605B7884F820303046F4F71F
:100A100015FC336872686084DDE400F07F00032811
:100A200028BF0020012413F0E3FA2346FEF711BD8E
:100A3000042A7EF4B6ACFFF73DBB1E4A13680124BE
:100A400023F4004313602346FEF703BD1A4BB97825
:100A50001A88012412FB00F2234692FBF1F2A8F857
:100A60000020FEF7F6BCC40800F007030134013390
:100A7000E4B2124F204619467B700FF03BFD9BE518
:100A800001241CF076FC2346FEF7E3BC5826002028
:100A90006437002030230020824600201D0B01080F
:100AA000855200201470002068700020D070002053
:100AB000EB29000810490020BA350020C855002055
:100AC0000C4B1B78DB0700D570470B490B68002BDC
:100AD000FAD04FF47A7202FB03F39842F4D3074B37
:100AE0001B781BB9064B9A681B69136000230B60C7
:100AF000704700BFBF550020BC4B0020B04B00200A
:100B00009C4B002008B514F021F8024B024ADA6031
:100B1000FEE700BF00ED00E00400FA05024A034BC7
:100B20001278197811F056BA3023002031230020B2
:100B30009F4B1B7803B170472DE9F0439D4D2B6807
:100B40008BB013B90BB0BDE8F0839B4E9B4A337852
:100B5000044601A8D75C0FF099FC736803F5C33312
:100B6000A0339C4205D9032F68D8DFE807F0485C22
:100B70003F10934B1B78DB07E4D42B68002BE1D0AC
:100B80001B681B68002BDDD020469847DAE704AFCE
:100B900038460FF07BFC97E8070007AB03C39DF8CE
:100BA00010101A80002974D108A811F0BDF90DF1B8
:100BB0001E0011F0D1F938460A2207A924F0F0F9F5
:100BC0007F4B1A78071C18BF012702F001027D49EC
:100BD000337808787460013393FBF0F100FB113334
:100BE0003370002AC9D0002FC7D1ABE7DFF8D0811E
:100BF00098F8002012F0010251D00027E7E79DF895
:100C00000430DFF8BC8143B398F80030D9075CD5D5
:100C10006C4A337811787460013393FBF1F201FB75
:100C2000123333708EE704A811F096F907460028B6
:100C300040D1634B1A7802F00102C8E7604A61496B
:100C400033780978107874600133C00793FBF1F2B0
:100C500001FB1233337090D574E798F80030DA074F
:100C6000D6D404A811F060F9002840F084805549DA
:100C70003378087898F800207460013302F001029C
:100C800093FBF0F100FB11333370002A3FF475AF92
:100C900058E70DF11D0107A811F06AF987E707A8C9
:100CA00011F04EF900284AD198F80020002702F0F0
:100CB00001028CE707A80FF0E9FB9DF81E009DF8E4
:100CC000103083422ED10027B3E704A90DF10300B1
:100CD00011F04EF90028CAD007A80FF0D7FB9DF8F5
:100CE0001C009DF803309DF81D10834203D19DF830
:100CF00010308B42BBD02B684BB11A79824206D39D
:100D00005A798A4203D31B68DB6803B198472D4A9E
:100D1000337811787460013393FBF1F201FB1233E5
:100D200033702AE72B68002B83D09A79824280D3D4
:100D30001B681B69002B3FF47CAF984779E727209D
:100D400014F070FC07460028AED01F4BDB88002B48
:100D5000AAD1272014F018FC9DF81C308146E8B178
:100D6000002BA1D1012011F00FF998F800204F4677
:100D700002F001022BE707A80FF088FBBDF8200066
:100D8000BDF8103083423FF472AF2B68002BBED009
:100D90001B689B69002BBAD09847B8E7002B83D01B
:100DA00011F0F2F898F8002002F001020FE700BFFE
:100DB0007F490020C455002058230020BD2C00206E
:100DC000BF550020C12C0020C85500202DE9F04F50
:100DD0002DED028BA0F10A0389B00C46ED2B00F239
:100DE0007A86DFE813F0220178067806780678061E
:100DF0007806780678067806780678067806780603
:100E000078067806780678067806780678067806F2
:100E10007806780678063402780678067806300672
:100E200078067806780699017806560178063E011C
:100E30007806330178062D02780608027806EF015D
:100E4000780678067806EA01E4017806D201780689
:100E50007806CC017806A5017806780678068E0417
:100E60007806780678067806700478060201780617
:100E70003F062D0578067806780678067806780607
:100E8000780601057806D3047806A004780669057B
:100E90007806640678067806780678060903F5056C
:100EA000EE05BD05EE00780678062C03AA0278064A
:100EB0007302ED027806780678067806E202780674
:100EC0007806C102780678067806B302F703BF03F6
:100ED0007E03780678067806700378067806500355
:100EE0007806780678067806780678067806780612
:100EF0007806780678067806780678067806090374
:100F000078067806780678067806780678067806F1
:100F100078067806780678067806780678067806E1
:100F200078067806780678067806780678067806D1
:100F300078067806780678067806780678067806C1
:100F400078067806780678064203780678067806EA
:100F500078067806780678067806780678067806A1
:100F60007806780678067806780678067806780691
:100F70007806780678067806780678067806780681
:100F80007806780678067806780678067806780671
:100F90007806780678067806780678067806780661
:100FA0007806780678067806780678067806780651
:100FB000780666043C047806780678067806780693
:100FC0000D04B24E337853B1B14F002537F8021FEC
:100FD0002046F4F771F933780135AB42F6DC012095
:100FE00009B0BDEC028BBDE8F08FA84E3378002B22
:100FF000F5D0A84F0025B846236817F81520591CCE
:1010000021601A7098F8011001EB810101EB810158
:1010100001F2EE2189B22046F4F74EF9337801351A
:10102000AB4208F10208E7DCD9E79B4D284621F0E6
:1010300013FF0028D3DD2B460544226813F8011B5B
:10104000501C9D4220601170F7D1C8E7934D05F107
:10105000800655F8041F2046F4F717F9AE42F8D180
:10106000BDE78F4D05F14006B5F880102046F4F736
:1010700023F9236895F88220591C21601A7023688F
:1010800095F883200435591CB54221601A70EBD1C4
:10109000A5E7844D0B682A7A591C21601A70A98B28
:1010A0002046F4F709F9298B2046F4F705F9698BF6
:1010B0002046F4F701F92368EA7C591C21601A7074
:1010C000A98C2046F4F7F8F8E98C2046F4F7F4F8F8
:1010D0002368AA7F591C21601A70236895F8202084
:1010E000591C21601A70698C2046F4F7E5F82368D2
:1010F000EA7A591C21601A70E9682046F4F7C5F8AD
:1011000023682A7C591C21601A70236895F82120D5
:10111000591C21601A7062E70B68634A581C1178E9
:101120002060197023685278591C21601A7056E7A4
:101130000B685D4A5D4D11785D4A581C206019703E
:1011400011682046F4F7A1F82368564A591C127A10
:1011500021601A7029882046F4F7AEF8A988204645
:10116000F4F7AAF829892046F4F7A6F820460021CA
:10117000F4F7A2F820460021F4F79EF82FE708467E
:1011800008224849F4F76AF829E70B68494A4A49AE
:1011900090785D1C2560187023685278581C206078
:1011A0001A7023680A79591C21601A7017E70B68B6
:1011B0000122991821601A7011E708460021F4F7FE
:1011C00064F80CE73D4D3E4E05F1180795F90230E5
:1011D00096F906209A4200F04B8596F90E209A4225
:1011E00000F0468596F916209A4200F041850835B0
:1011F000BD42EBD1F3E6334B03F15A05226859792E
:10120000501C2060117022681978501C20601170E9
:1012100022685978501C2060117022689978501CFF
:10122000206011702268D978501C206011702268EB
:1012300019790633501C9D4220601170DED1CEE634
:101240000B68184A591C527D21601A70C7E61E4D62
:1012500005F15006287821F07BFD2368027A591C9D
:1012600021601A7023686A78591C21601A702368FB
:10127000AA78591C21601A702368EA780435591C31
:10128000B54221601A70E5D1A9E600BF204A0020CE
:10129000947E00203C35002050370020AC3D0020DB
:1012A000B03D0020204D0020EC390020702C0020A3
:1012B000EC53002094370020342300204C4D0020B4
:1012C000705B0020F42F002028340020AF4D0B6805
:1012D0002A68591C127821601A702B682268997844
:1012E000531C2360002311702A6821681A440133BB
:1012F0005279481C032B20600A70F5D123682A68B4
:10130000591C127A21601A7023682A68591CD278F5
:1013100021601A7023682A68591C127921601A709A
:101320002B6820465989F3F7C7FF2A682368527A49
:10133000591C21601A702A68F4E620460021F3F750
:10134000A4FF20460021F3F7B7FF48E6904D08467A
:101350002988F3F7B1FF69882046F3F7ADFFA98824
:101360002046F3F7A9FF3AE68A4D05F16006A98801
:101370002046F3F7A1FFE9882046F3F79DFF29896E
:101380002046F3F799FF2368AA7A591C21601A7046
:101390002368EA7A591C21601A7055F80C1B204604
:1013A000F3F773FFB542E2D119E67B495223226875
:1013B000501C2060137011F8013F002BF7D10EE68E
:1013C000764800232268056803EB4301561C6D5CD8
:1013D00026601570026825680A446E1C52782660E3
:1013E0002A70026825680A4401339278691C0A2B26
:1013F00021602A70E6D1F2E500258146DFF8C88138
:10140000DFF8C8B1049503950595069501214FF6BF
:10141000FF7A05E001350B2D00F0608318F9011FFC
:101420004F1C4AFA05F3F5D0DE07F3D5BBF80030C0
:101430002B41D807EED505A8F4F70AFAEAE7584D8C
:1014400008462988F3F738FF69882046F3F734FF08
:10145000B5F90430534AD91782FB0323C1EBA3012A
:10146000204689B2F3F728FFB9E50B684E4A591CAC
:101470001278216005A81A70F3F714FE23685A1C2D
:1014800022601870ABE50B68484F591C3A78216010
:101490001A703B78002B3FF4A2AD0025EEB2304627
:1014A0000FF054F823684278591C216030461A70B6
:1014B0000FF04CF801892046F3F7FEFE3B7801352A
:1014C000AB42EBDC8BE53A4D0846298AF3F7F4FE94
:1014D000698A2046F3F7F0FEA98A2046F3F7ECFE6E
:1014E0007DE5DFF8ECE00027FEB2714600232268BC
:1014F000501C206016702268501C206013702268F7
:1015000011F8010F0133551C062B25601070EED128
:101510000137062F0EF1060EE6D126490023226878
:10152000501C206017702268501C206013702268C5
:1015300011F8010F0133551C0B2B25601070EED1F3
:1015400023681D4A581C0721206019702368002158
:10155000581C20601970236892F8F020591C2160F3
:101560001A703CE50B68154A15491078154A5D1C40
:101570002560187023688978581C206019702368CA
:101580009278591C21601A7029E500BF1C4900207F
:10159000BC4C00203C2E0020B05403081849002009
:1015A000C448002067666666123900208246002023
:1015B00020580020933E0020B03D0020684D0020C0
:1015C0007437002084370020E054030814490020B9
:1015D0006F3E00200A68AC4BAC491878551C25605A
:1015E000107022685878551C2560107022689B780E
:1015F000501C206013702046C988F3F75DFEEEE4AE
:1016000005A8F3F74FFD00283FF4E9ACBDF814102E
:101610002046F3F751FE23689DF81620591C2160DF
:101620001A7023689DF81720591C21601A702368CE
:101630009DF81820591C21601A7023689DF8192004
:10164000591C21601A7023689DF81A20591C2160CA
:101650001A702046BDF81C10F3F72EFEBFE48C4B29
:1016600003F1700522681978501C206011702268FF
:101670005978501C2060117022689978501C2060A5
:1016800011702268D978501C206011702268197975
:10169000501C2060117022685979501C2060117014
:1016A000226899790733501C9D4220601170D9D16E
:1016B00095E4784D0846E989F3F7FEFDA9892046AF
:1016C000F3F7FAFD8BE40B68734D591C2A792160FE
:1016D0001A7023686A79591C21601A70298820467B
:1016E000F3F7EAFD2368AA79591C21601A7069880A
:1016F0002046F3F7E1FD2368EA79591C21601A704E
:101700006DE40B6800255A1C0A60204629461D70AE
:10171000F3F7BBFD29462046F3F7B7FD29462046DF
:10172000F3F7B3FD5BE45D4E0B6872795C4D591CB9
:1017300021601A702B682046198CF3F7BDFD2B68C9
:101740002046D98BF3F7B8FD71892046F3F7B4FD35
:10175000B1892046F3F7B0FD2B682046598CF3F78A
:10176000ABFD2B682046998CF3F7A6FDF189204646
:10177000F3F7A2FD318A2046F3F79EFD2A6823681D
:1017800092F82620591C21601A7028E4434EF37801
:10179000002B00F09A820B680822591C21601A70F5
:1017A00023680122991821601A7023683D4D591C45
:1017B0002A7921601A702368AA78591C21601A704E
:1017C00029882046F3F778FDE9892046F3F774FD70
:1017D0002368F279591C21601A702368EA78591C31
:1017E00021601A70FFF7FBBB10F0D8FBFF280546FD
:1017F00000F07C8208A8002300F80C3D10F0A0FB4C
:101800002268294B511C2160157022681978501CE0
:101810002060117022685978501C20601170226875
:101820009978501C2060117022689DF81410501C8B
:101830002060117020469988F3F73EFDFFF7CFBB7B
:101840000B681A4D591C012221601A702368AA786E
:10185000591C21601A7009F00BFF2368144A1549BE
:101860005E1C26601870B1F90010B2F90000F3F7A1
:101870009DFE23685A1C2260187029882046F3F7C1
:101880001BFDFFF7ACBB00BF6C370020BC4C002039
:10189000FC2E002074370020D44C0020684D00201E
:1018A0001849002020580020C8550020BA530020B5
:1018B000BA350020C035002020460021F3F7FCFC9B
:1018C00020460021F3F7F8FC20460021F3F7F4FC52
:1018D0002368A24D00265A1C22601E7023682A68C5
:1018E000591C92F82C2021601A7023682A68591C10
:1018F00092F8362021601A7023682A68591C92F8E1
:10190000372021601A7023685A1C22601E702368D9
:101910005A1C22601E7023685A1C22601E702B689D
:101920002046598FF3F7C8FC2B682046198FF3F730
:10193000C3FC23682A68591C92F82E2021601A7073
:1019400023685A1C22601E702B682046598EF3F7BC
:10195000B3FC2B682046998EF3F7AEFCFFF73FBB34
:101960007F4D804E9FED808ADFF84482DFED7F8AD5
:1019700005F120070EE0FCEEE77ACDED017ABDF827
:10198000041020460435F3F797FCBD4206F1180613
:101990003FF425AB717C0029F3D0754BD5ED007A6F
:1019A0001B78012BE7D1734B1B68DB0440F183816B
:1019B000F5EE407AF1EE10FA40F0AB8140F2DC51E6
:1019C000DFE7084610226C49F3F748FCFFF707BB36
:1019D0006A4B9B8AB3F5006F00F27581B3F5806F97
:1019E00000F29581B3F5007F34BF01270227644DD3
:1019F00005F10C0655F8041B91FBF7F1204689B25E
:101A0000F3F75AFCB542F5D15E4D5F4F05F10C0678
:101A1000B5EC010AD7ED077A80EE270A22F02EFBFB
:101A200081B22046F3F748FCAE42F1D1574D05F1A3
:101A30000C0655F8041B204689B2F3F73DFCAE4274
:101A4000F7D1FFF7CCBA524D08462988F3F734FC9A
:101A5000A9882046F3F730FC29892046F3F72CFCAF
:101A6000FFF7BDBA0A684B4D511C0123216013706A
:101A700095F824204849002A40F067812268501CCC
:101A800020601370236841F2B4105A1C085C226075
:101A900041F27812187089582046890AF3F7F5FB4D
:101AA000A96A20464908F3F7F0FBFFF798BA0B68DC
:101AB0003A4A3B49D0783B4A5D1C25601870236840
:101AC0004979581C206019702368D278591C21600C
:101AD0001A70FFF784BA0020FFF782BADFF8D4A0AB
:101AE00000254FF0A8080135C5F1200208FA02F2DE
:101AF000A5F120032AFA05F6164328FA03F31E433C
:101B0000282D06F001024FF000030BD01343EAD05A
:101B1000E8B213F087FD0028E5D0294605A8F3F7C1
:101B200097FEE0E7204B1B78DA0700F1DA8000250A
:101B30001E4E2F4602E00135282D3DD02946304665
:101B4000F3F795FE0028F6D0294605A8F3F78FFE97
:101B5000002840F0AB800137EDE700BF18490020B6
:101B6000B4390020605700200000404200E0824469
:101B70004458002004500020A4390020CC48002004
:101B8000FC480020F84F00207C4D0020104D002024
:101B9000702C0020B47D0020B85B0020743700203A
:101BA0002445002084370020BF550020747F00208A
:101BB000DB9B914190E33FF47A4B7B4DB3F850109F
:101BC0002046F3F779FB794B1988204689B2F3F761
:101BD00073FB774B19684B0103F02002C1F34003FC
:101BE0001343C1F3800243EA4203C1F3C00243EA54
:101BF0008203C1F3401243EAC20301F0100119430A
